:0400000007EF00F016
:100008007D8225ED52F0AFEF4CF065C0D9FF66C098
:10001800DAFFDE6ADD6A64C00AF008EC45F00AC05F
:1000280088F00BC089F0000189BF0B0CD890883587
:10003800D96E8935DA6E480ED926010EDA22DECF5E
:100048009FF0DDCFA0F09F51A01101E10C0C65C01D
:10005800D9FF66C0DAFF9FC0DEFFA0C0DDFF679052
:100068009FC0D9FFA0C0DAFFDF5012E020EE01F0F8
:100078009F51D926A051DA22DF502BEC60F0000105
:10008800946F94B105D06750D8A494A5000C0A0CBD
:100098009FC0D9FFA0C0DAFFDF6A20EE01F09F51B0
:1000A800D926A051DA2288C0DFFF20EE01F09F5147
:1000B800D926A051DA22DF504EEC42F00001946FAD
:1000C80094B1030C675002E094B50A0C9FC048F045
:1000D800A0C049F04B6A4A6AD1EC46F048C09DF08E
:1000E80049C09EF0040E00019D199E1101E1010C0A
:1000F8009E5103E1020E9D5D01E30D0C20EE2BF0F5
:100108009F51D926A051DA22DECF90F0DECF91F0B0
:10011800DECF92F0DECF93F03A0E9F250A6E000EE6
:10012800A0210B6E49EC5EF0020E0B180A1001E0DC
:100138000D0C450E00019F250A6E000EA0210B6EC6
:1001480049EC5EF00AC099F00BC09AF000019B6B75
:100158009C6B99519A119B119C1110E1530E9F258C
:100168000A6E000EA0210B6ED3EC52F00AC099F073
:100178000BC09AF00CC09BF00DC09CF0000120EE63
:1001880017F09F51D926A051DA2299C0DEFF9AC0F4
:10019800DEFF9BC0DEFF9CC0DEFF20EE3FF09F51DC
:1001A800D926A051DA2210EE02F09F51E126A05183
:1001B800E222DFCFE7FF20EE02F09F51D926A051BF
:1001C800DA22DE040AE020EE02F09F51D926A0517F
:1001D800DA22020EDE1801E00D0C99C00AF09AC06E
:1001E8000BF09BC00CF09CC00DF020EE02F09F516C
:1001F800D926A051DA22DF500E6E0F6A106A116AF2
:1002080032EC57F00AC099F00BC09AF00CC09BF082
:100218000DC09CF020EE3CF09F51D926A051DA2267
:10022800DF50686E696A20EE09F09F51D926A05107
:10023800DA2268C0DEFF69C0DDFF20EE09F09F51B9
:10024800D926A051DA22DE50DE10D8B40D0C20EEEB
:1002580009F09F51D926A051DA22DECF68F0DDCF10
:1002680069F020EE09F09F51D926A051DA22DECF9D
:100278006AF0DDCF6BF0FF0E6A246C6EFF0E6B2008
:100288006D6E68506C146E6E69506D146F6E6E10E2
:1002980001E00D0C400E9F250A6E000EA0210B6E8A
:1002A80049EC5EF0000120EE07F09F51D926A051DD
:1002B800DA220AC0DEFF0BC0DDFF20EE07F09F51F7
:1002C800D926A051DA22DF50686E0F0E681601E0B9
:1002D8000D0C420E9F250A6E000EA0210B6E49ECF4
:1002E8005EF00AC08CF00BC08DF000018E6B8F6B36
:1002F8008C518D118E118F1110E14F0E9F250A6EB2
:10030800000EA0210B6ED3EC52F00AC08CF00BC08B
:100318008DF00CC08EF00DC08FF03D0E00019F25B2
:100328000A6E000EA0210B6E49EC5EF00AC08AF03E
:100338000BC08BF000018A518B1101E10D0C20EEEE
:1003480007F09F51D926A051DA22DECF68F0DDCF21
:1003580069F0040E6A6ED890693268326A2EFBD74B
:100368008A5168246B6E8B5169206C6E6D6AD8B0A7
:100378006D2A6E6A99516B24846F9A516C20856F2F
:100388009B516D20866F9C516E20876F84518C5DC8
:1003980085518D5986518E5987518F5901E20D0C1F
:1003A80084518C5D0A6E85518D590B6E86518E591C
:1003B8000C6E87518F590D6E20EE09F09F51D9268A
:1003C800A051DA22DECF68F0DDCF69F068C00EF008
:1003D80069C00FF0106A116A70EC58F00AC095F005
:1003E8000BC096F00CC097F00DC098F00001955125
:1003F80096119711981101E10D0C9D6B9E6BF60EED
:10040800955DFF0E9659FF0E97590F0E985903E206
:100418009E6B030E9D6F9851971108E1F60E955D3E
:10042800FF0E965903E29E6B020E9D6F985197112D
:1004380008E1F60E955D0F0E965903E29E6B010ECC
:100448009D6F9D519E1101E10D0C020E9525686E60
:10045800000E9621696E000E97216A6E000E982193
:100468006B6E20EE13F09F51D926A051DA2268C096
:10047800DEFF69C0DEFF6AC0DEFF6BC0DEFF20EE74
:100488001BF09F51D926A051DA2290C0DEFF91C0FF
:10049800DEFF92C0DEFF93C0DEFF8A519025686EB2
:1004A8008B519121696E000E92216A6E000E932184
:1004B8006B6E20EE1FF09F51D926A051DA2268C03A
:1004C800DEFF69C0DEFF6AC0DEFF6BC0DEFF84515D
:1004D8009025686E85519121696E865192216A6EC8
:1004E800875193216B6E20EE27F09F51D926A0519A
:1004F800DA2268C0DEFF69C0DEFF6AC0DEFF6BC0BB
:10050800DEFF030E9D199E114DE1590E9F250A6EBF
:10051800000EA0210B6E49EC5EF00A500B1001E0B2
:100528000D0C000120EE07F09F51D926A051DA22C8
:10053800DE50DE1001E00D0C5B0E9F250A6E000EEA
:10054800A0210B6ED3EC52F0000120EE23F09F5156
:10055800D926A051DA220AC0DEFF0BC0DEFF0CC08C
:10056800DEFF0DC0DEFF20EE13F09F51D926A0510B
:10057800DA22DECF68F0DECF69F0DECF6AF0DECFB8
:100588006BF0020ED890683669366A366B36E82EFC
:10059800F9D768C080F069C081F06AC082F06BC08A
:1005A80083F0B8D020EE07F09F51D926A051DA2267
:1005B800DE50DE1001E10D0C20EE1FF09F51D92610
:1005C800A051DA22DECF68F0DECF69F0DECF6AF024
:1005D800DECF6BF0995168246C6E9A5169206D6E6C
:1005E8009B516A206E6E9C516B206F6E20EE23F03B
:1005F8009F51D926A051DA226CC0DEFF6DC0DEFF04
:100608006EC0DEFF6FC0DEFF020E9D199E116BE00B
:1006180020EE13F09F51D926A051DA22DECF68F0E0
:10062800DECF69F0DECF6AF0DECF6BF0010E681422
:100638006C6E6D6A6E6A6F6A20EE13F09F51D92650
:10064800A051DA22DECF70F0DECF71F0DECF72F08B
:10065800DECF73F0030E7002F3CF74F0F4CF75F0B1
:10066800766A776A7102F3507526F4507622000E86
:1006780077227002F3507526F4507622000E772206
:10068800030E7202F3507626F4507722000E7102A0
:10069800F3507626F4507722000E7002F350762637
:1006A800F4507722030E7302F3507726000E72027D
:1006B800F3507726000E7102F3507726000E700271
:1006C800F3507726D89077327632753274326C5080
:1006D8007424806F6D507520816F6E507620826F04
:1006E8006F50772016D020EE13F09F51D926A051D5
:1006F800DA22DECF68F0DECF69F0DECF6AF0DECF37
:100708006BF0D8906834806F6934816F6A34826F77
:100718006B34836FFF0E8025686E010E8121696E30
:10072800000E82216A6E000E83216B6E0A0E05D0C0
:10073800D8906B326A3269326832E82EF9D720EEE7
:1007480017F09F51D926A051DA226850DE5C695013
:10075800DE586A50DE586B50DE5801E20D0C20EE70
:100768000FF09F51D926A051DA22DE68DE68DE68D4
:10077800DD68DD52DD5210EE0BF09F51E126A051ED
:10078800E222DECFE6FFDECFE6FFDECFE6FFDECFFA
:10079800E6FF20EE04F09F51D926A051DA22800E00
:1007A800DF6E030E9D199E1101E090D05F0E9F250C
:1007B8000A6E000EA0210B6E49EC5EF00A040B10C5
:1007C80001E084D09FC036F0A0C037F0010E0001D0
:1007D8009025386E000E9121396E000E92213A6EE6
:1007E800000E93213B6E17EC54F000096FE10001F5
:1007F80020EE04F09F51D926A051DA22DF6A2D0E8F
:100808009F250A6E020EA0210B6E49EC5EF0550E74
:100818000A185CE1AA0E0B1859E12F0E00019F255A
:100828000A6E000EA0210B6ED3EC52F0520E0A187D
:100838004DE1520E0B184AE1610E0C1847E1410ECA
:100848000D1844E1130E00019F250A6E020EA02127
:100858000B6ED3EC52F0720E0A1838E1720E0B18B8
:1008680035E1410E0C1832E1610E0D182FE1170E1B
:1008780000019F250A6E020EA0210B6ED3EC52F0E8
:10088800000120EE0FF09F51D926A051DA220AC0AC
:10089800DEFF0BC0DEFF0CC0DEFF0DC0DEFF1B0E4F
:1008A8009F250A6E020EA0210B6ED3EC52F00001B8
:1008B80020EE0BF09F51D926A051DA220AC0DEFFA4
:1008C8000BC0DEFF0CC0DEFF0DC0DEFF9FC0D9FFEE
:1008D800A0C0DAFF9DC0DFFF0101464B472B000196
:1008E80020EE05F09F51D926A051DA2246C1DEFF3D
:1008F80047C1DDFF000C466E456A02D3090E461853
:1009080018E10001FF5115E0456A8990456A010E1A
:10091800786E79501E0D1B0EF324D96E020EF4204A
:10092800DA6E200EDF6E030E0101586F446B456BC3
:10093800899046500AE10001FF5107E0456A01012C
:10094800456B0A0EBAD0899053D3020E461808E1B7
:100958000001FF5105E0456A0101456B140EADD059
:100968001F0E466439D0300E466036D00001FF5164
:1009780033E04650E00F796E456A0F0E791805E1AD
:1009880057C178F00101576BB7D27950220D0A0E82
:10099800F324D96E030EF420DA6EDE50DE10DE107A
:1009A800DE1003E0030E7964A7D2796A010E786E2F
:1009B80079501E0D1B0EF324D96E020EF420DA6E48
:1009C80079501E0D1B0EF324E16E020EF420E26E28
:1009D800E7501009DF6E90D23F0E466429D0480ECA
:1009E800466026D00001FF5123E079501E0D000E0D
:1009F800F324D96E020EF420DA6E4650C00FDF6E73
:100A080079501E0D000EF324D96E020EF420DA6E12
:100A1800DF500CE079501E0D1B0EF324D96E020E28
:100A2800F420DA6E100EDF6E010E786E456A64D21D
:100A3800480E461809E10001FF5106E0456A120E0A
:100A48000101456FC00E39D0310E461808E100018A
:100A5800FF5105E00C0E0101456F1D0E36D2340E14
:100A6800461808E10001FF5105E00101446B456BA0
:100A7800456A69D7350E461809E10001FF5106E0BD
:100A8800456A0D0E0101456FAC0E17D0370E46189A
:100A980009E10001FF5106E089800E0E0101456F52
:100AA800750E13D20D0E46180AE10001FF5107E03A
:100AB800456A020E0101456FBC0E446F44D7100E03
:100AC800461808E10001FF5105E0030E0101456FDA
:100AD800E90EFBD1180E461808E10001FF5105E0A8
:100AE800070E0101456F090EF0D13B0E461808E1CB
:100AF8000001FF5105E00E0E0101456F7E0EE5D1A4
:100B08003E0E461801E074D20001FF5101E170D297
:100B18000F0E0101456F3D0ED8D179501E0D010E03
:100B2800F324D96E020EF420DA6E46C0DFFF030EFE
:100B38000101456FEA0EC9D179501E0D020EF3244A
:100B4800D96E020EF420DA6E46C0DFFF030E0101F3
:100B5800456FEB0EBAD179501E0D030EF324D96EF2
:100B6800020EF420DA6E46C0DFFF030E0101456F66
:100B7800EC0EABD179501E0D040EF324D96E020E83
:100B8800F420DA6E46C0DFFF030E0101456FED0E5B
:100B98009CD179501E0D050EF324D96E020EF42057
:100BA800DA6E46C0DFFF030E0101456FEE0E8DD1F0
:100BB80079501E0D060EF324D96E020EF420DA6E5B
:100BC80046C0DFFF79501E0D050EF324D96E020EC4
:100BD800F420DA6EDF50226E22C023F0246A256AE0
:100BE800266A25C026F024C025F023C024F0236AF5
:100BF80079501E0D040EF324D96E020EF420DA6E1D
:100C0800DF50276E27C028F0296A2A6A2B6A29C074
:100C18002BF028C02AF0296A286A79501E0D030E85
:100C2800F324D96E020EF420DA6EDF502C6E2CC03D
:100C38002DF02E6A2F6A306A2DC030F02F6A2E6A86
:100C48002D6A28502D24316E29502E20326E2A50BC
:100C58002F20336E2B503020346E23503124356EC4
:100C680024503220366E25503320376E26503420DB
:100C7800386E79501E0D060EF324D96E020EF4203C
:100C8800DA6EDF503524396E000E36203A6E000ECB
:100C980037203B6E000E38203C6E39C03DF03AC01C
:100CA8003EF03BC03FF03CC040F0416A40BE416866
:100CB80041C042F041C043F041C044F079501E0D9C
:100CC800070EF324D96E020EF420DA6E3DC0DEFF63
:100CD8003EC0DEFF3FC0DEFF40C0DEFF41C0DEFF9A
:100CE80042C0DEFF43C0DEFF44C0DEFF79501E0D68
:100CF8001C0EF324D96E020EF420DA6EDECF22F039
:100D0800DDCF23F022C00AF023C00BF00C6A0D6A75
:100D18000E6A0F6A106A116A79501E0D070EF324C5
:100D2800D96E020EF420DA6EDECF24F0DECF25F085
:100D3800DECF26F0DECF27F0DECF28F0DECF29F099
:100D4800DECF2AF0DECF2BF024C012F025C013F03E
:100D580026C014F027C015F028C016F029C017F0D7
:100D68002AC018F02BC019F063EC56F00AC02CF01A
:100D78000BC02DF00CC02EF00DC02FF00EC030F0BF
:100D88000FC031F010C032F011C033F079501E0D91
:100D9800070EF324D96E020EF420DA6E2CC0DEFFA3
:100DA8002DC0DEFF2EC0DEFF2FC0DEFF30C0DEFF0D
:100DB80031C0DEFF32C0DEFF33C0DEFF89900101A3
:100DC800446B456B15D179501E0D1A0EF324D96E5C
:100DD800020EF420DA6E46C0DFFF070E0101456FF0
:100DE8000A0E73D079501E0D190EF324D96E020E17
:100DF800F420DA6E46C0DFFF070E0101456F0B0EC7
:100E080064D079501E0D180EF324D96E020EF4200A
:100E1800DA6E46C0DFFF070E0101456F0C0E55D094
:100E280079501E0D170EF324D96E020EF420DA6ED7
:100E380046C0DFFF61D00101446B456B786A83D5FA
:100E480046C030F10F0E0101456F3E0E3ED046C040
:100E580031F10F0E0101456F3F0E37D046C032F118
:100E68000F0E0101456F400E30D046C033F10F0E12
:100E78000101456F410E29D046C034F10F0E010122
:100E8800456F420E22D046C035F10F0E0101456F65
:100E9800430E1BD046C036F10F0E0101456F440EBC
:100EA80014D046C037F128D00C0E0101456F1E0E34
:100EB8000CD00C0E0101456F1C0E446F0A0E456ED6
:100EC80042D50E0E0101456F760E446F91D0010197
:100ED800446B456B090E456E89808AD046500CE0FC
:100EE80079501E0D1B0EF324D96E020EF420DA6E13
:100EF800080EDF6E010E786E0101446B456B23D539
:100F080044C122F045C123F0235013E0030A15E041
:100F1800040A27E00B0A33E0010A37E0030A3BE042
:100F2800010A42E01D0A5AE00E0A5DE03B0A5EE053
:100F38005FD0225001E1E2D45BD02250E90A01E1FE
:100F4800ECD5030A01E1F8D5010A01E104D6070A44
:100F580001E110D6010A01E11CD6030A01E128D6F5
:100F680047D02250090A01E12ED7030A01E13AD7F6
:100F7800010A01E146D7070A01E152D739D02250C8
:100F88001D0A92E0030A95E033D02250480A01E195
:100F980016D7E40A2DD02250750A93E0030A97E089
:100FA800080A01E148D724D022503D0A01E148D778
:100FB800030A01E14CD7010A01E150D77F0A01E198
:100FC80054D7010A01E158D7030A01E15CD7010AA5
:100FD80001E160D7070A01E164D70AD02250C00AAC
:100FE80001E17CD705D022502A0A02D022500F0AEC
:100FF800455012000B6A0A6AE6EC5FF00101F26FD5
:101008005C6B070E966E010EF16F626B04009268BE
:1010180093689468948E9290929289820382FDECF0
:101028005EF092948984928C899C929E898E9568B0
:101038009368FA0E0001806FF80E816FA60E826F1A
:10104800FF0E836FB40E846FFE0E856F3F0E866FA2
:10105800FF0E876FD0CF88F0896BDAEC5FF0949839
:101068008B88CEEC5FF0630E0001806FFB0E816F02
:10107800F2C182F0836BDAEC5FF00101F22901E141
:10108800F26B0F0EF21765EC47F00101F26F7B0E61
:101098000001806FFB0E816FF2C182F0836BDAEC86
:1010A8005FF00400190E0101BA6F5A0EB96FB10E44
:1010B800E82EFED7B92FFCD7BA2FFAD700D0D09E8A
:1010C800F286F180F288F19CF28EF28CF28E2BEC93
:1010D8005AF08992899404007BEC4FF07BEC4FF036
:1010E8005A0E0E6EFF0E0F6E33EC58F0A60E0E6EF3
:1010F800FF0E0F6E33EC58F082A22FD0290E01019B
:10110800BA6F960EB96F7F0EE82EFED7B92FFCD7AF
:10111800BA2FFAD7000E0A6E800EECEC5BF0270EA1
:101128000E6EFE0E0F6E33EC58F017D0690E0001EC
:10113800806FFE0E816F82CF82F0836BDAEC5FF0F6
:10114800290E0101BA6F960EB96F7F0EE82EFED7F1
:10115800B92FFCD7BA2FFAD7040082B2E7D7898013
:1011680004009CEC49F0F30E0001806FFC0E816FC7
:1011780061C182F0836BDAEC5FF0000E0A6EC00E7C
:10118800ECEC5BF0660E5B6E010E5C6E7B0E5D6ECA
:10119800FC0E5E6E61C15FF0606A63EC5EF0660E25
:1011A8000E6E010E0F6E33EC58F0190E0101BA6F76
:1011B8005A0EB96FB10EE82EFED7B92FFCD7BA2F49
:1011C800FAD700D096EC34F001016151200FDB6FA3
:1011D8006151400FDA6F6151600FD96F899EF10537
:1011E8000EE160510CE1540E0001806FFD0E816F1D
:1011F800DAEC5FF0020E0101606F220E5F6FF151B1
:101208000EE160510CE1440E0001806FFD0E816F0C
:10121800DAEC5FF0010E0101606F040E5F6F5B5145
:1012280002E0E9EC3FF0D8C1C8FFDCEC2CF012EC8E
:1012380051F0000E0A6E800EECEC5BF0D4EC5EF020
:10124800000E0A6E800EECEC5BF00101F2510F0DFE
:101258002F0EF3240E6E090EF4200F6E33EC58F0A7
:10126800010162BFBFEC43F00101BE6BC36B000E0E
:10127800C16F010EC06FC1BF05D0C15166E1040E38
:10128800C05D63E20F0EC003F3CFB9F1F4CFBAF13A
:10129800C103F350BA271F0EB9250A6E0A0EBA21E8
:1012A8000B6EC5EC5CF00B5003E1030E0A5C49E3DE
:1012B800B10E0001806FFD0E816F0F0E0101C0039A
:1012C800F3CFB9F1F4CFBAF1C103F350BA271F0E27
:1012D800B9250001826F0A0E0101BA210001836F4E
:1012E800DAEC5FF0220E0101C003F3CFB9F1F4CFBD
:1012F800BAF1C103F350BA27000EB9250001B96F3E
:10130800030E0101BA210001BA6F0F0E0101C003DB
:10131800F3CFBBF1F4CFBCF1C103F350BC271F0ED0
:10132800BB250001BB6F0A0E0101BC210001BC6F87
:10133800030EBD6F56EC11F00101BF6FBF511AECDF
:101348005BF00101C04BC12B96D75D5101E196902E
:101358005D0501E056D1070E966E53D18A928A94A4
:1013680081A8939404EC60F00A500B1001E108D1B5
:10137800C3C1BDF1C20E0A6E010E0B6E8EEC5FF09A
:101388000101C36FC2B9C39F62511CE0350EC31976
:1013980007E12A0E0001806FF90E816FDAEC5FF029
:1013A800480E0001806FFF0E816FC3C182F0836B0E
:1013B8000101C2390F0B030B0001846F856BDAEC56
:1013C8005FF004D0A00E00D0E82EFDD70101F15146
:1013D80009E10D0E0101B96F760EE82EFED7B92F7F
:1013E800FCD700000101C2A930D0D951C3192DE1A1
:1013F8005F0EBD192AE1620E0001806FFF0E816F3A
:10140800DAEC5FF00382030E0001806FFF0E816F3C
:1014180060C182F0836B5FC184F0856BDAEC5FF0AA
:1014280027EE2FF060C1DFFF27EE30F05FC1DFFF4E
:101438008984020ED5EC55F0899403920101636BFF
:101448003EEC60F00101C36BDCD0F15147E0C251C2
:10145800100B0001D16F000ED26F0101C35134ECA3
:1014680038F0D1C0C4F1D2C0C5F1080E0101C419C9
:10147800C51101E10000070E0101C419C51102E1FF
:101488008EEC5AF0C405C51102E1FBEC54F0020ED3
:101498000101C419C51102E110EC37F0030E010176
:1014A800C419C51104E1B2EC24F00101BE6F050EA8
:1014B800C419C51104E153EC3BF00101BE6F090EDC
:1014C800C419C51102E16EEC51F00A0E0101C419EC
:1014D800C51101E096D02BEC4DF093D0C2C1A6F017
:1014E8000001A76B0101C3511DEC14F0A6C0C4F1A3
:1014F800A7C0C5F1070E0101C419C51102E1F8EC36
:1015080059F0020EC419C51102E156EC59F0C40590
:10151800C51102E15AEC1EF0030EC419C51102E10F
:1015280050EC50F0040EC419C51102E17CEC5EF0D9
:10153800050EC419C51102E124EC4AF0060E01019A
:10154800C419C51102E135EC60F0080EC419C511C3
:1015580002E160EC3AF0090EC419C51102E120EC71
:101568004EF00A0E0101C419C51102E146EC5DF006
:101578000C0E0101C419C51144E139EC33F041D016
:1015880065EC47F001015C6F5D513BE0F2515C197D
:1015980038E0898E000E0A6EC00EECEC5BF0D4ECDD
:1015A8005EF0000E0A6EC00EECEC5BF0F80E0E6EEC
:1015B800FE0E0F6E33EC58F05CC1F2F1000E526E65
:1015C800030E536EDBEC5DF096EC34F001015B51D9
:1015D80002E0E9EC3FF0420E0001806FFA0E816FE5
:1015E800F2C182F0836B60C184F0856B5FC186F0C5
:1015F800876BDAEC5FF00101F15103E0F251B6ECD0
:101608005FF082B22ED0050E0101BE192AE0A6D6DF
:10161800690E0001806FFE0E816F82CF82F0836BAE
:10162800DAEC5FF0290E0101BA6F960EB96F7F0EE2
:10163800E82EFED7B92FFCD7BA2FFAD70400000E30
:101648000A6EC00EECEC5BF0D4EC5EF0000E0A6E95
:10165800C00EECEC5BF06A0E0E6EFF0E0F6E33ECF4
:1016680058F082B2D5D7090E0101BA6F1E0EB96FB4
:10167800E40EE82EFED7B92FFCD7BA2FFAD7000010
:10168800899489920001A16BA26B2C0EA36FF90EAD
:10169800A46FA56B8DEC55F063D572C0A0F073C034
:1016A800A1F07650D96EDA6ADE6ADD6A70C00BF096
:1016B80071C00CF0B00E0D6E7DEC52F000019F6F02
:1016C8009F510AE120EE0FF07050D9267150DA22AE
:1016D800DF509F6F9F5102E09F51120020EE0EF0E5
:1016E8007050D9267150DA22DFA2070C20EE10F0D4
:1016F8007050D9267150DA2210EE10F07050E126A1
:101708007150E222E6CF93F0E6CF94F0E6CF95F061
:10171800E6CF96F074509325976F75509421986F83
:10172800000E9521996F000E96219A6FDE50975DF5
:10173800DE509859DE509959DE509A5901E3D7D2B4
:1017480020EE10F07050D9267150DA22DECF8FF0DB
:10175800DDCF90F08F1D746E901D756EC8D220EE8F
:1017680010F07050D9267150DA22FF0EDE148F6FF8
:10177800010EDE14906F000EDE14916F000EDE1461
:10178800926F8F5190119111921101E0FCD120EECE
:1017980010F07050D9267150DA22DECF8FF0DECFEC
:1017A80090F0DECF91F0DECF92F00A0E05D0D890FF
:1017B8009233913390338F33E82EF9D720EE09F026
:1017C800B051D926B151DA22DECF93F0DDCF94F0B3
:1017D800FF0E9325956FFF0E9421966F8F519515E7
:1017E800A26F90519615A36FA21101E091D020EE3F
:1017F80010F07050D9267150DA22DE50DE10DE105B
:10180800DE101EE120EE06F07050D9267150DA2263
:10181800DECFAAF0DECFABF0DECFACF0DECFADF09E
:10182800AA51AB11AC11AD1127E170C062F071C0C3
:1018380063F0646A656A666A676AC4EC26F014D065
:1018480070C062F071C063F020EE14F07050D926B9
:101858007150DA22DECF64F0DECF65F0DECF66F0BD
:10186800DECF67F0C4EC26F062C0AAF063C0ABF02C
:1018780064C0ACF065C0ADF0AA51AB11AC11AD11AC
:1018880001E139D2AA05AB11AC11AD1109E120EE85
:101898000FF07050D9267150DA22020EDF6E020C5A
:1018A800AA290FE1AB290DE1AC290BE1AD2909E12A
:1018B80020EE0FF07050D9267150DA22010EDF6E3B
:1018C800010C20EE14F07050D9267150DA22AAC00B
:1018D800DEFFABC0DEFFACC0DEFFADC0DEFF20EE3A
:1018E80006F07050D9267150DA22DE50DE10DE1074
:1018F800DE100EE120EE06F07050D9267150DA2283
:10190800AAC0DEFFABC0DEFFACC0DEFFADC0DEFFAD
:1019180020EE18F07050D9267150DA2210EE2BF014
:10192800B051E126B151E222DE50E61812E1DE5054
:10193800E6180FE1DE50E6180CE1DE50E61809E182
:10194800B0C023F0B1C024F00CEC43F0000901E072
:10195800AFD7B0C00AF0B1C00BF020EE14F0705051
:10196800D9267150DA22DECF0CF0DECF0DF0DECFB3
:101978000EF0DECF0FF012EC49F00AC0A6F00BC053
:10198800A7F00CC0A8F00DC0A9F00001A651A7113E
:10199800A811A91101E17BD7A251A627A351A7231A
:1019A800000EA823A92374C08FF075C090F0090E0B
:1019B800916FD89090338F33912FFBD78FC0A4F0BD
:1019C80090C0A5F0A451A51101E1A2D0A451A2256F
:1019D8008F6FA551A321906F20EE09F0B051D92641
:1019E800B151DA228F51DE5C9051DE5810E220EEC0
:1019F80009F0B051D926B151DA22DECF8FF0DDCF10
:101A080090F0A2518F5DA46FA3519059A56FA0C00B
:101A180019F0A1C01AF0A6C01BF0A7C01CF0A8C0FE
:101A28001DF0A9C01EF0A4C01FF0A5C020F020EE34
:101A380001F0B051D926B151DA22DF5098EC4EF0BE
:101A4800000901E035D70001A4518F6FA551906FAF
:101A5800916B926B20EE2BF0B051D926B151DA225E
:101A6800DECF93F0DECF94F0DECF95F0DECF96F0A8
:101A7800A651935D976FA7519459986FA85195599E
:101A8800996FA95196599A6F8F51975D90519859AE
:101A98009151995992519A592CE22F0EB0250A6EFC
:101AA800000EB1210B6E20EE2BF0B051D926B151AA
:101AB800DA22DECF8FF0DDCF90F0A6518F5FA751ED
:101AC800905B090ED8908F379037E82EFBD78F514F
:101AD800A0250C6E9051A1210D6E020E0F6E0E6A9C
:101AE800A4EC5CF020EE03F0B051D926B151DA2213
:101AF800DF6AA4C08FF0A5C090F0090ED8908F3788
:101B08009037E82EFBD78FC0AEF090C0AFF0A0D0D2
:101B180020EE0AF07050D9267150DA2210EE10F03B
:101B28007050E1267150E222DE50E65CDE50E65845
:101B3800DE50E658DE50E65818E3B0C023F0B1C0D6
:101B480024F00CEC43F0000901E0B2D6000120EECD
:101B58002BF0B051D926B151DA22A6C0DEFFA7C0BA
:101B6800DEFFA8C0DEFFA9C0DEFF20EE18F070502F
:101B7800D9267150DA22A6C0DEFFA7C0DEFFA8C0B2
:101B8800DEFFA9C0DEFF20EE10F07050D92671509C
:101B9800DA22DECF8FF0DDCF90F08F51916F010EFA
:101BA8009015926F91510008AE6F9251D8A0E82A13
:101BB8000208AF6FAE51745CAF51755804E274C03F
:101BC800AEF075C0AFF0B0C036F0B1C037F020EE5F
:101BD80018F07050D9267150DA22DECF38F0DECFF7
:101BE80039F0DECF3AF0DECF3BF017EC54F00009C5
:101BF80001E05ED620EE10F07050D9267150DA223E
:101C0800DECF8FF0DDCF90F000018F51916F010E84
:101C18009015926F9151B025936F9251B121946FA5
:101C28002F0E93250A6E000E94210B6EA0C00CF0A7
:101C3800A1C00DF0AEC00EF0AFC00FF0A4EC5CF088
:101C480020EE03F0B051D926B151DA22010EDF6E31
:101C5800AE51745EAF51755A7650D96EDA6AAE518C
:101C6800DE26AF51DD22AE51A027AF51A12320EED1
:101C780010F07050D9267150DA22AE51DE26AF51DD
:101C8800DE22000EDE22DE2220EE10F07050D92671
:101C98007150DA2210EE0AF07050E1267150E222FB
:101CA800DE50E65CDE50E658DE50E658DE50E65878
:101CB80020EE0AF0D8A020EE10F07050D92671500E
:101CC800DA22DECF9BF0DECF9CF0DECF9DF0DECFB8
:101CD8009EF020EE0AF07050D9267150DA229BC08F
:101CE800DEFF9CC0DEFF9DC0DEFF9EC0DEFF74509D
:101CF800751001E034D520EE0EF07050D9267150E1
:101D0800DA22000EDB8C000C70C00BF071C00CF0F6
:101D1800A70E0D6E7DEC52F00001A96FA95108E1E4
:101D280020EE0FF07050D9267150DA22DF50A96FDB
:101D3800A95102E0A951120020EE0AF07050D926EC
:101D48007150DA227250DE5C7350DE587450DE58DF
:101D58007550DE5816E220EE0EF07050D9267150FC
:101D6800DA22DFB20ED020EE0AF07050D926715078
:101D7800DA22DECF72F0DECF73F0DECF74F0DECF82
:101D880075F020EE10F07050D9267150DA22DECFAF
:101D98009FF0DECFA0F0DECFA1F0DECFA2F0A36BE4
:101DA800A46BA56BA66B20EE10F07050D92671506D
:101DB800DA22A3C0DEFFA4C0DEFFA5C0DEFFA6C0F6
:101DC800DEFF725073107410751001E100D220EE1E
:101DD80009F0A751D926A851DA22DECF8FF0DDCF3E
:101DE80090F08F51916F9051926F936B946B090E95
:101DF800D8909137923793379437E82EF9D791C016
:101E0800AAF092C0ABF093C0ACF094C0ADF09F5173
:101E1800A011A111A21101E196D0FF0E72240A6E41
:101E2800FF0E73200B6EFF0E74200C6EFF0E7520D4
:101E38000D6EAAC00EF0ABC00FF0ACC010F0ADC074
:101E480011F070EC58F00AC08FF00BC090F00CC085
:101E580091F00DC092F0FF0E00019F250A6EFF0E53
:101E6800A0210B6EFF0EA1210C6EFF0EA2210D6E9C
:101E7800AAC00EF0ABC00FF0ACC010F0ADC011F0AE
:101E880070EC58F00A5000018F5D0B5090590C50BF
:101E980091590D50925957E3FF0EAA258F6FFF0EE7
:101EA800AB21906FFF0EAC21916FFF0EAD21926FA9
:101EB8008F1D936F901D946F911D956F921D966F56
:101EC800FF0E9F25976FFF0EA021986FFF0EA1218F
:101ED800996FFF0EA2219A6F935197159B6F94519A
:101EE80098159C6F955199159D6F96519A159E6FEF
:101EF80020EE10F07050D9267150DA229BC0DEFF18
:101F08009CC0DEFF9DC0DEFF9EC0DEFF20EE10F00D
:101F18007050D9267150DA22DE50725EDE50735A44
:101F2800DE50745ADD50755A20EE14F07050D926E0
:101F38007150DA22DECFAEF0DECFAFF0DECFB0F0F8
:101F4800DECFB1F060D020EE06F07050D926715087
:101F5800DA22DECFAEF0DECFAFF0DECFB0F0DECFEC
:101F6800B1F0AE51AF11B011B1113FE170C062F0E4
:101F780071C063F0646A656A666A676AC4EC26F0D1
:101F880062C0AEF063C0AFF064C0B0F065C0B1F03D
:101F9800AE05AF11B011B11109E120EE0FF070508C
:101FA800D9267150DA22020EDF6E020CAE290FE13B
:101FB800AF290DE1B0290BE1B12909E120EE0FF0BD
:101FC8007050D9267150DA22010EDF6E010C20EE16
:101FD80006F07050D9267150DA22AEC0DEFFAFC0CD
:101FE800DEFFB0C0DEFFB1C0DEFF20EE14F070509F
:101FF800D9267150DA22AEC0DEFFAFC0DEFFB0C016
:10200800DEFFB1C0DEFFAE51AF11B011B11101E07A
:1020180085D0DDD0AA51725EAB51735AAC51745A57
:10202800AD51755A20EE10F07050D9267150DA2251
:10203800AA51DE26AB51DE22AC51DE22AD51DE22A2
:1020480020EE0EF07050D9267150DA22DFA220D08F
:1020580070C062F071C063F0AEC064F0AFC065F0EC
:10206800B0C066F0B1C067F0C4EC26F062C0AEF054
:1020780063C0AFF064C0B0F065C0B1F0AE51AF114D
:10208800B011B1111BE1726A736A746A756A50D033
:1020980070C041F071C042F0AEC043F0AFC044F030
:1020A800B0C045F0B1C046F099EC2EF041C0AEF09A
:1020B80042C0AFF043C0B0F044C0B1F00001AE2957
:1020C80007E1AF2905E1B02903E1B12901E176D79C
:1020D800B151B011AF1104E1020EAE5D01E25DD75E
:1020E80020EE13F0A751D926A851DA22DE50AE5DB2
:1020F800DE50AF59DE50B059DE50B15901E34DD72B
:1021080020EE14F07050D9267150DA22AEC0DEFFEE
:10211800AFC0DEFFB0C0DEFFB1C0DEFF7250AA5D07
:102128007350AB597450AC597550AD5901E272D720
:1021380020EE10F07050D9267150DA227250DE2647
:102148007350DE227450DE227550DE2272508F6F7B
:10215800010E7314906F916B926B8F119111921104
:1021680036E0A7C00AF0A8C00BF0AEC00CF0AFC0B4
:102178000DF0B0C00EF0B1C00FF012EC49F00AC07B
:10218800A3F00BC0A4F00CC0A5F00DC0A6F0000190
:10219800A351A411A511A61101E1FFD672C08FF0B9
:1021A80073C090F074C091F075C092F00A0E05D01B
:1021B800D8909233913390338F33E82EF9D78F51DB
:1021C800A3279051A4239151A5239251A62320EE31
:1021D80010F07050D9267150DA2210EE0AF07050C3
:1021E800E1267150E222DE50E65CDE50E658DE5011
:1021F800E658DE50E6581CE220EE10F07050D92662
:102208007150DA2210EE0AF07050E1267150E22285
:10221800DECFE6FFDECFE6FFDECFE6FFDECFE6FF6E
:1022280020EE0EF07050D9267150DA22000EDB8CA9
:1022380020EE10F07050D9267150DA22FF0EDE140D
:102248008F6F010EDE14906F000EDE14916F000E7A
:10225800DE14926F8F5190119111921101E16AD59C
:1022680020EE18F07050D9267150DA22A351DE18EA
:102278000AE1A451DE1807E1A551DE1804E1A651D0
:10228800DE1801E157D520EE18F07050D9267150AC
:10229800DA22A3C0DEFFA4C0DEFFA5C0DEFFA6C011
:1022A800DEFF48D5B951BA1101E1090C3F0EBD173F
:1022B800BB0E646E8E0E656E010E666EBDC067F055
:1022C80009EC00F00101906F905101E0A7D28EC196
:1022D80091F18FC192F1910E0001AB6F010EAC6FBD
:1022E800BBC0ADF0BCC0AEF084EC41F00101906F12
:1022F800905104E1B8AF02D0060E906FBDC0BEF099
:102308001C0E0001BE1701E1D0D0010190510FE071
:10231800040E901909E1910E0001AE6F010EAF6F26
:10232800B4EC50F00101906F0001BD870DD095C14C
:10233800BEF0110E0001BE1702E0070E03D0BDA5C6
:1023480003D0080E0101906F0101905101E0BCD04B
:102358000001BDA7B9D08EC111F08FC112F0ABC179
:1023680013F0ACC114F0ABEC58F011C07EF112C000
:102378007FF113C080F114C081F10E0E0101AB256D
:102388000A6E000EAC210B6E0C6A0D6A210E0E6EE1
:10239800500E0F6EC2EC59F0010120EE0BF0AB515C
:1023A800D926AC51DA22200EDF6E8EC10EF08FC115
:1023B8000FF0ABC110F0ACC111F0126A136A146AC5
:1023C800156A26EC5DF01C0E0101AB250A6E000EA5
:1023D800AC210B6E0C6A0D6A0E6A0F6AC2EC59F0DA
:1023E800010120EE03F08E51D9268F51DA22010E19
:1023F800DF6E7E517F118011811166E020EE2BF097
:102408008E51D9268F51DA22DECF82F1DECF83F1C9
:10241800DECF84F1DECF85F1910E626E010E636E20
:102428007EC164F07FC165F080C166F081C167F04C
:10243800686A696A6A6A6B6AB8EC40F00101906F71
:10244800905142E18EC136F08FC137F082C138F029
:1024580083C139F084C13AF085C13BF017EC54F0E0
:102468000101906FFF0E7E250001BE6FFF0E010176
:102478007F210001BF6FFF0E010180210001C06FA5
:10248800FF0E010181210001C16F010120EE0BF057
:102498008E51D9268F51DA22BEC0DEFFBFC0DEFFC3
:1024A800C0C0DEFFC1C0DEFF0FD0010190510CE1BA
:1024B80095A902D0040E07D00001BDA305D00101E3
:1024C80095A102D0070E906F0101905123E1000100
:1024D800BDB7BD8D010120EE2BF08E51D9268F514D
:1024E800DA22000110EE1CF0B951E126BA51E222BD
:1024F800DECFE6FFDECFE6FFDECFE6FFDECFE6FF8C
:1025080020EE20F0B951D926BA51DA22ABC1DEFF4C
:10251800ACC1DDFF0101905101E080D18EC111F005
:102528008FC112F0ABC113F0ACC114F0ABEC58F092
:10253800000120EE06F0B951D926BA51DA2211C0AD
:10254800DEFF12C0DEFF13C0DEFF14C0DEFF1C0E6C
:102558000101AB250A6E000EAC210B6ED3EC52F0D4
:10256800000120EE0AF0B951D926BA51DA220AC080
:10257800DEFF0BC0DEFF0CC0DEFF0DC0DEFFB9C002
:10258800D9FFBAC0DAFF8EC1DEFF8FC1DDFF0101BE
:1025980020EE05F08E51D9268F51DA22000110EE77
:1025A80002F0B951E126BA51E222DECFE6FFDDCFD3
:1025B800E5FF20EE0EF0B951D926BA51DA22BDC096
:1025C800DFFF20EE0FF0B951D926BA51DA22DF6ABF
:1025D80020EE18F0B951D926BA51DA22DE6ADE6A3D
:1025E800DE6ADD6A20EE10F0B951D926BA51DA2236
:1025F800DE6ADE6ADE6ADD6ABDAB10D120EE0AF063
:10260800B951D926BA51DA22DE50DE10DE10DE10BA
:1026180001E104D120EE0AF0B951D926BA51DA22E3
:1026280010EE10F0B951E126BA51E222DECFE6FFF2
:10263800DECFE6FFDECFE6FFDECFE6FF010120EECC
:1026480009F08E51D9268F51DA22DECFBEF0DDCFC8
:10265800BFF00001BE51C06FBF51C16FC26BC36BE9
:10266800090ED890C037C137C237C337E82EF9D71B
:10267800C0C07AF1C1C07BF1C2C07CF1C3C07DF19A
:1026880020EE06F0B951D926BA51DA22DECF8AF106
:10269800DECF8BF1DECF8CF1DECF8DF120EE0AF0AC
:1026A800B951D926BA51DA22DECF86F1DECF87F1C9
:1026B800DECF88F1DECF89F132D0B9C041F0BAC09F
:1026C80042F08AC143F08BC144F08CC145F08DC102
:1026D80046F099EC2EF041C08AF142C08BF143C01C
:1026E8008CF144C08DF101018D518C118B1105E1E4
:1026F800020E8A5D02E2020E906F8A2908E18B2998
:1027080006E18C2904E18D2902E1010E906F7A51CE
:10271800865F7B51875B7C51885B7D51895B0101BA
:10272800905109E186517A5D87517B5988517C59CE
:1027380089517D59C2E3000120EE14F0B951D92620
:10274800BA51DA228AC1DEFF8BC1DEFF8CC1DEFFFF
:102758008DC1DEFF0101905161E186510001BE6F1C
:10276800010E010187150001BF6FC06BC16BBE115F
:10277800C011C11153E08EC10AF08FC10BF08AC19C
:102788000CF08BC10DF08CC10EF08DC10FF012EC66
:1027980049F00AC082F10BC083F10CC084F10DC06E
:1027A80085F10101825183118411851103E1020E23
:1027B800906F34D086C1BEF087C1BFF088C1C0F029
:1027C80089C1C1F00A0E06D00001D890C133C033C8
:1027D800BF33BE33E82EF8D7010182510001BE2570
:1027E800C26F010183510001BF21C36F01018451F0
:1027F8000001C021C46F010185510001C121C56FCD
:1028080020EE18F0B951D926BA51DA22C2C0DEFF3B
:10281800C3C0DEFFC4C0DEFFC5C0DEFF01019051AA
:1028280006E0B9C0D9FFBAC0DAFFDE6ADD6A9051A6
:102838001200606E0001A651100B5E6EA75102E0F7
:1028480012EC51F05F6A5E5001E126D2609E040EE0
:10285800601803E10101545103E1140E601808E106
:102868000101406B416B0001A76B070EA66F070CB7
:102878003F0E601808E10101546B406B416B000189
:10288800A66BA76B12005F0E601808E10101556B7B
:10289800406B416B0001A66BA76B12003F0E606492
:1028A8000CD05F0E606009D00101DA51601805E0B4
:1028B800556B0001A66BA76B12000101DA51601875
:1028C80009E1010E556F546B406B416B0001A66B1B
:1028D800A76B1200DB51601801E0DED1010E546FC6
:1028E800F3D7600E60180CE10101555109E052510F
:1028F800080ED8B4030E5F6E0101406B416B34D2F1
:10290800600E601809E10101545106E0525102E0DD
:10291800090EF1D7050EEFD7680E601809E101011D
:10292800545106E01A0E416F900E60D189801CD276
:10293800680E601805E10101555102E0020EDBD76F
:102948006A0E601807E10101545104E01A0E416F44
:10295800F40E4CD16C0E601807E10101545104E0EB
:102968001A0E416F2C0E42D1700E601808E1010159
:10297800555105E0040E5F6E406B416BD7D7700E62
:10298800601801E0F1D10101545101E1EDD11B0EB4
:10299800416F620E2BD1898060500DE10001A6AB1A
:1029A80005D05F6A0101406B416B89901A0E0101E5
:1029B800416FAF0E406F020E601805E11A0E01015B
:1029C800416F920E406F050E601805E11A0E010165
:1029D800416FAE0E406F070E601805E11A0E010137
:1029E800416FB80E406F080E601805E11A0E01011C
:1029F800416FCC0E406F030E601802E060280CE1B6
:102A08008980680E5C6EE40EE82EFED75C2EFCD73B
:102A180000D05F6A899070D7140E601805E11A0E0D
:102A28000101416F9E0E406F160E601801E09CD1A7
:102A38001A0E0101416FA40ECAD0050E601805E1F7
:102A48001A0E0101416FF50E406F080E601801E083
:102A58008BD11A0E0101416FCC0E406F010E526FDF
:102A680083D160C079F01A0E0101416F950EAFD085
:102A780060505D6E5C6A79500C0D000EF324D96EBF
:102A8800010EF420DA6E5CC0DEFF5DC0DDFF1A0EB9
:102A98000101416F960E9BD060505C6E5D6A795063
:102AA8000C0D000EF324D96E010EF420DA6E5CC012
:102AB800DEFF5DC0DDFF1A0E0101416F970E87D062
:102AC80079500C0D020EF324D96E010EF420DA6E43
:102AD80060C0DFFF1A0E0101416F980E78D079505F
:102AE8000C0D030EF324D96E010EF420DA6E60C0CB
:102AF800DFFF0101406B416B010E37D01A0E010157
:102B0800416FB90E73D01A0E0101416FBA0E5FD032
:102B18001A0E0101416FBB0E406F350E0001806F28
:102B2800FE0E816FDAEC5FF00101536B406B416B75
:102B380055D00101406B416B350E0001806FFE0ED0
:102B4800816FDAEC5FF04AD00E0E0001806FFF0E45
:102B5800816FDAEC5FF00101406B416B010E506F41
:102B68003DD00101406B416B060E5F6EFDD060C029
:102B780079F00101406B416B5F6A30D00101526B03
:102B88001A0E416FF70E406F29D01A0E0101416FDE
:102B9800F70E1DD08990270E0101416F0F0E17D037
:102BA800180E601801E0E0D01A0E0101416F2D0ED9
:102BB8000ED01A0E0101416F2E0E09D01A0E010116
:102BC800416F2F0E04D01A0E0101416F300E406F75
:102BD800CBD00101406B416B0A0E5F6E8990C4D067
:102BE800040E5F6E270E0101416F0F0E406F9ED6D7
:102BF8008980010104D08990010E0101526F406B58
:102C0800416B5F6AB1D08990010E0101526F406B30
:102C1800416B5F6A79500C0D000EF324D96E010EDA
:102C2800F420DA6EDE6ADD6A79500C0D020EF324A8
:102C3800D96E010EF420DA6E6044E846030BDF6EAD
:102C480079500C0D030EF324D96E010EF420DA6EC0
:102C580060503F0BDF6E9E0E0001806FFC0E816F8F
:102C680060C082F0836B79500C0D020EF324D96E8C
:102C7800010EF420DA6EDF50846F856B79500C0DED
:102C8800030EF324D96E010EF420DA6EDF50866F3E
:102C9800876BDAEC5FF068D040C15CF041C15DF051
:102CA8005D5007E01A0A09E0010A54E03C0A5AE0BC
:102CB8005BD05C5001E115D657D05C502C0A01E17D
:102CC8006FD7010A01E175D7030A01E177D7010A35
:102CD80001E179D71F0A01E17CD7A00A01E15BD69F
:102CE800020A01E1BED6070A01E1C2D6030A01E1E0
:102CF800D3D6010A01E1E4D60F0A01E1F0D6060AAB
:102D080001E122D73A0A01E12CD70A0A01E173D777
:102D1800010A01E178D7170A01E1F0D6010A01E1B9
:102D2800F2D6030A01E1F4D6010A01E102D7790AD1
:102D380001E104D60E0A01E11AD7380A01E17DD66D
:102D4800010A01E11BD7030A01E11FD7010A01E1CA
:102D580021D70AD05C50580A01E142D73A0A01E16A
:102D680047D702D05C500F0A5FC0A6F00001A76BDE
:102D7800120019C0F6FF1AC0F7FFF86A0800F5CF6D
:102D88005AF0194A1A2A5A5001E11200250E5A1807
:102D98000AE017C00BF018C00CF05AC00DF00E6A0C
:102DA8006FEC5FF0E6D7526A536A506A516A200E98
:102DB800416E5468556819C0F6FF1AC0F7FFF86AE3
:102DC8000800F5CF5AF0194A1A2A300E5A180DE1A0
:102DD800300E416E19C0F6FF1AC0F7FFF86A0800F6
:102DE800F5CF5AF0194A1A2A07D02D0E5A1804E1BD
:102DF800516A020E506EEED72A0E5A1845E11B5042
:102E0800D96EDA6A020EDF26DF5CD96EDA6ADECFA7
:102E180048F0DECF49F049AE0BD048500008486E64
:102E28004950D8A0E82A0008496E516A020E506E2F
:102E380048C052F049C053F019C0F6FF1AC0F7FF56
:102E4800F86A0800F5CF5AF0194A1A2A23D00A0E50
:102E58005202F3CF1CF0F4CF1DF05302F3501D269D
:102E68005A501C26000E1D22D00E1C24526EFF0E36
:102E78001D20536E19C0F6FF1AC0F7FFF86A080044
:102E8800F5CF5AF0194A1A2A2F0E5A6403D0390E70
:102E98005A64DDD72E0E5A184AE119C0F6FF1AC037
:102EA800F7FFF86A0800F5CF5AF0194A1A2A2A0ECD
:102EB8005A1817E11B50D96EDA6A020EDF26DF5C5A
:102EC800D96EDA6ADECF54F0DECF55F019C0F6FFBE
:102ED8001AC0F7FFF86A0800F5CF5AF0194A1A2AFB
:102EE80026D0546A556A1DD00A0E5402F3CF1CF03E
:102EF800F4CF1DF05502F3501D265A501C26000E23
:102F08001D22D00E1C24546EFF0E1D20556E19C0B4
:102F1800F6FF1AC0F7FFF86A0800F5CF5AF0194A09
:102F28001A2A2F0E5A6403D0390E5A64DDD76C0E54
:102F38005A180BE1508419C0F6FF1AC0F7FFF86A57
:102F48000800F5CF5AF0194A1A2A5A5001E0A8D0B9
:102F58001200436A020E08D0436A080E05D0436A7D
:102F68000A0E02D0436A100E426EBAD017C00BF098
:102F780018C00CF01B50D96EDA6ADF50DF2ADF2A3E
:102F8800D96EDA6ADF500D6E0E6A6FEC5FF0F1D61B
:102F98001B50D96EDA6A020EDF26DF5CD96EDA6A58
:102FA800DECF4EF0DECF4FF04E504F1004E12C0E26
:102FB8004E6EF90E4F6E4EC00AF04FC00BF0C5ECC6
:102FC8005CF00AC056F00BC057F055BE15D05650ED
:102FD800545C5750555810E254C056F055C057F03D
:102FE8000BD017C00BF018C00CF041C00DF00E6AE2
:102FF8006FEC5FF0564A572A50B221D05250565CB7
:10300800535057581CE2EDD717C00BF018C00CF0FE
:103018004EC0F6FF4FC0F7FF000EF86E0F0EF764B4
:1030280003D00800F55005D0F6CFE9FFF7CFEAFF47
:10303800EF500D6E0E6A6FEC5FF04E4A4F2A4EC08D
:10304800F6FF4FC0F7FF000EF86E0F0EF76403D0BF
:103058000800F55005D0F6CFE9FFF7CFEAFFEF50AB
:10306800000911E05406D8A055065428CDE155288A
:103078000AE0CAD717C00BF018C00CF00E6A200E71
:103088000D6E6FEC5FF056501C6E57501D6E564A11
:10309800572A52501C5C53501D5801E36AD6EAD790
:1030A8005A501C6E1D6A1D5001E073D61C50580AF8
:1030B80001E158D73A0A01E14CD7010A01E156D794
:1030C800070A01E14CD70B0A01E146D71C0A01E1C6
:1030D8005FD7060A01E143D70D0A01E143D759D664
:1030E80050A411D01B50D96EDA6A040EDF26DF5CBB
:1030F800D96EDA6ADECF4AF0DECF4BF0DECF4CF085
:10310800DECF4DF027D0640E5A1813E01B50D96E4D
:10311800DA6ADF50DF2ADF2AD96EDA6ADECF1CF0DE
:10312800DDCF1DF01CC04AF01DC04BF04C6A4D6A43
:1031380011D01B50D96EDA6ADF50DF2ADF2AD96E28
:10314800DA6ADECF4AF0DDCF4BF0000E4BBEFF0E41
:103158004C6E4D6E640E5A180CE14DAE0AD04A6C96
:103168004B1ED8B04B2A4C1ED8B04C2A000E4D56D8
:103178005080586A596A4AC044F04BC045F04CC068
:1031880046F04DC047F044C00AF045C00BF046C0B9
:103198000CF047C00DF042C00EF043C00FF0106AAB
:1031A800116A5DEC5AF00A50406E44C00AF045C0FE
:1031B8000BF046C00CF047C00DF042C00EF043C003
:1031C8000FF0106A116A70EC58F00AC044F00BC096
:1031D80045F00CC046F00DC047F0090E40640BD016
:1031E800780E5A1803E03F6A070E02D03F6A270E8E
:1031F8003E6E3E50402658501E0FD96EDA6A405037
:10320800300FDF6E584A592A44504510461047106F
:1032180005E0595003E1200E585CB5E350A008D0F2
:1032280058501E0FD96EDA6A2D0EDF6E584A592A89
:1032380058C056F059C057F00BD017C00BF018C043
:103248000CF041C00DF00E6A6FEC5FF0564A572A39
:1032580050B205D05250565C53505758EEE317C041
:103268000BF018C00CF05806D8A0590658501E0F7D
:10327800D96EDA6ADF500D6E0E6A6FEC5FF0585047
:1032880059100AE0ECD717C00BF018C00CF00E6A02
:10329800200E0D6E6FEC5FF056501C6E57501D6E71
:1032A800564A572A52501C5C53501D5801E361D5A9
:1032B800EAD75DC089F05EC08AF06150D96EDA6ADB
:1032C800DE6ADD6A5BC00BF05CC00CF0950E0D6E1B
:1032D8007DEC52F00001846F84510AE120EE0FF07A
:1032E8005B50D9265C50DA22DF50846F845102E0AB
:1032F8008451120020EE0EF05B50D9265C50DA2281
:10330800DFA0070C20EE10F05B50D9265C50DA22C3
:10331800DECF62F0DECF63F0DECF64F0DECF65F0A3
:1033280020EE0AF05B50D9265C50DA22DECF66F038
:10333800DECF67F0DECF68F0DECF69F06250665C02
:10334800806F63506758816F64506858826F65500A
:103358006958836F5F50626E6050636E646A656A15
:103368006250805D63508159645082596550835919
:1033780001E319D280C05FF081C060F014D220EE62
:1033880010F05B50D9265C50DA22FF0EDE14626E14
:10339800010EDE14636E000EDE14646E000EDE1481
:1033A800656E625063106410651001E083D120EEF1
:1033B80010F05B50D9265C50DA22DECF62F0DECF07
:1033C80063F0DECF64F0DECF65F00A0E05D0D8904A
:1033D8006532643263326232E82EF9D720EE09F0A2
:1033E8009551D9269651DA22DECF66F0DDCF67F007
:1033F800FF0E6624686EFF0E6720696E62506814BF
:103408008B6F635069148C6F8B1166E120EE10F09E
:103418005B50D9265C50DA22DE50DE10DE10DE105A
:103428000FE120EE06F05B50D9265C50DA22DECFA1
:1034380085F0DECF86F0DECF87F0DECF88F01CD0B7
:103448005BC041F05CC042F020EE14F05B50D9261E
:103458005C50DA22DECF43F0DECF44F0DECF45F019
:10346800DECF46F099EC2EF041C085F042C086F0E0
:1034780043C087F044C088F0000188518711861145
:103488000CE1020E855D09E220EE0FF05B50D926B3
:103498005C50DA22020EDF6E020C85290FE18629C4
:1034A8000DE187290BE1882909E120EE0FF05B5037
:1034B800D9265C50DA22010EDF6E010C20EE14F0E2
:1034C8005B50D9265C50DA2285C0DEFF86C0DEFF5D
:1034D80087C0DEFF88C0DEFF95C00AF096C00BF0FB
:1034E80020EE14F05B50D9265C50DA22DECF0CF0C7
:1034F800DECF0DF0DECF0EF0DECF0FF012EC49F08C
:103508000AC08DF00BC08EF00CC08FF00DC090F08B
:1035180000018D518E118F11901101E1B5D78B519A
:103528008D278C518E23000E8F2390235FC062F06D
:1035380060C063F0090E646ED89063326232642E04
:10354800FBD762C091F063C092F09151921101E1F2
:10355800A3D091518B25626E92518C21636E20EE1F
:1035680009F09551D9269651DA226250DE5C6350F3
:10357800DE5810E220EE09F09551D9269651DA224C
:10358800DECF62F0DDCF63F08B51625C916F8C51BE
:103598006358926F89C019F08AC01AF08DC01BF069
:1035A8008EC01CF08FC01DF090C01EF091C01FF09F
:1035B80092C020F020EE01F09551D9269651DA22DA
:1035C800DF5027EC53F0000901E06FD7000120EE2F
:1035D80003F09551D9269651DA22DF504EE09151E9
:1035E800626E9251636E646A656A20EE2BF09551A3
:1035F800D9269651DA22DECF66F0DECF67F0DECF2D
:1036080068F0DECF69F08D51665C6A6E8E5167583E
:103618006B6E8F5168586C6E905169586D6E625020
:103628006A5C63506B5864506C5865506D5825E25D
:1036380020EE2BF09551D9269651DA22DECF62F092
:10364800DDCF63F08D51625E8E51635A090ED890BA
:1036580062366336E82EFBD7625089250A6E6350BE
:103668008A210B6E2F0E95250C6E000E96210D6E7D
:10367800020E0F6E0E6AA4EC5CF091C062F092C06C
:1036880063F0090ED89062366336E82EFBD762C025
:1036980093F063C094F06BD020EE18F05B50D926FD
:1036A8005C50DA228DC0DEFF8EC0DEFF8FC0DEFFE9
:1036B80090C0DEFF20EE10F05B50D9265C50DA2275
:1036C800DECF62F0DDCF63F06250646E010E6314EA
:1036D800656E64500008936F6550D8A0E82A020808
:1036E800946F93515F5C9451605804E25FC093F00B
:1036F80060C094F095C036F096C037F020EE18F010
:103708005B50D9265C50DA22DECF38F0DECF39F0B4
:10371800DECF3AF0DECF3BF017EC54F0000901E0C1
:10372800C4D689C00AF08AC00BF020EE10F05B50B6
:10373800D9265C50DA22DECF62F0DDCF63F062502A
:10374800646E010E6314656E645000019525666E03
:1037580065509621676E2F0E66240C6E000E67204A
:103768000D6E93C00EF094C00FF0A4EC5CF0935172
:103778005F5E9451605A6150D96EDA6A9351DE26C1
:103788009451DD229351892794518A2320EE10F019
:103798005B50D9265C50DA229351DE269451DE2202
:1037A800000EDE22DE225F50601001E0E8D5000C3A
:1037B800670EF66EF80EF76E000EF86E0900F5CF7C
:1037C800C9F00A00F5CFCAF00001CD6BD06B01013A
:1037D800E76BD85144EC60F0CE6ACF6A0FD1D16B59
:1037E8002F0E136E070E146EC90E156E44EC55F0AD
:1037F80013C0CEF014C0CFF0CEC0D9FFCFC0DAFFCF
:103808003B0EDE1801E0F5D0F9D0D15113E1CEC05E
:103818000EF0CFC00FF01EEC59F00001D06F800EF3
:10382800D06503D0D051800FCD6F030ECD65D5D0B4
:10383800CD6BD3D0D10511E10101F2510001D019AE
:1038480003E07F0ED01909E1CEC00EF0CFC00FF013
:103858001EEC59F00101606FC0D0020ED11911E1C0
:103868000101F2510001D01903E07F0ED01909E1DE
:10387800CEC00EF0CFC00FF01EEC59F001015F6F03
:10388800ACD0020ED1652CD0080ED16129D001012F
:10389800F2510001D0190CE07F0ED01909E0810E19
:1038A800D01906E0820ED01903E0830ED01918E172
:1038B800CD51050DAC0EF324CB6F020EF420CC6F66
:1038C800CEC00EF0CFC00FF01EEC59F00001A66F6D
:1038D800D151CB25A76F000ECC21A86FFD0E5DD06E
:1038E800070ED1652CD01B0ED16129D00101F251F0
:1038F8000001D0190CE07F0ED01909E0810ED01913
:1039080006E0820ED01903E0830ED01918E1CD51DC
:10391800130DAA0EF324CB6F030EF420CC6FCEC088
:103928000EF0CFC00FF01EEC59F00001A66FD15178
:10393800CB25A76F000ECC21A86FF80E2ED01A0E3B
:10394800D16533D0280ED16130D00101F251000188
:10395800D0190CE07F0ED01909E0810ED01906E0CD
:10396800820ED01903E0830ED0191FE1CD510D0D41
:10397800780EF324CB6F020EF420CC6FCEC00EF07D
:10398800CFC00FF01EEC59F00001A66FD151CB2526
:10399800A76F000ECC21A86FE50EA725D96EFF0EE4
:1039A800A821DA6EA6C0DFFF18D0280ED11915E1BC
:1039B8000101F2510001D01903E07F0ED0190DE189
:1039C800E70E0A6E010E0B6ECEC00CF0CFC00DF0E4
:1039D8000F6A080E0E6E45EC5BF00001D12B136ADE
:1039E800146AC90E156E44EC55F013C0CEF014C01D
:1039F800CFF00001CE51CF1101E007D72F0E6E6E28
:103A0800070E6F6E716A910E706E000E726E030E65
:103A1800736E65EC54F06E506F1001E0E0D6D16B18
:103A2800D1510D0D820EF324D96E020EF420DA6EF8
:103A3800DF50A66FA6C0A7F0A86BA96BAA6BA9C098
:103A4800AAF0A8C0A9F0A7C0A8F0A76BD1510D0D86
:103A5800810EF324D96E020EF420DA6EDF50AB6FBC
:103A6800ABC0ACF0AD6BAE6BAF6BADC0AFF0ACC084
:103A7800AEF0AD6BAC6BD1510D0D800EF324D96E49
:103A8800020EF420DA6EDF50B06FB0C0B1F0B26B46
:103A9800B36BB46BB1C0B4F0B36BB26BB16BAC5178
:103AA800B125B56FAD51B221B66FAE51B321B76F25
:103AB800AF51B421B86FA751B525B96FA851B62138
:103AC800BA6FA951B721BB6FAA51B821BC6FD151A8
:103AD8000D0D830EF324D96E020EF420DA6EDF503A
:103AE800B925BD6F000EBA21BE6F000EBB21BF6F96
:103AF800000EBC21C06FBDC0C1F0BEC0C2F0BFC0C7
:103B0800C3F0C0C0C4F0C56BC4BFC569C5C0C6F0AA
:103B1800C5C0C7F0C5C0C8F0D1511E0D0F0EF324A3
:103B2800D96E020EF420DA6EC1C0DEFFC2C0DEFF1D
:103B3800C3C0DEFFC4C0DEFFC5C0DEFFC6C0DEFFF7
:103B4800C7C0DEFFC8C0DEFFD151130DAE0EF3248F
:103B5800D96E030EF420DA6EDF50A76FA66BD15131
:103B6800130DAF0EF324D96E030EF420DA6EDF5076
:103B7800A625A86F000EA721A96FD1511E0D1C0EF6
:103B8800F324D96E020EF420DA6EA8C0DEFFA9C0B5
:103B9800DDFFD1511E0D1C0EF324D96E020EF42048
:103BA800DA6EDECFA6F0DDCFA7F0A6C00AF0A7C078
:103BB8000BF00C6A0D6A0E6A0F6A106A116AD1510D
:103BC8001E0D0F0EF324D96E020EF420DA6EDECF2E
:103BD800A8F0DECFA9F0DECFAAF0DECFABF0DECFC3
:103BE800ACF0DECFADF0DECFAEF0DECFAFF0A8C0E8
:103BF80012F0A9C013F0AAC014F0ABC015F0ACC005
:103C080016F0ADC017F0AEC018F0AFC019F063ECF5
:103C180056F00AC0B0F00BC0B1F00CC0B2F00DC045
:103C2800B3F00EC0B4F00FC0B5F010C0B6F011C0BC
:103C3800B7F00001D1511E0D0F0EF324D96E020EFC
:103C4800F420DA6EB0C0DEFFB1C0DEFFB2C0DEFF26
:103C5800B3C0DEFFB4C0DEFFB5C0DEFFB6C0DEFF16
:103C6800B7C0DEFF600E806FFA0E816FD1C082F0A0
:103C7800836BD1511E0D1C0EF324D96E020EF42055
:103C8800DA6EDECF84F0DDCF85F0DAEC5FF000018C
:103C9800D12B030ED165C4D6E70E806FFA0E816F63
:103CA800E70E826F010E836FDAEF5FF079500C0D2B
:103CB800000EF324D96E010EF420DA6E79500C0D43
:103CC800080EF324E16E010EF420E26EE6CFB4F0A4
:103CD800E5CFB5F0FF0E0001B425B66FFF0EB52194
:103CE800B76FDE50B65DB751800AB86FDE50800AF4
:103CF800B85948E379500C0D020EF324D96E010E21
:103D0800F420DA6EDF50B26FB36B79500C0D0A0EE7
:103D1800F324D96E010EF420DA6EDF50B46FFF0E73
:103D2800B425B56FB66BFF0EB623B251B55DB6516B
:103D3800800AB76FB351800AB75924E379500C0D44
:103D4800030EF324D96E010EF420DA6EDF50B26F41
:103D5800B36B79500C0D0B0EF324D96E010EF420C1
:103D6800DA6EDF50B46FFF0EB425B56FB66BFF0E79
:103D7800B623B251B55DB651800AB76FB351800A08
:103D8800B75961E21F0E0101516F010E536F8990FF
:103D9800530E0001806FF90E816F79500C0D000EE3
:103DA800F324D96E010EF420DA6EDECF82F0DDCF77
:103DB80083F079500C0D080EF324D96E010EF4200F
:103DC800DA6EDECFB2F0DDCFB3F0FF0EB225846F2E
:103DD800FF0EB321856F79500C0D020EF324D96EB6
:103DE800010EF420DA6EDF50866F876B79500C0D68
:103DF8000A0EF324D96E010EF420DA6EDF50B46F88
:103E0800FF0EB425886F896BFF0E892379500C0D3E
:103E1800030EF324D96E010EF420DA6EDF508A6F98
:103E28008B6B79500C0D0B0EF324D96E010EF42018
:103E3800DA6EDF50B56FFF0EB5258C6F8D6BFF0EF8
:103E48008D23DAEC5FF079500C0D0B0EF324D96E4C
:103E5800010EF420DA6EDF500001B26FB2C0B3F089
:103E6800B46BB56BB66B79500C0D000EF324D96E9C
:103E7800010EF420DA6EDECFB7F0DDCFB8F0B7C0B0
:103E8800B9F0B8C0BAF0000EBABFFF0EBB6FBC6F76
:103E9800B951B303F3CFBDF0F4CFBEF0BF6BC06B25
:103EA800B403F350BE27F450BF23000EC023BA5109
:103EB800B303F350BE27F450BF23000EC023B951FB
:103EC800B503F350BF27F450C023BA51B403F350DD
:103ED800BF27F450C023BB51B303F350BF27F4509E
:103EE800C023B651B903F350C027BA51B503F350F4
:103EF800C027BB51B403F350C027BC51B303F350E0
:103F0800C027BDC0C2F0BEC0C3F0BFC0C4F0C0C0AF
:103F1800C5F0C2C00AF0C3C00BF0C4C00CF0C5C0E5
:103F28000DF079500C0D0A0EF324D96E010EF42011
:103F3800DA6EDF50B26FB2C0B3F0B46BB56BB66B6C
:103F4800B5C0B6F0B4C0B5F0B3C0B4F0B36BB3C08D
:103F58000EF0B4C00FF0B5C010F0B6C011F032ECDE
:103F680057F00AC0C2F00BC0C3F00CC0C4F00DC0BB
:103F7800C5F079500C0D0B0EF324D96E010EF42008
:103F8800DA6EDF50B26FB2C0B3F0B46BB56BB66B1C
:103F980079500C0D020EF324D96E010EF420DA6E5E
:103FA800DF50B76FB7C0B8F0B96BBA6BBB6BBAC0AC
:103FB800BBF0B9C0BAF0B8C0B9F0B86BB851B30328
:103FC800F3CFBCF0F4CFBDF0BE6BBF6BB403F350BE
:103FD800BD27F450BE23000EBF23B951B303F350DD
:103FE800BD27F450BE23000EBF23B851B503F350CC
:103FF800BE27F450BF23B951B403F350BE27F45081
:10400800BF23BA51B303F350BE27F450BF23B651B0
:10401800B803F350BF27B951B503F350BF27BA51BE
:10402800B403F350BF27BB51B303F350BF27BC51B0
:10403800C227BD51C323BE51C423BF51C5237950E4
:104048000C0D030EF324D96E010EF420DA6EDF5046
:10405800B26FB2C0B3F0B46BB56BB66BB5C0B6F0A7
:10406800B4C0B5F0B3C0B4F0B36BB351C227B45108
:10407800C323B551C423B651C5237950220D000E70
:10408800F324706E030EF420716EC2C072F0C3C0C8
:1040980073F0C4C074F0C5C075F088EC0EF0C16F41
:1040A800C15111E0330E806FFB0E816FC2C082F0E8
:1040B800C3C083F0C4C084F0C5C085F0C1C086F019
:1040C800876BDAEC5FF079500C0D040EF324D96E8F
:1040D800010EF420DA6EC2C0DEFFC3C0DEFFC4C02A
:1040E800DEFFC5C0DEFF0101536B899012007950D5
:1040F8000C0D030EF324D96E010EF420DA6EDF2ABC
:1041080079500C0D030EF324D96E010EF420DA6EEB
:10411800DF500001B26FB36B79500C0D0B0EF32416
:10412800D96E010EF420DA6EDF50B46FFF0EB4259D
:10413800B56FB66BFF0EB623B251B55DB651800AA6
:10414800B76FB351800AB7594AE279500C0D030E84
:10415800F324D96E010EF420DA6EDF6A79500C0D63
:10416800020EF324D96E010EF420DA6EDF2A79509C
:104178000C0D020EF324D96E010EF420DA6EDF5016
:10418800B26FB36B79500C0D0A0EF324D96E010E81
:10419800F420DA6EDF50B46FFF0EB425B56FB66B3E
:1041A800FF0EB623B251B55DB651800AB76FB35151
:1041B800800AB75914E279500C0D020EF324D96E17
:1041C800010EF420DA6EDF6A79500C0D000EF3242C
:1041D800D96E010EF420DA6EDE2A000EDD22795047
:1041E8000C0D0B0EF324D96E010EF420DA6EDF509D
:1041F800B26FB2C0B3F0B46BB56BB66B79500C0D3F
:10420800000EF324D96E010EF420DA6EDECFB7F07B
:10421800DDCFB8F0B7C0B9F0B8C0BAF0000EBABF79
:10422800FF0EBB6FBC6FB951B303F3CFBDF0F4CF32
:10423800BEF0BF6BC06BB403F350BE27F450BF236E
:10424800000EC023BA51B303F350BE27F450BF2366
:10425800000EC023B951B503F350BF27F450C02353
:10426800BA51B403F350BF27F450C023BB51B30372
:10427800F350BF27F450C023B651B903F350C027F9
:10428800BA51B503F350C027BB51B403F350C0274C
:10429800BC51B303F350C02779500C0D040EF3241E
:1042A800D96E010EF420DA6EBDC0DEFFBEC0DEFF9F
:1042B800BFC0DEFFC0C0DEFF79500C0D0A0EF3242C
:1042C800D96E010EF420DA6EDF50B26FB2C0B3F0CF
:1042D800B46BB56BB66B79500C0D040EF324D96E24
:1042E800010EF420DA6EDECFB7F0DECFB8F0DECF05
:1042F800B9F0DECFBAF0B9C0BAF0B8C0B9F0B7C0FB
:10430800B8F0B76BB751B303F3CFBBF0F4CFBCF041
:10431800BD6BBE6BB403F350BC27F450BD23000E35
:10432800BE23B851B303F350BC27F450BD23000E8D
:10433800BE23B751B503F350BD27F450BE23B8517F
:10434800B403F350BD27F450BE23B951B303F3505F
:10435800BD27F450BE23B651B703F350BE27B8515A
:10436800B503F350BE27B951B403F350BE27BA5171
:10437800B303F350BE2779500C0D040EF324D96E05
:10438800010EF420DA6EBBC0DEFFBCC0DEFFBDC08C
:10439800DEFFBEC0DEFF79500C0D0B0EF324D96E84
:1043A800010EF420DA6EDF50B26FB2C0B3F0B46B16
:1043B800B56BB66B79500C0D020EF324D96E010E55
:1043C800F420DA6EDF50B76FB7C0B8F0B96BBA6BCC
:1043D800BB6BBAC0BBF0B9C0BAF0B8C0B9F0B86B23
:1043E800B851B303F3CFBCF0F4CFBDF0BE6BBF6BD5
:1043F800B403F350BD27F450BE23000EBF23B951B8
:10440800B303F350BD27F450BE23000EBF23B851A9
:10441800B503F350BE27F450BF23B951B403F3508A
:10442800BE27F450BF23BA51B303F350BE27F4504C
:10443800BF23B651B803F350BF27B951B503F350A2
:10444800BF27BA51B403F350BF27BB51B303F3508E
:10445800BF2779500C0D040EF324D96E010EF420F9
:10446800DA6EBC51DE26BD51DE22BE51DE22BF51BE
:10447800DE2279500C0D030EF324D96E010EF420C0
:10448800DA6EDF50B26FB2C0B3F0B46BB56BB66B17
:10449800B5C0B6F0B4C0B5F0B3C0B4F0B36B7950E2
:1044A8000C0D040EF324D96E010EF420DA6EB3510C
:1044B800DE26B451DE22B551DE22B651DE22795015
:1044C800220D000EF324706E030EF420716E7950E5
:1044D8000C0D040EF324D96E010EF420DA6EDECF33
:1044E80072F0DECF73F0DECF74F0DECF75F088ECBB
:1044F8000EF0766E765019E0330E806FFB0E816FEA
:1045080079500C0D040EF324D96E010EF420DA6EE6
:10451800DECF82F0DECF83F0DECF84F0DECF85F011
:1045280076C086F0876BDAEC5FF00101536B1200FE
:10453800000E5B6E030E5C6E2F0E5D6E070E5E6ED8
:10454800020E606E5F6AD50E616E5DEC19F07B6ECF
:10455800740E0001806FFD0E816FD5C082F0D6C049
:1045680083F0DAEC5FF00001D76BD86BD36BD46BB8
:10457800D96BDA6BD951B50FD96EDA6ADF6AD951BE
:10458800C40FD96EDA6ADF6AD94BDA2BDABFF2D7F1
:10459800DA5103E10F0ED95DEDE3DB6BDC6B54D12F
:1045A8002F0EDB25D96E070EDC21DA6E0D0EDE1814
:1045B80001E00FD19A0E0A6EFF0E0B6EB50E0C6E4F
:1045C800B0EC54F00A500B1007E1C40E0A6ECAECA6
:1045D80051F00A500101F16F940E0A6EFF0E0B6E36
:1045E800B50E0C6EB0EC54F00A500B1007E1C40E77
:1045F8000A6ECAEC51F00A500101626F790E0A6E18
:10460800FF0E0B6EB50E0C6EB0EC54F00A500B108A
:1046180007E1C40E0A6ECAEC51F00A5001015D6F41
:10462800D70E0A6EFF0E0B6EB50E0C6EB0EC54F082
:104638000A500B1007E1C40E0A6ECAEC51F00A507A
:1046480001015B6FDF0E0A6EFF0E0B6EB50E0C6E6E
:10465800B0EC54F00A500B1007E1C40E0A6ECAEC15
:1046680051F00A500101D86FDB0E0A6EFF0E0B6E77
:10467800B50E0C6EB0EC54F00A500B1008E1C40EE5
:104688000A6ECAEC51F00AC04CF10BC04DF1AB0EEA
:104698000A6EFF0E0B6EB50E0C6EB0EC54F00A509D
:1046A8000B1007E1C40E0A6ECAEC51F00A50010162
:1046B800616F0001DD6BDE6BA60E5B6E5C6A800EBF
:1046C8005D6EFF0E5E6EDDC05FF0DEC060F063EC15
:1046D8005EF0A60E0A6E0B6AB50E0C6EB0EC54F0C6
:1046E8000A500B1018E10F0E0001DD03F3CF6EF036
:1046F800F4CF6FF0DE03F3506F262F0E6E240A6E90
:10470800090E6F200B6EC40E0C6E0D6A0F6A0F0E29
:104718000E6E45EC5BF00001DD4BDE2BDEBFCCD727
:10472800DE5103E1100EDD5DC7E3DE6B010EDD6FC8
:10473800A60E5B6E5C6A870E5D6EFF0E5E6EDDC058
:104748005FF0DEC060F063EC5EF0A60E0A6E0B6AE6
:10475800B50E0C6EB0EC54F00A500B1018E10F0EA9
:104768000001DD03F3CF6EF0F4CF6FF0DE03F350FA
:104778006F261F0E6E240A6E0A0E6F200B6EC40E73
:104788000C6E0D6A0F6A0F0E0E6E45EC5BF00001A1
:10479800DD4BDE2BDEBFCCD7DE5103E1040EDD5D41
:1047A800C7E3D96BDA6BD951B50FD96EDA6ADF6A0C
:1047B800D951C40FD96EDA6ADF6AD94BDA2BDABF5E
:1047C800F2D7DA5103E10F0ED95DEDE3D36BD46B69
:1047D80015D02F0EDB25D96E070EDC21DA6E0A0EF6
:1047E800DE1830E02F0EDB25D96E070EDC21DA6EDD
:1047F800200EDE1806E1D46B010ED36FD76BD86B91
:1048080021D0D351D41109E02F0EDB25D96E070E24
:10481800DC21DA6ED751C40F08D02F0EDB25D96EF4
:10482800070EDC21DA6ED751B50FE16EE26ADFCFF1
:10483800E7FFD8BF05D0D85105E10F0ED75D02E2DA
:10484800D74BD82BDB4BDC2BD551DB5DD651DC5954
:1048580001E2A6D6640E806FFD0E816F5DC182F005
:10486800836BDAEC5FF0DE0E0001806FFD0E816F66
:10487800F1C182F0836BDAEC5FF0C00E0001806F4B
:10488800FD0E816F62C182F0836BDAEC5FF0CF0EB0
:104898000001806FFD0E816FD8C182F0836BDAEC66
:1048A8005FF0430E0001806FFC0E816F4CC182F0F7
:1048B8004DC183F0DAEC5FF00001DD6BDE6BD10EE9
:1048C800806FFC0E816FDDC082F0DEC083F00F0EBA
:1048D800DD03F3CF6EF0F4CF6FF0DE03F3506F26F5
:1048E8002F0E6E24846F090E6F20856FDAEC5FF04F
:1048F8000001DD4BDE2BDEBFE2D7DE5103E1100EF7
:10490800DD5DDDE3DC6B010EDB6FE20E806FFC0E1C
:10491800816FDBC082F0DCC083F00F0EDB03F3CFC6
:104928006EF0F4CF6FF0DC03F3506F261F0E6E2489
:10493800846F0A0E6F20856FDAEC5FF00001DB4BA5
:10494800DC2BDCBFE2D7DC5103E1040EDB5DDDE3E9
:104958002A0E806FF90E816FDAEF5FF0898E8980F9
:10496800020E0CEC60F031EC3DF0FB6FFB5118E0EF
:1049780079501E0D1B0EF324D96E020EF420DA6E48
:1049880079501E0D1B0EF324E16E020EF420E26E28
:10499800E7500409DF6E23EC5FF00001FB511200C1
:1049A80001015B5150E0385139113A113B114BE08C
:1049B800795049E179501E0D070EF324D96E020E85
:1049C800F420DA6E38C1E4F039C1E5F03AC1E6F016
:1049D8000001E36B000EE325E76F010EE421E86FA9
:1049E800000EE521E96F000EE621EA6FEB6BEC6B38
:1049F800ED6BEE6BDE50E71926E1DE50E81923E196
:104A0800DE50E91920E1DE50EA191DE1DE50EB190C
:104A18001AE1DE50EC1917E1DE50ED1914E1DE5011
:104A2800EE1911E12F0EAA6F070EAB6F01015B5152
:104A3800A6EC4DF00392000ED5EC55F00392786A7F
:104A480089907850120079501E0D170EF324D96EF4
:104A5800020EF420DA6EDE50DE10DE10DE101EE0EC
:104A680079501E0D170EF324D96E020EF420DA6E5B
:104A7800DE50DE10DE1002E1DE0410E079501E0D7B
:104A8800170EF324D96E020EF420DA6EDE280DE13B
:104A9800DE280BE1DE2809E1DE2807E10001EF69E5
:104AA800F069F169F269F96B2ED079501E0D170E75
:104AB800F324D96E020EF420DA6EDECFDBF0DECFFF
:104AC800DCF0DECFDDF0DECFDEF0DCC0DBF0DDC019
:104AD800DCF0DEC0DDF00001DE6BDBC0EFF0DCC037
:104AE800F0F0DDC0F1F0DEC0F2F079501E0D170EC7
:104AF800F324D96E020EF420DA6EDECFDBF0DDCFC0
:104B0800DCF0DB51F96FFA6B0392F56BF66BF76B20
:104B1800F86BF36BF46BBCD081A881AA09D0D70ECF
:104B2800806FFE0E816FDAEC5FF0ACD08994ACD068
:104B3800F3C0DBF0F4C0DCF0000EDCBFFF0EDD6F6D
:104B4800DE6FFF0EEF25DF6FFF0EF021E06FFF0E27
:104B5800F121E16FFF0EF221E26FDB51DF190DE168
:104B6800DC51E0190AE1DD51E11907E1DE51E219F2
:104B780004E1F951FA1101E103827950220D000E86
:104B8800F3245B6E030EF4205C6E2F0E5D6E070E31
:104B98005E6E010E606E5F6AFC0E616E5DEC19F070
:104BA8000001FE6FFE5101E0E3D6FC51FD1101E169
:104BB800DFD681A881AA07D0E20E806FFE0E816F32
:104BC800DAEC5FF05FD0FC51D5EC55F081B808D035
:104BD800E20E0001806FFE0E816FDAEC5FF052D0BA
:104BE8000001FC51F527FD51F623000EF723F823A9
:104BF80079501E0D070EF324D96E020EF420DA6EDA
:104C0800000EDE24DB6F010EDE20DC6F000EDE20DE
:104C1800DD6F000EDE20DE6F000EDE20DF6F000E7F
:104C2800DE20E06F000EDE20E16F000EDE20E26F76
:104C380079501E0D070EF324D96E020EF420DA6E99
:104C4800DBC0DEFFDCC0DEFFDDC0DEFFDEC0DEFF76
:104C5800DFC0DEFFE0C0DEFFE1C0DEFFE2C0DEFF56
:104C680081A881AA07D0ED0E806FFE0E816FDAEC65
:104C78005FF008D081BC0AD0220E806FFF0E816FD2
:104C8800DAEC5FF0786A52D7899078D0F34BF42B3E
:104C9800F3C0DBF0F4C0DCF0000EDCBFFF0EDD6F0C
:104CA800DE6FEF51DB5DF051DC59F151DD59F25106
:104CB800DE5901E231D7F951FA115DE07950220D40
:104CC800000EF3245B6E030EF4205C6E2F0E5D6EF7
:104CD800070E5E6EF9C05FF0FAC060F0FC0E616E00
:104CE8005DEC19F00001FE6FFE5101E041D6038230
:104CF800F951D5EC55F00001FC51F527FD51F6238B
:104D0800000EF723F82379501E0D070EF324D96EF1
:104D1800020EF420DA6E000EDE24DB6F010EDE20B8
:104D2800DC6F000EDE20DD6F000EDE20DE6F000E71
:104D3800DE20DF6F000EDE20E06F000EDE20E16F68
:104D4800000EDE20E26F79501E0D070EF324D96E97
:104D5800020EF420DA6EDBC0DEFFDCC0DEFFDDC051
:104D6800DEFFDEC0DEFFDFC0DEFFE0C0DEFFE1C049
:104D7800DEFFE2C0DEFF0392786A86D7899E61D69D
:104D880062C0D9FF63C0DAFFDECF89F0DDCF8AF0D9
:104D9800645065106610671028E120EE0BF0895109
:104DA800D9268A51DA22DECF81F0DECF82F0DECF3B
:104DB80083F0DECF84F081518211831184110FE0DA
:104DC80020EE13F08951D9268A51DA22DE50815D0E
:104DD800DE508259DE508359DE50845952E3010E69
:104DE800816F826B836B846B4CD062C041F063C06F
:104DF80042F064C043F065C044F066C045F067C047
:104E080046F099EC2EF041C08BF042C08CF043C0C4
:104E18008DF044C08EF000018E518D118C1109E186
:104E2800020E8B5D06E2010E626E636A646A656A51
:104E3800000C8B290FE18C290DE18D290BE18E29BE
:104E480009E18BC062F08CC063F08DC064F08EC045
:104E580065F0120020EE13F08951D9268A51DA2222
:104E6800DE508B5DDE508C59DE508D59DE508E59E8
:104E7800E8E364C081F065C082F066C083F067C073
:104E880084F020EE0FF08951D9268A51DA22DE50BB
:104E9800DE10DE10DE1005E1626A636A646A656A24
:104EA8001200856B866B876B886B6450811909E1EA
:104EB8006550821906E1665083197DE167508419AF
:104EC800D8A479D08129856F000E8221866F000EC3
:104ED8008321876F000E8421886F20EE13F089519B
:104EE800D9268A51DA22DE50855DDE508659DE5099
:104EF8008759DE50885905E3020E856F866B876BEC
:104F0800886B62C041F063C042F085C043F086C040
:104F180044F087C045F088C046F099EC2EF041C0B7
:104F28008BF042C08CF043C08DF044C08EF000017D
:104F38008B058C118D118E1184E08B2907E18C294A
:104F480005E18D2903E18E2901E17BD78B518C1175
:104F58008D118E1130E020EE0BF08951D9268A513F
:104F6800DA22DECF8BF0DECF8CF0DECF8DF0DECF15
:104F78008EF08E518D118C1103E1020E8B5D17E3BB
:104F880020EE13F08951D9268A51DA22DE508B5D42
:104F9800DE508C59DE508D59DE508E5908E28BC098
:104FA80081F08CC082F08DC083F08EC084F0856B58
:104FB800866B876B886B855186118711881162E132
:104FC80081C085F082C086F083C087F084C088F0F5
:104FD800852B000E86238723882320EE13F0895122
:104FE800D9268A51DA22DE50855DDE508659DE5098
:104FF8008759DE5088590DE3020E856F866B876BE3
:10500800886B84518311821104E1020E815D01E2F3
:1050180043D762C041F063C042F085C043F086C008
:1050280044F087C045F088C046F099EC2EF041C0A6
:105038008BF042C08CF043C08DF044C08EF000016C
:105048008B518C118D118E111DE08B058C118D11DA
:105058008E1101E1F6D68B2907E18C2905E18D290E
:1050680003E18E2901E1EDD681518519B1E1825123
:105078008619AEE183518719ABE18451881901E1A2
:105088000BD7A6D789C041F08AC042F085C043F04B
:1050980086C044F087C045F088C046F04768486835
:1050A80049684A68E2EC2AF00001806F80511DE1EE
:1050B800645065106610671018E089C041F08AC016
:1050C80042F064C043F065C044F066C045F067C074
:1050D80046F085C047F086C048F087C049F088C0D0
:1050E8004AF0E2EC2AF00001806F805143E120EEA3
:1050F8000BF08951D9268A51DA2285C0DEFF86C095
:10510800DEFF87C0DEFF88C0DEFF20EE0FF089518A
:10511800D9268A51DA2210EE13F08951E1268A51F4
:10512800E222FE0EE6246C6EFF0EE6206D6EFF0E88
:10513800E6206E6EFF0EE6206F6EDE506C5CDE5071
:105148006D58DE506E58DE506F580BE320EE0FF0AE
:105158008951D9268A51DA22DE06000EDE5ADE5A35
:10516800DE5A20EE04F08951D9268A51DA22000E3F
:10517800DB800DD0800507E0010E856F000E866B81
:10518800876B886B04D0856986698769886985C05B
:1051980062F086C063F087C064F088C065F01200D2
:1051A800376E1AC03EF01BC03FF0375001E0040CC8
:1051B800010E3C6E7CB0030CE4D1C2EC5FF0000938
:1051C80001E1F8D13C6AF6D1136A146A156A166AC5
:1051D800090EF7EC5DF0000901E0ECD1270E0A6E2C
:1051E8000B6A0D6A100E0C6EBEEC5AF0000901E154
:1051F800E1D12744E846030BE80647E12EC01CF03E
:105208003F0E1C161CC01DF01E6A1F6A206A1EC0B5
:1052180020F01DC01FF01E6A1D6A2F50226E3050EC
:10522800216E21501D24236E22501E20246E000E54
:105238001F20256E000E2020266E2328386E000EB3
:105248002420396E000E25203A6E000E26203B6E73
:1052580038C01CF039C01DF03AC01EF03BC01FF02A
:105268000A0ED8901C361D361E361F36E82EF9D782
:105278001AC0D9FF1BC0DAFF1CC0DEFF1DC0DEFF4D
:105288001EC0DEFF1FC0DEFF9DD71C6A31AE01D0F5
:105298001C2A010E1C162CC01DF00F0E1D163050B6
:1052A800030B020DF3501D241C24020F3D6E2D50DC
:1052B800030B1C6E1D6A0A0ED8901C361D36E82E8C
:1052C800FBD72E501E6E1F6AD8901E361F36D890F8
:1052D8001E361F362F44E846030B1E24206E000E90
:1052E8001F20216E1C502024226E1D502120236E69
:1052F800222A000E232222C038F023C039F03A6A4D
:105308003B6A3DC01CF0F70E1C2638C01DF039C0A2
:105318001EF03AC01FF03BC020F01C2A05D0D890E0
:105328001D361E361F3620361C2EF9D734D07AA4E7
:105338003FD0136A146A156A166A8D0EF7EC5DF091
:10534800000901E037D124EC60F0270E0A6E0B6AE1
:105358000D6A100E0C6EBEEC5AF0000901E12AD15C
:10536800300E3D6E03D024EC60F03D063D50FBE16D
:1053780031C01CF01C3A0F0E1C16100E1D6E1E6A52
:105388001F6A206A1C2A05D0D8901D361E361F3683
:1053980020361C2EF9D71AC0D9FF1BC0DAFF1DC052
:1053A800DEFF1EC0DEFF1FC0DEFF20C0DEFF0AD703
:1053B800136A146A156A166A090EF7EC5DF000099B
:1053C80001E0F8D0270E0A6E0B6A0D6A100E0C6EFB
:1053D800BEEC5AF0000901E1EDD07AA232D034C017
:1053E8001CF0060E1D6ED8901C321D2EFCD7FF0E29
:1053F8001C2631503F0B1E6E1F6AD8901E361F3672
:105408003244010B1E26000E1F221E2A1F221C2AB0
:1054180003D0D8901E361F361C2EFBD71E50206E88
:105428001F50216E226A236A1AC0D9FF1BC0DAFFF7
:1054380020C0DEFF21C0DEFF22C0DEFF23C0DEFF6A
:10544800C1D63250030B1C6E1D6AD8901C361D360F
:10545800D8901C361D36D8901C361D363238E84296
:10546800070B1C26000E1D221C2A1D223140E84273
:105478003F0B1F0B1E6E1F6A1E2A000E1F221C5098
:105488001E02F3CF20F0F4CF21F01F02F3502126A3
:105498001D501E02F35021262050226E2150236EEB
:1054A800246A256A1AC0D9FF1BC0DAFF22C0DEFFB2
:1054B80023C0DEFF24C0DEFF25C0DEFF83D63EC04A
:1054C800D9FF3FC0DAFF7AC0DFFF7CD6136A146ABF
:1054D800156A166A090EF7EC5DF000096BE13EC02B
:1054E8000AF03FC00BF00D6A100E0C6EBEEC5AF0BD
:1054F800000901E067D65ED0136A146A156A166A55
:105508000A0EF7EC5DF0000955E13EC00AF03FC015
:105518000BF00D6A100E0C6EBEEC5AF0E9D7136A48
:10552800146A156A166A3A0EF7EC5DF0000942E152
:10553800040E3D6E0AD024EC60F03EC0D9FF3FC097
:10554800DAFFDF6E3E4A3F2A3D063D5001E13AD67A
:10555800F2D7136A146A156A166A8D0EF7EC5DF0B5
:10556800000928E124EC60F03EC00AF03FC00BF0CF
:105578000D6A400E0C6EBEEC5AF0BAD7040E3C6EA3
:1055880019D019501C6E1D6A1D50F8E11C5001E11C
:1055980014D6010A01E118D6020A01E1C8D6090A9F
:1055A8008EE0010A93E0070AA7E0010AB8E0030ABF
:1055B800D0E0E4D731EC60F03C501200020E616E8E
:1055C80046504510441004E1020E435C01E2EED15E
:1055D80020EE13F04150D9264250DA22DE50435CC7
:1055E800DE504458DE504558DE50465801E2CBD1D3
:1055F800DDD143C05FF044C060F0D89060304C6E9D
:105608005F304B6E4B505F264C50602241C036F0E5
:1056180042C037F020EE1FF04150D9264250DA221E
:10562800DECF4BF0DECF4CF0DECF4DF0DECF4EF0CC
:105638005FC04FF060C050F0090E516ED8905032E4
:105648004F32512EFBD74F504B24386E50504C20C0
:10565800396E000E4D203A6E000E4E203B6E17EC50
:1056680054F0616E615001E0A1D15F504B6E010EA4
:1056780060144C6E4B5041244D6E4C5042204E6E7F
:105688002F0E4D245D6E000E4E205E6E5F4A602A1E
:1056980043B004D047C059F05A6A1AD047504B6EED
:1056A8004C6A4B3A4C3AF00E4C164B500F0B4C12BE
:1056B800F00E4B165DC0D9FF5EC0DAFFDF500F0B4E
:1056C8004D6E4E6A4B504D10596E4C504E105A6EDE
:1056D8005DC0D9FF5EC0DAFF59C0DFFF20EE03F0DE
:1056E8004150D9264250DA22010EDF6E41C036F011
:1056F80042C037F020EE1FF04150D9264250DA223E
:10570800DECF4BF0DECF4CF0DECF4DF0DECF4EF0EB
:105718005FC04FF060C050F0090E516ED890503203
:105728004F32512EFBD74F504B24386E50504C20DF
:10573800396E000E4D203A6E000E4E203B6E17EC6F
:1057480054F0616E615001E031D15F504B6E010E33
:1057580060144C6E4B5041244D6E4C5042204E6E9E
:105768002F0E4D245D6E000E4E205E6E43B00CD0A1
:1057780048C04BF00F0E4B165DC0D9FF5EC0DAFF74
:10578800DF50F00B4B1012D047C04BF048C04CF024
:1057980049C04DF04AC04EF0050E05D0D8904E32A3
:1057A8004D324C324B32E82EF9D74B505B6E5C6A67
:1057B8005DC0D9FF5EC0DAFF5BC0DFFFDBD041C050
:1057C80036F042C037F020EE1FF04150D926425043
:1057D800DA22DECF4BF0DECF4CF0DECF4DF0DECF5D
:1057E8004EF044504F6E4550506E4650516E526ABE
:1057F8004B504F24386E4C505020396E4D5051202C
:105808003A6E4E5052203B6E17EC54F0616E615068
:1058180001E0CCD043C04BF044C04CF0D8904B369C
:105828004C364B504D6E010E4C144E6E4D5041246B
:105838004F6E4E504220506E2F0E4F240A6E000EAF
:1058480050200B6E47C00CF048C00DF0E9EC5EF03C
:1058580091D041C036F042C037F020EE1FF04150E1
:10586800D9264250DA22DECF4BF0DECF4CF0DECF25
:105878004DF0DECF4EF043C04FF044C050F045C06D
:1058880051F046C052F0080E05D0D890523251322D
:1058980050324F32E82EF9D74B504F24386E4C50C7
:1058A8005020396E4D5051203A6E4E5052203B6E6A
:1058B80017EC54F0616E615079E143C04BF044C07D
:1058C8004CF0D8904B364C36D8904B364C364B5023
:1058D8004D6E010E4C144E6E4D5041244F6E4E507D
:1058E8004220506E2F0E4F240A6E000E50200B6E71
:1058F800D3EC52F0516A526A536AF00E0D14546E8A
:105908004750556E4850566E4950576E0F0E4A1400
:10591800586E51505510476E52505610486E53509D
:105928005710496E545058104A6E43C04BF044C04B
:105938004CF0D8904B364C36D8904B364C364B50B2
:105948004D6E010E4C144E6E4D5041244F6E4E500C
:105958004220506E2F0E4F240A6E000E50200B6E00
:1059680047C00CF048C00DF049C00EF04AC00FF017
:10597800C2EC59F020EE03F04150D9264250DA2209
:10598800010EDF6E13D041C0D9FF42C0DAFFDF50ED
:105998004B6E4C6A4C500AE14B50010A01E129D682
:1059A800030A01E10CD7010A01E153D76150120043
:1059B800796A0101566B796A030E796401D0A8D11E
:1059C800795003E15C6A5D6A03D05D6A010E5C6E22
:1059D80079501E0D1B0EF324D96E020EF420DA6ED8
:1059E800DF6A79501E0D000EF324D96E020EF420E2
:1059F800DA6EDF6A79501E0D070EF324D96E020E97
:105A0800F420DA6E070EDE6AE806FDE20D0E5C028F
:105A1800F3CFA6F0F4CFA7F05D02F3500001A7275B
:105A2800820EA625D96E020EA721DA6EDF50A86F66
:105A3800A8C0A9F0AA6BAB6BAC6BABC0ACF0AAC0AA
:105A4800ABF0A9C0AAF0A96B0D0E5C02F3CFADF0C4
:105A5800F4CFAEF05D02F350AE27810EAD25D96EBE
:105A6800020EAE21DA6EDF50AF6FAFC0B0F0B16B8F
:105A7800B26BB36BB1C0B3F0B0C0B2F0B16BB06B86
:105A88000D0E5C02F3CFB4F0F4CFB5F05D02F35025
:105A9800B527800EB425D96E020EB521DA6EDF5017
:105AA800B66FB6C0B7F0B86BB96BBA6BB7C0BAF01F
:105AB800B96BB86BB76BB051B725BB6FB151B82193
:105AC800BC6FB251B921BD6FB351BA21BE6FA95194
:105AD800BB25BF6FAA51BC21C06FAB51BD21C16F9F
:105AE800AC51BE21C26F0D0E5C02F3CFC3F0F4CFF0
:105AF800C4F05D02F350C427830EC325D96E020E8D
:105B0800C421DA6EDF50BF25C56F000EC021C66FF5
:105B1800000EC121C76F000EC221C86FC5C0C9F0F1
:105B2800C6C0CAF0C7C0CBF0C8C0CCF0CD6BCCBFE4
:105B3800CD69CDC0CEF0CDC0CFF0CDC0D0F079507A
:105B48001E0D0F0EF324D96E020EF420DA6EC9C0B2
:105B5800DEFFCAC0DEFFCBC0DEFFCCC0DEFFCDC09B
:105B6800DEFFCEC0DEFFCFC0DEFFD0C0DEFF795043
:105B78001E0D1C0EF324D96E020EF420DA6EDECF51
:105B8800A6F0DDCFA7F0A6C00AF0A7C00BF00C6AFC
:105B98000D6A0E6A0F6A106A116A79501E0D0F0E8F
:105BA800F324D96E020EF420DA6EDECFA8F0DECF31
:105BB800A9F0DECFAAF0DECFABF0DECFACF0DECFBF
:105BC800ADF0DECFAEF0DECFAFF0A8C012F0A9C0C6
:105BD80013F0AAC014F0ABC015F0ACC016F0ADC0FD
:105BE80017F0AEC018F0AFC019F063EC56F00AC059
:105BF800B0F00BC0B1F00CC0B2F00DC0B3F00EC0E5
:105C0800B4F00FC0B5F010C0B6F011C0B7F07950BD
:105C18001E0D0F0EF324D96E020EF420DA6EB0C0FA
:105C2800DEFFB1C0DEFFB2C0DEFFB3C0DEFFB4C02E
:105C3800DEFFB5C0DEFFB6C0DEFFB7C0DEFF7950BD
:105C48001E0D170EF324D96E020EF420DA6EDE6AEA
:105C5800DE6ADE6A010EDD6E040E0001806FFA0E48
:105C6800816F79C082F0836B79501E0D0F0EF3247B
:105C7800D96E020EF420DA6EDECFA6F0DECFA7F0E2
:105C8800DECFA8F0DECFA9F0DECFAAF0DECFABF0F2
:105C9800DECFACF0DECFADF0A6C084F0A7C085F0B3
:105CA800A8C086F0A9C087F0AAC088F0ABC089F068
:105CB800ACC08AF0ADC08BF079501E0D0F0EF324E6
:105CC800D96E020EF420DA6EDECFAEF0DECFAFF082
:105CD800DECFB0F0DECFB1F0DECFB2F0DECFB3F082
:105CE800DECFB4F0DECFB5F0AEC08CF0AFC08DF033
:105CF800B0C08EF0B1C08FF0B2C090F0B3C091F0D8
:105D0800B4C092F0B5C093F0DAEC5FF0792A54D6BB
:105D18000101596B0001FF6B0101586B446B456B26
:105D2800020E786E576F8990020C41C0D9FF42C0AD
:105D3800DAFFDECF59F0DDCF5AF046504510441057
:105D480003E1020E435C0FE320EE13F05950D9260D
:105D58005A50DA22DE50435CDE504458DE50455833
:105D6800DE50465807E3010E516E000E526A536A20
:105D7800546A71D1516852685368546858D143C005
:105D880057F044C058F0D8905830486E5730476E96
:105D9800475057264850582259C036F05AC037F055
:105DA80020EE1FF05950D9265A50DA22DECF47F09C
:105DB800DECF48F0DECF49F0DECF4AF057C04BF0D7
:105DC80058C04CF0090E4D6ED8904C324B324D2EC7
:105DD800FBD74B504724386E4C504820396E000E84
:105DE80049203A6E000E4A203B6E17EC54F0000929
:105DF80001E031D15750476E010E5814486E475094
:105E08005924496E48505A204A6E2F0E4924D96E9B
:105E1800000E4A20DA6EDF50556E566A574A582AE5
:105E280059C036F05AC037F020EE1FF05950D92625
:105E38005A50DA22DECF47F0DECF48F0DECF49F005
:105E4800DECF4AF057C04BF058C04CF0090E4D6EEB
:105E5800D8904C324B324D2EFBD74B504724386EDE
:105E68004C504820396E000E49203A6E000E4A20E8
:105E78003B6E17EC54F0000901E0EDD05750476E27
:105E8800010E5814486E47505924496E48505A20FC
:105E98004A6E2F0E4924D96E000E4A20DA6EDF5062
:105EA8004C6E4B6A4B5055124C50561243B006D0AC
:105EB80055504F6E0F0E5614506E0FD055C047F008
:105EC80056C048F0040E496ED89048324732492EE1
:105ED800FBD747C04FF048C050F04FC051F050C0FA
:105EE80052F048D059C036F05AC037F020EE1FF0B3
:105EF8005950D9265A50DA22DECF47F0DECF48F083
:105F0800DECF49F0DECF4AF044504B6E45504C6E20
:105F180046504D6E4E6A47504B24386E48504C20C0
:105F2800396E49504D203A6E4A504E203B6E17EC60
:105F380054F0000901E08FD043C047F044C048F056
:105F4800D890473648364750496E010E48144A6E75
:105F5800495059244B6E4A505A204C6E2F0E4B24F0
:105F68000A6E000E4C200B6E49EC5EF00AC051F030
:105F78000BC052F0536A546A6ED059C036F05AC0FA
:105F880037F020EE1FF05950D9265A50DA22DECFCA
:105F980047F0DECF48F0DECF49F0DECF4AF043C00D
:105FA8004BF044C04CF045C04DF046C04EF0080ED2
:105FB80005D0D8904E324D324C324B32E82EF9D7BC
:105FC80047504B24386E48504C20396E49504D206C
:105FD8003A6E4A504E203B6E17EC54F000093BE1F4
:105FE80043C047F044C048F0D89047364836D89068
:105FF800473648364750496E010E48144A6E495094
:1060080059244B6E4A505A204C6E2F0E4B240A6E60
:10601800000E4C200B6ED3EC52F00A50516E0B5010
:10602800526E0C50536E0F0E0D14546E14D059C08E
:10603800D9FF5AC0DAFFDF50476E486A485001E07E
:1060480092D64750010A01E19AD6030A01E14AD7DC
:10605800010A93E088D651C041F052C042F053C0C3
:1060680043F054C044F0120070C0D9FF71C0DAFF89
:10607800DECF9FF0DDCFA0F020EE0EF07050D926D5
:106088007150DA22DECF8FF0DECF90F0DECF91F0C4
:10609800DECF92F0200E00018F259B6F000E90211D
:1060A8009C6F000E91219D6F000E92219E6F9E5154
:1060B80003E1200E9D5D0AE320EE16F07050D9260C
:1060C8007150DA22DE6ADE6ADE6ADD6A20EE16F0D8
:1060D8007050D9267150DA22DE50DE10DE10DE1044
:1060E80001E1040C9B518F6F010E9C15906F916B11
:1060F800926B8F119111921101E027D120EE16F0C9
:106108007050D9267150DA22DE2A000EDE22DE22F5
:10611800DE2220EE12F07050D9267150DA22DE50BD
:10612800DE10DE10DE102CE120EE07F09F51D9269C
:10613800A051DA22DECF8FF0DDCF90F08F51916F32
:106148009051926F936B946B9BC095F09CC096F0A6
:106158009DC097F09EC098F0060E05D0D890983351
:10616800973396339533E82EF9D79151955D92512F
:106178009659935197599451985901E2E6D06ED0A7
:1061880020EE09F09F51D926A051DA22DECF8FF0F8
:10619800DDCF90F0FF0E8F25916FFF0E9021926F4B
:1061A8009BC093F09CC094F09DC095F09EC096F063
:1061B8000A0E05D0D8909633953394339333E82E4E
:1061C800F9D791519315976F92519415986F996BD0
:1061D8009A6B971199119A1101E0B7D070C041F0EC
:1061E80071C042F020EE12F07050D9267150DA22B8
:1061F800DECF43F0DECF44F0DECF45F0DECF46F011
:1062080099EC2EF041C0A1F042C0A2F043C0A3F027
:1062180044C0A4F00001A451A311A21104E1020E8C
:10622800A15D01E2020CA12907E1A22905E1A32948
:1062380003E1A42901E1010C20EE13F09F51D926B6
:10624800A051DA22DE50A15DDE50A259DE50A359DA
:10625800DE50A45950E3725073100BE120EE16F093
:106268007050D9267150DA22DE6ADE6ADE6ADD6A8B
:10627800040C70C062F071C063F020EE12F0705030
:10628800D9267150DA22DECF64F0DECF65F0DECF9A
:1062980066F0DECF67F0C4EC26F062C0A1F063C000
:1062A800A2F064C0A3F065C0A4F0A151A211A3118B
:1062B800A41101E1070CA105A211A311A41101E188
:1062C800020CA12907E1A22905E1A32903E1A429D8
:1062D80001E1010C9FC036F0A0C037F0A1C038F032
:1062E800A2C039F0A3C03AF0A4C03BF032EC4BF0A6
:1062F800000901E0010C20EE12F07050D92671500F
:10630800DA22A1C0DEFFA2C0DEFFA3C0DEFFA4C068
:10631800DEFF9FC00AF0A0C00BF0A1C00CF0A2C025
:106328000DF0A3C00EF0A4C00FF012EC49F020EE5F
:1063380016F07050D9267150DA220AC0DEFF0BC061
:10634800DEFF0CC0DEFF0DC0DEFF20EE0EF0705049
:10635800D9267150DA229BC0DEFF9CC0DEFF9DC0AB
:10636800DEFF9EC0DEFF00019B518F6F010E9C1562
:10637800906F8F519F25916F9051A021926F2F0E92
:106388009127000E922320EE1AF07050D9267150F2
:10639800DA2291C0DEFF92C0DDFF000C5BC0D9FF9E
:1063A8005CC0DAFFDECF73F0DDCF74F0605009E136
:1063B800200E5F5CD8B0020C5DC061F01F0E611644
:1063C80001E0020C20EE0EF05B50D9265C50DA2278
:1063D8005DC0DEFF5EC0DEFF5FC0DEFF60C0DEFFC7
:1063E80020EE06F05B50D9265C50DA22DECF6FF043
:1063F800DECF70F0DECF71F0DECF72F06F5070102C
:106408007110721015E173C0D9FF74C0DAFF020E63
:10641800DF640ED020EE23F07350D9267450DA22B0
:10642800DECF6FF0DECF70F0DECF71F0DECF72F02E
:106438006F5070107110721040E120EE07F0735029
:10644800D9267450DA22DECF61F0DDCF62F06150D8
:10645800636E6250646E656A666A5DC067F05EC0AE
:1064680068F05FC069F060C06AF0060E05D0D89089
:106478006A32693268326732E82EF9D76350675C4E
:10648800645068586550695866506A5801E3020CB0
:1064980020EE23F07350D9267450DA2210EE16F04D
:1064A8005B50E1265C50E222DECFE6FFDECFE6FF5E
:1064B800DECFE6FFDECFE6FF85D020EE09F0735091
:1064C800D9267450DA22DECF61F0DDCF62F0615058
:1064D800636E6250646E656A666A090ED8906336A8
:1064E800643665366636E82EF9D763C06BF064C04B
:1064F8006CF065C06DF066C06EF03FD05BC041F0D7
:106508005CC042F06FC043F070C044F071C045F009
:1065180072C046F099EC2EF041C06FF042C070F0A6
:1065280043C071F044C072F06F2807E1702805E19C
:10653800712803E1722801E1010C7250711070108A
:1065480004E1020E6F5CD8A0020C20EE13F0735029
:10655800D9267450DA22DE506F5CDE507058DE5057
:106568007158DE50725801E3020C6B505D5E6C503E
:106578005E5A6D505F5A6E50605A6B505D5C6C503D
:106588005E586D505F586E506058B8E273C00AF09C
:1065980074C00BF06FC00CF070C00DF071C00EF03D
:1065A80072C00FF012EC49F020EE16F05B50D926BD
:1065B8005C50DA220AC0DEFF0BC0DEFF0CC0DEFF33
:1065C8000DC0DEFF20EE12F05B50D9265C50DA22B7
:1065D8006FC0DEFF70C0DEFF71C0DEFF72C0DEFF7D
:1065E80020EE16F05B50D9265C50DA22DE50DE1021
:1065F800DE10DE1001E1020C5DC061F05EC062F0E9
:106608005FC063F060C064F00A0E05D0D8906432B1
:10661800633262326132E82EF9D720EE16F05B5011
:10662800D9265C50DA226150DE266250DE226350A1
:10663800DE226450DE225D50616E010E5E14626ED1
:1066480061507324636E62507420646E2F0E63264B
:10665800000E642220EE1AF05B50D9265C50DA2234
:1066680063C0DEFF64C0DDFF000C79500C0D0B0E1B
:10667800F324D96E010EF420DA6EDF500001C56FE5
:10668800C5C0C6F0C76BC86BC96B79500C0D000E3E
:10669800F324D96E010EF420DA6EDECFCAF0DDCF16
:1066A800CBF0CAC0CCF0CBC0CDF0000ECDBFFF0EF2
:1066B800CE6FCF6FCC51C603F3CFD0F0F4CFD1F06B
:1066C800D26BD36BC703F350D127F450D223000EFB
:1066D800D323CD51C603F350D127F450D223000E53
:1066E800D323CC51C803F350D227F450D323CD5130
:1066F800C703F350D227F450D323CE51C603F35027
:10670800D227F450D323C951CC03F350D327CD510A
:10671800C803F350D327CE51C703F350D327CF5123
:10672800C603F350D327D0C0D5F0D1C0D6F0D2C01D
:10673800D7F0D3C0D8F0D5C00AF0D6C00BF0D7C078
:106748000CF0D8C00DF079500C0D0A0EF324D96E58
:10675800010EF420DA6EDF50C56FC5C0C6F0C76BF6
:10676800C86BC96BC8C0C9F0C7C0C8F0C6C0C7F0FD
:10677800C66BC6C00EF0C7C00FF0C8C010F0C9C0C5
:1067880011F032EC57F00AC0D5F00BC0D6F00CC0AF
:10679800D7F00DC0D8F079500C0D0B0EF324D96E3C
:1067A800010EF420DA6EDF50C56FC5C0C6F0C76BA6
:1067B800C86BC96B79500C0D020EF324D96E010E0B
:1067C800F420DA6EDF50CA6FCAC0CBF0CC6BCD6B49
:1067D800CE6BCDC0CEF0CCC0CDF0CBC0CCF0CB6B67
:1067E800CB51C603F3CFCFF0F4CFD0F0D16BD26B3F
:1067F800C703F350D027F450D123000ED223CC5135
:10680800C603F350D027F450D123000ED223CB5126
:10681800C803F350D127F450D223CC51C703F35007
:10682800D127F450D223CD51C603F350D127F450C9
:10683800D223C951CB03F350D227CC51C803F3500C
:10684800D227CD51C703F350D227CE51C603F350F8
:10685800D227CF51D527D051D623D151D723D251C2
:10686800D82379500C0D030EF324D96E010EF420B1
:10687800DA6EDF50C56FC5C0C6F0C76BC86BC96B91
:10688800C8C0C9F0C7C0C8F0C6C0C7F0C66BC651FB
:10689800D527C751D623C851D723C951D8237950F2
:1068A800220D000EF324706E030EF420716ED5C015
:1068B80072F0D6C073F0D7C074F0D8C075F088EC09
:1068C8000EF0D46FD45111E0330E806FFB0E816F40
:1068D800D5C082F0D6C083F0D7C084F0D8C085F088
:1068E800D4C086F0876BDAEC5FF0900E0001806F01
:1068F800FE0E816FDAEC5FF0899079500C0D040E72
:10690800F324D96E010EF420DA6ED5C0DEFFD6C0AE
:10691800DEFFD7C0DEFFD8C0DEFF0101536B526B2C
:1069280060EF3AF0000E0001D76F250ED66F000E0B
:10693800D56F050ED46F0101F15105E1000E00017C
:10694800D76F280ED66F01015D510CE1F26B2F0E47
:106958001C6E090E1D6E830E1E6EFE0E1F6EBFECA2
:106968005DF00DD0240E0001806FFA0E816F5DC1BD
:1069780082F0836BF2C184F0856BDAEC5FF0FC0E79
:106988000001806FFD0E816F0101F2510F0D2F0E76
:10699800F3240001826F090EF420836FDAEC5FF0B4
:1069A800050E0001D36F0F0ED26FF10EE82EFED741
:1069B800D22FFCD7D32FFAD7BDD0C00E0B6EFC0E4A
:1069C8000C6EBFEC5EF00101D85144EC60F0000E93
:1069D8000001B96F030EBA6F760EBB6FFE0EBC6F67
:1069E800010EBD6F56EC11F07B6E7B501AEC5BF01C
:1069F8007B5009E1DCEC1BF0000E526E030E536E67
:106A0800DBEC5DF07B6E7B501AEC5BF00001D76B22
:106A1800280ED66F8BD00101F2510F0D2F0EF324E3
:106A2800D96E090EF420DA6E200EDE1806E1F22B7C
:106A38000F0EF2657BD0F26B79D0C10E0001806F2A
:106A4800FB0E816F0101F2510F0D2F0EF32400018F
:106A5800826F090EF420836FDAEC5FF0000E0001FC
:106A6800B96F030EBA6F0101F2510F0D2F0EF32407
:106A78000001BB6F090EF420BC6F030EBD6F56EC0E
:106A880011F07B6E7B501AEC5BF07B5004E1000147
:106A9800D76B3C0ED66F040E7B1804E10001D76B50
:106AA800410ED66F050E0001D36F0F0ED26FF10E97
:106AB800E82EFED7D22FFCD7D32FFAD737D0560ED1
:106AC800806FFC0E816F0101F2510F0D2F0EF32420
:106AD8000001826F090EF420836FDAEC5FF026D094
:106AE800560E806FFC0E816F0101F2510F0D2F0EB3
:106AF800F3240001826F090EF420836FDAEC5FF053
:106B080015D0D6C0D2F0D7C0D3F0D3510FE1D251AF
:106B1800250A01E152D70D0A01E17DD7050A06E0F1
:106B28001F0A04E00E0ACBE07D0ADAE00001D40770
:106B3800D8A0D5070001D5BF08D0D55102E1D405AA
:106B480004E33C0ED619D711DCE1030E01015D19EF
:106B58003BE1899E000E0A6EC00EECEC5BF0D4ECB3
:106B68005EF0000E0A6EC00EECEC5BF03C0E00010D
:106B7800D619D71116E10101E7510CE0E70E0E6EA8
:106B8800010E0F6E33EC58F08B0E0E6EFC0E0F6E6E
:106B980033EC58F0A00E0E6EFF0E0F6E33EC58F06B
:106BA800000C2F0E5B6E090E5C6E510E5D6EFF0EB3
:106BB8005E6E7BC05FF0606A63EC5EF02F0E0E6E57
:106BC800090E0F6E33EC58F0000C1450D96EDA6AC7
:106BD800DECF1CF0DDCF1DF01C0E1224206E000E3F
:106BE8001320216E20C00AF021C00BF00D6A200E80
:106BF8000C6E0F6A0B0E0E6E49EC5FF0226A236A68
:106C08001E6A1F6A1B6A080E1A6E1E501C24156E17
:106C18001F501D20166E15C0F6FF16C0F7FF000E98
:106C2800F86E0F0EF76403D00800F55005D0F6CFC4
:106C3800E9FFF7CFEAFFEF50246E1E4A1F2A210E04
:106C4800246001D0B9D02F0E241806E05C0E241859
:106C580003E035D01E4A1F2A1E501C24156E1F50F3
:106C68001D20166E15C0F6FF16C0F7FF000EF86E51
:106C78000F0EF76403D00800F55005D0F6CFE9FFF2
:106C8800F7CFEAFFEF502F0AE5E01E501C24156EDF
:106C98001F501D20166E15C0F6FF16C0F7FF000E18
:106CA800F86E0F0EF76403D00800F55005D0F6CF44
:106CB800E9FFF7CFEAFFEF505C0A7EE1CBD72E0E53
:106CC800241805E01A50225C1B5023580FE30B0EC2
:106CD8001A181B10D8B4060C2E0E241801E0060C46
:106CE800236A080E226E1B6A0B0E8ED72450EDEC19
:106CF8005AF00A500B1040E01E501C24156E1F500D
:106D08001D20166E15C0F6FF16C0F7FF000EF86EB0
:106D18000F0EF76403D00800F55005D0F6CFE9FF51
:106D2800F7CFEAFFEF50196E1E4A1F2A1950F5ECEB
:106D380057F00A500B10D8B4060CFF0E1A24156E23
:106D4800FF0E1B20166E1550225C1650235801E3C7
:106D5800060C22502024D96E23502120DA6E24C03C
:106D6800DFFF224A232A22502024D96E23502120D3
:106D7800DA6E19C0DFFF1DD0A20E0A6EFD0E0B6E73
:106D880024C00CF00D6A65EC5DF00A500B1001E0B0
:106D9800060C600E246405D07B0E246002D0200E01
:106DA800245E22502024D96E23502120DA6E24C07C
:106DB800DFFF224A232A29D71E501C24156E1F5094
:106DC8001D20166E1450D96EDA6A15C0DEFF16C083
:106DD800DDFF2250231001E1060C20C0D9FF21C09D
:106DE800DAFFE50EDE1806E120C0D9FF21C0DAFF80
:106DF800050EDF6E200E246403D0176A186A03D0CC
:106E0800186A040E176E20EE0BF02050D926215078
:106E1800DA2217C0DFFF000C0F0E7916E20E000110
:106E2800806FF90E816F79C082F0836B79501E0DE7
:106E38001B0EF324D96E020EF420DA6EDF50846F35
:106E4800856BDAEC5FF003822F0E0A6E070E0B6E6D
:106E58000D6A0C6A010E0F6E0E6AAAEC5EF0040E43
:106E6800791804E10F0EE8CF2FF704D027EE2FF0A2
:106E780079C0DFFFFF0EE8CF30F702011B5102E0B7
:106E8800000E0BD0395102E0010E07D0575102E035
:106E9800020E03D0755103E0030EE8CF30F7050E5C
:106EA80079605BD079501E0D1B0EF324D96E020E4B
:106EB800F420DA6EDFA403D0810EE8CF31F77950E1
:106EC8001E0D1B0EF324D96E020EF420DA6EDFA815
:106ED80003D0020EE8CF31F779501E0D1B0EF324B4
:106EE800D96E020EF420DA6EDFA003D0020EE8CFCE
:106EF80033F779501E0D1B0EF324D96E020EF420C1
:106F0800DA6EDFA203D0020EE8CF33F779501E0DF8
:106F18001B0EF324D96E020EF420DA6EDFA603D01E
:106F2800800EE8CF32F779501E0D1B0EF324D96E70
:106F3800020EF420DA6EDFAA03D0040EE8CF31F790
:106F480079501E0D1B0EF324D96E020EF420DA6E52
:106F5800DFAC03D0020EE8CF34F782A403D0080ECA
:106F6800E8CF35F75E6A5F6A300E5E24D96E010E8F
:106F78005F20DA6EDF1C5D6E310E5E24D96E070E5F
:106F88005F20DA6E310E5E24E16E070E5F20E26E3E
:106F9800E7505D14DF6E5E4A5F2A5FBEE5D75F503B
:106FA80003E1070E5E5CE0E3786A020E01015665B4
:106FB80048D079501E0D010EF324D96E020EF4202C
:106FC800DA6EDF505C6E5CC039F779501E0D020E28
:106FD800F324D96E020EF420DA6EDF505C6E5CC0CA
:106FE8003AF779501E0D030EF324D96E020EF420E1
:106FF800DA6EDF505C6E5CC03BF779501E0D040EF4
:10700800F324D96E020EF420DA6EDF505C6E5CC099
:107018003CF779501E0D050EF324D96E020EF420AC
:10702800DA6EDF505C6E5CC03DF779501E0D060EBF
:10703800F324D96E020EF420DA6EDF505C6E5CC069
:107048003EF779501E0D1B0EF324D96E020EF42064
:10705800DA6EDF6A140ED5EC55F0039289901200AF
:10706800696E0001D25102E0DCEC2CF0686A000184
:10707800D15101E1FBD0040E691802E1FF5103E18F
:10708800140E691809E10101586B446B456B000146
:10709800D26B070ED16F070C3F0E691807E1FF6B23
:1070A8000101586B0001D16BD26B12005F0E691899
:1070B80007E10101596B586B0001D16BD26B1200CB
:1070C8003F0E696407D05F0E696004D00101DA5190
:1070D8006918EFE10101DA51691808E1010E596FE9
:1070E8000101586B0001D16BD26B1200DB5169189A
:1070F80004E1010E0001FF6FF3D7650E69180AE17C
:107108000001FF5107E00101446B456B010E586F08
:107118008980E8D76E0E69180AE10001FF5103E182
:107128000101595104E08980020E0101586F700E67
:10713800691807E10101595104E0446B456B030EDE
:10714800586F700E691809E10001FF5106E0898047
:107158000101446B456B040E10D0720E691801E0F2
:1071680085D00001FF5101E181D089800101566B72
:107178001C0E456F2A0E446F050E586FB3D7695021
:107188007FEC04F0686E85D0BC0E441909E1020E4C
:10719800451906E110EC37F00101586B786AA2D75F
:1071A8006950A3EC45F0686E586B73D089802F0E38
:1071B8000A6E070E0B6E0D6A0C6A010E0F6E0E6AD0
:1071C800AAEC5EF0038227EE2FF078C0DFFF010102
:1071D800424B432B4C51421907E14D51431904E1ED
:1071E8004C514D1101E0929C4C51421907E14D510F
:1071F800431904E14C514D1101E09690010ED5EC74
:1072080055F00392080E686E0101586B786A41D0F8
:107218008990686A3ED0080E691815E18990796AE4
:10722800686A786A030E566509D00F0E561906E08B
:10723800010E786E02011B5110091B6F010109D064
:10724800446B456B26D0090E691805E18990686A78
:10725800786A586BF5D71F0E69641BD0300E6960C9
:1072680018D069500F0B566F686AD0D70101585172
:10727800666E676A67500DE166500BE0010A01E12E
:107288007ED7030A81E0010A91E0070AC1E0010AFA
:10729800C2E068C0D1F00001D26B12002F0EEE6F71
:1072A800070EEF6FD4C00AF0D5C00BF0C5EC5CF048
:1072B8000A500001E26FB20E706E716A726A736AE8
:1072C800746A756A88EC0EF0EB6FEB510CE0010EF6
:1072D800806FFB0E816FDAEC5FF00001B26BB36B6D
:1072E800B46BB56B1200B20E5B6E5C6AEEC05DF0FB
:1072F800EFC05EF0010E606E5F6AE90E616E5DECD4
:1073080019F00001EB6FEB5107E0AA0E806FFB0E3E
:10731800816FDAEC5FF0E1D7EEC0D9FFEFC0DAFF9A
:10732800800EDE1807E0AF0E806FFC0E816FDAEC7E
:107338005FF0D3D720EE0AF0EE51D926EF51DA22CA
:10734800DF50D76FD66B20EE0BF0EE51D926EF51F8
:10735800DA22DF50D625E76F000ED721E86F930EAB
:10736800806FFB0E816FE7C082F0E8C083F0DAEC33
:107378005FF0B20E706E716A0001E751D76FD66B7D
:10738800D6C072F0D7C073F0746A756A88EC0EF0D4
:10739800EB6FEB51A2E1B20E5B6E5C6AEEC05DF082
:1073A800EFC05EF0010E606E5F6AE90E616E5DEC23
:1073B80019F00001EB6FEB5190E1EC6BED6BD4C071
:1073C8000AF0D5C00BF0ECC0D6F0EDC0D7F0050E32
:1073D800D890D637D737E82EFBD7D651EE250C6E86
:1073E800D751EF210D6EE2C00EF00F6A75EC57F021
:1073F8000A500B1055E1ECC0D6F0EDC0D7F0050EE1
:10740800D890D637D737E82EFBD7D651EE25D86F88
:10741800D751EF21D96F0E0ED825D96E000ED9217C
:10742800DA6EDF50DB6FDA6BECC0DCF0EDC0DDF05C
:10743800050ED890DC37DD37E82EFBD7DC51EE257A
:10744800DE6FDD51EF21DF6F0F0EDE25D96E000EE6
:10745800DF21DA6EDF50DA25E06F000EDB21E16F05
:10746800E0C0E3F0E1C0E4F0000EE4BFFF0EE56F1A
:10747800E66F840E806FFD0E816FE3C082F0E4C07A
:1074880083F0E5C084F0E6C085F0DAEC5FF0E3C095
:10749800B2F0E4C0B3F0E5C0B4F0E6C0B5F0120055
:1074A800EC4BED2BEDBF8BD7ED5105E10F0EEC5DED
:1074B80001E313D784D711D70001BF6B010EBE6F4C
:1074C800898E8980BA6BBB6BBC6BBD6BDED0795083
:1074D800220D000EF3245B6E030EF4205C6E2F0E5B
:1074E8005D6E070E5E6E010E606E5F6AC20E616EA3
:1074F8005DEC19F00001C46FC45118E0180E0101C9
:10750800516F010E536F0001C36BC26FC00E806FC5
:10751800F90E816F79C082F0836BC4C084F0856BEB
:10752800C2C086F0C3C087F0DAEC5FF001015B519E
:1075380035E0385139113A113B1130E079500C0DD2
:10754800040EF324D96E010EF420DA6E38C1B1F0BE
:1075580039C1B2F03AC1B3F00001B06B000EB025EA
:10756800B46F010EB121B56F000EB221B66F000ED7
:10757800B321B76FDE50B41911E1DE50B5190EE131
:10758800DE50B6190BE1DE50B71908E12F0EAA6FCD
:10759800070EAB6F01015B51A6EC4DF003920101A0
:1075A800515101E003820001C251D5EC55F00001B0
:1075B800C06FC16B010E806FFF0E816FDAEC5FF058
:1075C8000001C051BA27C151BB23000EBC23BD2303
:1075D80081BC81A85FD0C251C01903E1C351C11950
:1075E8000CE0420E806FFE0E816FC0C082F0C1C0F9
:1075F80083F0DAEC5FF089944DD03EEC60F004EC57
:1076080060F00A500B1004E0010E0101536F42D0E4
:107618000001B96B050EB86F1CD0D00E0001AC6F1D
:10762800C90EE82EFED7AC2FFCD700D004EC60F0D2
:107638000A500B100EE00001BE6BBF6B040E806F8A
:10764800FD0E816FB8C082F0B9C083F0DAEC5FF04C
:1076580008D00001B807D8A0B907B829DEE1B929D0
:10766800DCE181B80AD0360E0001806FFF0E816F11
:10767800DAEC5FF00001BE6BBF6B04EC60F00A50FF
:107688000B1003E00001BE6BBF6B0001BE51BF11C0
:1076980001E01DD70101536B899E89901200898EE4
:1076A8008980786A31EC3DF00101966F965102E0CD
:1076B80096511200636B8E6B8F6B906B916B946B12
:1076C800010E936F996BD0D0976B986B1CD004EC1C
:1076D80060F00A500B1015E0990E0A6E010E0B6E41
:1076E8008EEC5FF00101926F000E6325D96EDA6AA5
:1076F800040EDA2292C1DFFF632B974B982B99BBBC
:1077080005D081AC03D001019805E1E3010197514F
:107718008E2798518F23000E9023912379501E0DA8
:10772800170EF324D96E020EF420DA6EDE508E5D49
:10773800DE508F59DE509059DE50915902E3936B19
:10774800946B99AB02D0936B946B81BC02D0936B12
:10775800946B980519E2000E63250A6E0B6A040EF5
:107768000B22FF0E6325D96EDA6A030EDA22DF5088
:107778000C6E0D6A635100080E6E000ED8A0E82A40
:1077880001080F6EAAEC5EF001015B5145E038512B
:1077980039113A113B1140E079503EE179501E0D04
:1077A800070EF324D96E020EF420DA6E38C183F185
:1077B80039C184F13AC185F1826B000E8225866F4A
:1077C800010E8321876F000E8421886F000E8521AA
:1077D800896F8A6B8B6B8C6B8D6BDE5086191CE105
:1077E800DE50871919E1DE50881916E1DE50891933
:1077F80013E1DE508A1910E1DE508B190DE1DE50DD
:107808008C190AE1DE508D1907E1000E216E040E75
:10781800226E5B511CEC56F0ABEC4AF00101956FFF
:10782800636B955121E04B0E0001806FFB0E816F59
:1078380095C182F0836BDAEC5FF0010E786E7950B7
:107848001E0D1B0EF324D96E020EF420DA6E795049
:107858001E0D1B0EF324E16E020EF420E26EE750BB
:107868000409DF6E785012009351941101E02CD76F
:1078780082A402D0010E786E8990899E000C81A6A0
:1078880005D08A0E0001A66FFC0E04D0BA0E0001C6
:10789800A66FFF0EA76F81AA04D08A0EA86FFC0EF0
:1078A80003D0B50EA86FFF0EA96F81A804D08A0E69
:1078B800AA6FFC0E03D0D20EAA6FFE0EAB6F81AE7C
:1078C80004D08A0EAC6FFC0E03D0BF0EAC6FFF0E57
:1078D800AD6F81AC04D08A0EAE6FFC0E03D0B00E33
:1078E800AE6FFF0EAF6F81A404D08A0EB06FFC0E8E
:1078F80003D0C90EB06FFF0EB16F81A204D08A0EFB
:10790800B26FFC0E03D0CE0EB26FFF0EB36F81A024
:1079180004D08A0EB46FFC0E03D0C40EB46FFF0EF1
:10792800B56F83AE04D08A0EB66FFC0E03D0FC0E82
:10793800B66FFF0EB76F83AC04D08A0EB86FFC0E1B
:1079480003D0F90EB86FFF0EB96F83AA04D08A0E60
:10795800BA6FFC0E03D0F60EBA6FFF0EBB6F83A88A
:1079680004D08A0EBC6FFC0E03D0F30EBC6FFF0E62
:10797800BD6F83A604D08A0EBE6FFC0E03D0F00E36
:10798800BE6FFF0EBF6F83A404D08A0EC06FFC0EBB
:1079980003D0ED0EC06FFF0EC16F83A204D08A0E14
:1079A800C26FFC0E03D0EA0EC26FFF0EC36F83A036
:1079B80004D08A0EC46FFC0E03D0E70EC46FFF0E0E
:1079C800C56FAE0E806FF80E816F831C826F836B5C
:1079D80081CF84F0856BC4C086F0C5C087F0C2C073
:1079E80088F0C3C089F0C0C08AF0C1C08BF0BEC0A7
:1079F8008CF0BFC08DF0BCC08EF0BDC08FF0BAC097
:107A080090F0BBC091F0B8C092F0B9C093F0B6C086
:107A180094F0B7C095F0B4C096F0B5C097F0B2C076
:107A280098F0B3C099F0B0C09AF0B1C09BF0AEC066
:107A38009CF0AFC09DF0ACC09EF0ADC09FF0AAC056
:107A4800A0F0ABC0A1F0A8C0A2F0A9C0A3F0A6C046
:107A5800A4F0A7C0A5F0DAEF5FF079501E0D070E6D
:107A6800F324D96E020EF420DA6EDECFD6F0DECF24
:107A7800D7F0DECFD8F0DECFD9F079501E0D070E43
:107A8800F324D96E020EF420DA6E79501E0D0F0E13
:107A9800F324E16E020EF420E26EDE50E65CDE5066
:107AA800E658DE50E658DE50E658DE50E658DE501E
:107AB800E658DE50E658DE50E65815E2010E786EBC
:107AC80079501E0D1B0EF324D96E020EF420DA6EC7
:107AD80079501E0D1B0EF324E16E020EF420E26EA7
:107AE800E7500409DF6E79501E0D070EF324D96E96
:107AF800020EF420DA6EDECFB2F0DECFB3F0DECFC6
:107B0800B4F0DECFB5F0DECFB6F0DECFB7F0DECF23
:107B1800B8F0DECFB9F079501E0D170EF324D96EE8
:107B2800020EF420DA6EDECFBAF0DECFBBF0DECF85
:107B3800BCF0DECFBDF00001BA51BE6FBB51BF6FC4
:107B4800BC51C06FBD51C16FC26BC36BC46BC56BF9
:107B5800B251BE25C66FB351BF21C76FB451C02102
:107B6800C86FB551C121C96FB651C221CA6FB7518B
:107B7800C321CB6FB851C421CC6FB951C521CD6F8A
:107B880079501E0D0F0EF324D96E020EF420DA6E12
:107B9800C651DE5CC751DE58C851DE58C951DE589F
:107BA800CA51DE58CB51DE58CC51DE58CD51DE5883
:107BB80015E2010E786E79501E0D1B0EF324D96E56
:107BC800020EF420DA6E79501E0D1B0EF324E16EBE
:107BD800020EF420E26EE7500409DF6E786A7950ED
:107BE800220D000EF324706E030EF420716ED6C0C1
:107BF80072F0D7C073F0D8C074F0D9C075F088ECB3
:107C08000EF0DA6FDA5115E0010E786E79501E0D1C
:107C18001B0EF324D96E020EF420DA6E79501E0D75
:107C28001B0EF324E16E020EF420E26EE750040905
:107C3800DF6E78501200070E0A24196E000E0B2012
:107C48001A6E0AC0D9FF0BC0DAFFDF500E6E0E386D
:107C58000F0B0A0DF3CF0FF0F4CF10F00AC0D9FFC5
:107C68000BC0DAFFDF500F0B0F26000E10220F2873
:107C7800176E000E1020186E1C6A010E1B6E1D6A0E
:107C88001E6A1F6A206AB2D01B501C1054E01DC027
:107C98000EF01EC00FF01FC010F020C011F00A0E29
:107CA8000E02F3CF12F0F4CF13F0146A156A0F0224
:107CB800F3501326F4501422000E15220E02F3502E
:107CC8001326F4501422000E15220A0E1002F35047
:107CD8001426F4501522000E0F02F3501426F45007
:107CE8001522000E0E02F3501426F45015220A0E27
:107CF8001102F3501526000E1002F3501526000E3F
:107D08000F02F3501526000E0E02F350152619C067
:107D1800D9FF1AC0DAFFDF50166E16380F0B12247F
:107D28001D6E000E13201E6E000E14201F6E000E16
:107D38001520206E54D01DC00EF01EC00FF01FC0BD
:107D480010F020C011F00A0E0E02F3CF12F0F4CF9B
:107D580013F0146A156A0F02F3501326F450142214
:107D6800000E15220E02F3501326F4501422000EB2
:107D780015220A0E1002F3501426F4501522000E94
:107D88000F02F3501426F4501522000E0E02F35081
:107D98001426F45015220A0E1102F3501526000E6F
:107DA8001002F3501526000E0F02F3501526000E90
:107DB8000E02F350152619C0D9FF1AC0DAFFDF509A
:107DC8000F0B12241D6E000E13201E6E000E1420C1
:107DD8001F6E000E1520206E1906D8A01A061B501B
:107DE8001C10010ED8A4000E1B6E1C6A1706D8A022
:107DF8001806172802E11828D8A446D71DC00AF08B
:107E08001EC00BF01FC00CF020C00DF0120040C0C7
:107E180023F041C024F00CEC43F04A6E4A5001E0D4
:107E2800D2D040C0D9FF41C0DAFF030EDE1801E00E
:107E3800BAD020EE04F04050D9264150DA22DE04B0
:107E480001E0B1D02F0E40240A6E000E41200B6EC7
:107E58000D6A0C6A020E0F6E0E6A49EC5FF02D0E69
:107E680040240A6E020E41200B6EAA0E0D6E550EAE
:107E78000C6EE9EC5EF02F0E40240A6E000E4120D5
:107E88000B6E520E0C6E0D6E610E0E6E410E0F6E65
:107E9800C2EC59F0130E40240A6E020E41200B6EFC
:107EA800720E0C6E0D6E410E0E6E610E0F6EC2ECF0
:107EB80059F0170E40240A6E020E41200B6E20EE78
:107EC8000FF04050D9264150DA22DECF0CF0DECF39
:107ED8000DF0DECF0EF0DECF0FF0C2EC59F01B0E26
:107EE80040240A6E020E41200B6E20EE0BF040502B
:107EF800D9264150DA22DECF0CF0DECF0DF0DECFEE
:107F08000EF0DECF0FF0C2EC59F020EE1BF040501F
:107F1800D9264150DA22DECF42F0DECF43F0DECF61
:107F280044F0DECF45F04228466E000E4320476EEF
:107F3800000E4420486E000E4520496E20EE2BF0BE
:107F48004050D9264150DA2246C0DEFF47C0DEFF46
:107F580048C0DEFF49C0DEFF2F0E4024196E000E18
:107F680041201A6E20EE2BF04050D9264150DA22DB
:107F7800DECF1BF0DECF1CF0DECF1DF0DECF1EF013
:107F8800206A010E1F6E20EE01F04050D9264150A4
:107F9800DA22DF5098EC4EF020EE04F04050D9265B
:107FA8004150DA22DF6A196A1A6A1B6A20EE01F068
:107FB8004050D9264150DA22DF50D4EC28F000098D
:107FC80002E0010E4A6E4A5012005B51D8B412000A
:107FD800340E0001806FFD0E816FDAEC5FF079ECF2
:107FE80053F0A6C0F6F0A7C0F7F0A8C0F8F0A9C0F3
:107FF800F9F00001F651F711F811F91116E1EF0E39
:10800800806FFB0E816FF6C082F0F7C083F0F8C076
:1080180084F0F9C085F0DAEC5FF00A0E0D6E000E00
:108028000E6A0F6A106A9AEC5BF00001FA6BFB6B40
:10803800E30E806FFF0E816FFA51F60FD96EDA6A80
:10804800DF50826F836BDAEC5FF00001FA4BFB2B99
:10805800FBBFEED7FB5103E1040EFA5DE9E32A0EFC
:10806800806FF90E816FDAEC5FF0CD0E0001806F42
:10807800FA0E816FDAEC5FF023EE00F000EEB2F05A
:10808800210EDBCFEBFFE806FCE2D70E0001D46F30
:10809800FF0ED56F52EC39F0B2C038F1B3C039F1E8
:1080A800B4C03AF1B5C03BF10101385139113A1168
:1080B8003B11D8B41200B30E0001806FFA0E816F25
:1080C80038C182F039C183F03AC184F03BC185F0F0
:1080D800DAEC5FF0000E706E030E716E38C1F1F0CD
:1080E80039C1F2F03AC1F3F00001F06B000EF0254F
:1080F800726E010EF121736E000EF221746E000E85
:10810800F321756E88EC0EF07B6E000E5B6E030E2D
:108118005C6E2F0E5D6E070E5E6E606A080E5F6EF7
:10812800F40E616E5DEC19F07B6E0001FC6BFD6B6B
:10813800AB0E806FFC0E816F2F0EFC25D96E070EDB
:10814800FD21DA6EDF50826F836BDAEC5FF000019D
:10815800FC4BFD2BFDBFECD7FD5105E1080EFC5D86
:10816800D8B01200E5D7120062C0D9FF63C0DAFFA9
:10817800DECF85F0DDCF86F067506610651004E12C
:10818800020E645CD8A0020C000120EE13F08551A9
:10819800D9268651DA22DE50645CDE506558DE50FE
:1081A8006658DE50675801E3020C685069106A107F
:1081B8006B1018E085C041F086C042F068C043F0FB
:1081C80069C044F06AC045F06BC046F0476848682B
:1081D80049684A68E2EC2AF00001846F845102E0A1
:1081E8008451120062C041F063C042F064C043F0A1
:1081F80065C044F066C045F067C046F099EC2EF0C3
:1082080041C080F042C081F043C082F044C083F096
:108218000001805181118211831171E08005811163
:108228008211831101E1020C802907E1812905E10E
:10823800822903E1832901E1010C85C041F086C050
:1082480042F064C043F065C044F066C045F067C0C2
:1082580046F0476A486A496A4A6AE2EC2AF000012D
:10826800846F8451BDE120EE13F08551D9268651E3
:10827800DA22FE0EDE246C6EFF0EDE206D6EFF0E1F
:10828800DE206E6EFF0EDE206F6E20EE0FF0855141
:10829800D9268651DA226C50DE5C6D50DE586E505D
:1082A800DE586F50DE5813E220EE0FF08551D926C4
:1082B8008651DA22DE2A000EDE22DE22DE2220EEBF
:1082C80004F08551D9268651DA22000EDB8080C061
:1082D80064F081C065F082C066F083C067F020EE6C
:1082E80013F08551D9268651DA22DE50645CDE50BF
:1082F8006558DE506658DE50675801E273D7000CA7
:10830800ABC0D9FFACC0DAFFDECFB5F0DDCFB6F039
:1083180003D00001AD4BAE2BADC0F6FFAEC0F7FFEA
:10832800000EF86E0F0EF76403D00800F55005D064
:10833800F6CFE9FFF7CFEAFFEF502F0AEAE0ADC02A
:10834800F6FFAEC0F7FF000EF86E0F0EF76403D00D
:108358000800F55005D0F6CFE9FFF7CFEAFFEF5058
:108368005C0AD7E0000120EE06F0AB51D926AC51EB
:10837800DA22DE6ADE6ADE6ADD6AADC0F6FFAEC00A
:10838800F7FF000EF86E0F0EF76403D00800F550E3
:1083980005D0F6CFE9FFF7CFEAFFEF500001AF6F46
:1083A800200EAF6115D020EE27F0AB51D926AC5185
:1083B800DA22800EDF6EABC05BF0ACC05CF0000E62
:1083C8005D6E5E6E5F6E606ED2EC31F0000123D0A0
:1083D800ABC012F0ACC013F0AD0E146EE9EC35F082
:1083E8000001B86FB85154E1ABC075F0ACC076F07D
:1083F800F5EC47F0B86F20EE27F0AB51D926AC5119
:10840800DA22DF50B76FB85108E0040EB81940E11E
:10841800B7B53ED0050EB86F3BD0B7B539D020EE12
:1084280004F0AB51D926AC51DA22DFA8F3D7B5C096
:1084380011F0B6C012F020EE0EF0AB51D926AC51B7
:10844800DA22DECFAFF0DDCFB0F0AF51B16F010E61
:10845800B015B26FB151B525B36FB251B621B46F33
:108468002F0EB325136E000EB421146EABEC58F02A
:10847800000120EE06F0AB51D926AC51DA2211C02A
:10848800DEFF12C0DEFF13C0DEFF14C0DEFFA0D780
:10849800B85112001A6E1A5001E0010C7CA202D0E9
:1084A8007C501200000EA9EC5FF00A0E256E03D076
:1084B80024EC60F025062550FBE1226A000E136AC1
:1084C800146A156A166AF7EC5DF0E80601E097D0C1
:1084D800AA0E136E010E146E156A166A080EF7ECD2
:1084E8005DF0E80651E1256A25501B0FD96EDA6A5E
:1084F80024EC60F0DF6E252A030E2564F5D71D04F1
:108508007EE1AA0E1E187BE1030E246EE80E236E90
:1085180015D0136A146A156A400E166EA90EF7EC88
:108528005DF000090EE0150E196EC60EE82EFED796
:10853800192EFCD700D02306D8A0240623502410D7
:10854800E8E1235024105BE0136A146A156A166A7E
:108558003A0EF7EC5DF0000952E1256A25501B0F31
:10856800D96EDA6A24EC60F0DF6E252A030E2564E2
:10857800F5D71BBC03D0206A040E02D0206A0C0E6B
:108588001F6E1FC022F03BD0136A146A156A166A60
:10859800A90EF7EC5DF0196E020E196003D0226E79
:1085A800A90E02D0010E226E216E030E246EE80E73
:1085B800236E14D0136A146A156A166A2150F7ECF0
:1085C8005DF000090EE0150E196EC60EE82EFED7F6
:1085D800192EFCD700D02306D8A024062350241037
:1085E800E9E1235024100AE0136A020E146E156A9A
:1085F800166A100EF7EC5DF0000901E0226A22C04D
:108608007AF031EC60F0225001E14AD77C9048D7EB
:10861800356A20EE03F02350D9262450DA22DF50A1
:1086280001E1A7D02F0E2324196E000E24201A6E04
:1086380020EE2BF02350D9262450DA22DECF1BF06F
:10864800DECF1CF0DECF1DF0DECF1EF0206A010E5B
:108658001F6E20EE01F02350D9262450DA22DF5075
:1086680098EC4EF0000901E082D020EE03F0235090
:10867800D9262450DA22DF6A20EE17F02350D926B3
:108688002450DA2210EE1FF02350E1262450E22273
:10869800E6CF29F0E6CF2AF0E6CF2BF0E6CF2CF094
:1086A80010EE2BF02350E1262450E222E6CF2DF0E5
:1086B800E6CF2EF0E6CF2FF0E6CF30F029502D5C34
:1086C800316E2A502E58326E2B502F58336E2C5044
:1086D8003058346EDE50315CDE503258DE5033583C
:1086E800DE50345846E220EE02F02350D9262450BA
:1086F800DA22020EDE183DE12F0E2324196E000E39
:1087080024201A6E20EE17F02350D9262450DA229E
:10871800DECF25F0DECF26F0DECF27F0DECF28F043
:1087280020EE2BF02350D9262450DA22DECF29F070
:10873800DECF2AF0DECF2BF0DECF2CF02550292417
:108748001B6E26502A201C6E27502B201D6E285089
:108758002C201E6E206A010E1F6E20EE01F02350A1
:10876800D9262450DA22DF5098EC4EF002D0010EC0
:10877800356E3550120093689568F29E81280BE19A
:108788001A0E0001806FFB0E816F81CF82F0836B20
:10879800DAEC5FF00AD0780E0001806FF90E816F75
:1087A80081CF82F0836BDAEC5FF083280BE1D80E7F
:1087B8000001806FFB0E816F81CF82F0836BDAEC52
:1087C8005FF00AD09D0E0001806FF90E816F81CF96
:1087D80082F0836BDAEC5FF0290E5D6E960E5C6EAC
:1087E8007F0EE82EFED75C2EFCD75D2EFAD7000050
:1087F8005C0E0001806FFE0E816FDAEC5FF09398DB
:108808008A98090E5D6E1E0E5C6EE40EE82EFED789
:108818005C2EFCD75D2EFAD700D04F0E0001806F7A
:10882800FE0E816FDAEC5FF0939A8A9A090E5D6EFC
:108838001E0E5C6EE40EE82EFED75C2EFCD75D2E75
:10884800FAD700D0C00E0001806FFE0E816FDAECFF
:108858005FF09290809083280BE0D80E0001806F23
:10886800FB0E816F83CF82F0836BDAEC5FF00AD066
:108878002D0E0001806FF90E816F83CF82F0836B1C
:10888800DAEC5FF08080A30E5D6E570E5C6E020E10
:10889800E82EFED75C2EFCD75D2EFAD700D0936861
:1088A8009568946889928982290E5D6E960E5C6E31
:1088B8007F0EE82EFED75C2EFCD75D2EFAD700007F
:1088C80043EC3CF0EFD74BC00BF04CC00CF04E0E15
:1088D8000D6E7DEC52F04D6E4D5001E093D020EEC0
:1088E8000EF04B50D9264C50DA22DFAC8BD04EC05C
:1088F80036F04FC037F020EE1CF04B50D9264C50C4
:10890800DA22DECF38F0DECF39F0DECF3AF0DECF34
:108918003BF017EC54F04D6E4D5074E120EE20F012
:108928004B50D9264C50DA22DECF50F0DDCF51F033
:1089380020EE0BF05050D9265150DA22000EDB8A77
:108948004BC0D9FF4CC0DAFFDECF0EF0DDCF0FF001
:1089580050C010F051C011F020EE06F04B50D9264F
:108968004C50DA22DECF12F0DECF13F0DECF14F057
:10897800DECF15F026EC5DF01C0E50240A6E000EBA
:1089880051200B6E20EE0AF04B50D9264C50DA22BB
:10899800DECF0CF0DECF0DF0DECF0EF0DECF0FF025
:1089A800C2EC59F0160E50240A6E000E51200B6EC0
:1089B8000C6A0D6A210E0E6E500E0F6EC2EC59F045
:1089C800120E50240A6E000E51200B6E000E0D6A16
:1089D8000C6AE9EC5EF020EE03F04E50D9264F50B9
:1089E800DA22010EDF6E4EC040F04FC041F00BECB2
:1089F8003FF04D6E20EE0EF04B50D9264C50DA2247
:108A0800BF0EDF164D501200136814680A50D96E55
:108A1800DA6ADECF15F0DDCF16F015C010F016C0FB
:108A280011F01550161003E10A680B68120010C007
:108A3800F6FF11C0F7FF000EF86E0F0EF76403D0B3
:108A48000800F55005D0F6CFE9FFF7CFEAFFEF5061
:108A5800126E104A112A200E126403D03A0E121810
:108A6800E6E13A0E121868E1000E0F6E010E0E6E66
:108A780015C0F6FF16C0F7FF000EF86E0F0EF7646C
:108A880003D00800F55005D0F6CFE9FFF7CFEAFF8D
:108A9800EF500C6E2F0E0C6439D015C0F6FF16C0BF
:108AA800F7FF000EF86E0F0EF76403D00800F550BC
:108AB80005D0F6CFE9FFF7CFEAFFEF500C6E3A0E7C
:108AC8000C6024D0020E15240C6E000E16200D6EBC
:108AD80010500C181BE111500D1818E115C0F6FFC5
:108AE80016C0F7FF000EF86E0F0EF76403D00800EB
:108AF800F55005D0F6CFE9FFF7CFEAFFEF500C6E3F
:108B0800D00E0C240E6E0F6AFF0E0F220FBE04D07B
:108B18000F500DE10E040BE20EC013F00FC014F05D
:108B28000A50D96EDA6A10C0DEFF11C0DDFF13C02B
:108B38000AF014C00BF012000A6A0B6A120064688B
:108B4800930E0001806FFD0E816F44C182F045C114
:108B580083F042C184F043C185F0DAEC5FF089808C
:108B680003D02D0E1CEC60F081A881AA03D0640606
:108B78006428F7E179501E0D070EF324D96E020E12
:108B8800F420DA6EDECF5CF0DECF5DF0DECF5EF093
:108B9800DECF5FF0DECF60F0DECF61F0DECF62F0D7
:108BA800DECF63F05CC00BF05DC00CF05EC00DF072
:108BB8005FC00EF060C00FF061C010F062C011F02D
:108BC80063C012F0C9EC53F00D0E1CEC60F00A0EF5
:108BD8001CEC60F001014C51421907E14D51431959
:108BE80004E14C514D1101E0929C4C51421918E19D
:108BF8004D51431915E14C514D1112E0969010D08A
:108C0800030E0AD0050E656E446B456B2ED00A0E16
:108C180003D0010E01D0020E656E27D0656A25D0FB
:108C280044C15CF045C15DF05D5009E0020A0EE008
:108C38000E0A10E0010A12E02A0A14E0EFD75C508D
:108C4800DFE00A0ADDE01E0ADDE0E8D75C50BC0A76
:108C5800E2E0E4D75C501C0ADAE0E0D75C50AC0AEA
:108C6800D8E0DCD75C500F0AD9E1655012002F6CB0
:108C7800696664617461302E62696E20002F6C69C8
:108C88006664617461312E62696E20002F6C6966BA
:108C980064617461322E62696E20002F6C696664AB
:108CA800617461332E62696E20002F6C696664619D
:108CB8007461342E62696E20002F6C696664617479
:108CC80061352E62696E20002F6C6966646174617B
:108CD800362E62696E20002F6C6966646174613794
:108CE8002E62696E20002F6C696664617461382E8B
:108CF80062696E20002F6C696664617461392E6246
:108D0800696E20002F6C696664617461612E626906
:108D18006E20002F6C696664617461622E62696EF0
:108D280020002F6C696664617461632E62696E202D
:108D3800002F6C696664617461642E62696E20003C
:108D48002F6C696664617461652E62696E20002FFC
:108D58006C696664617461662E62696E2000000049
:108D680000000000000000000000000000000000FB
:108D780000000000000000000000000000000000EB
:108D880000000000000000000000000000000000DB
:108D98000000000000000000000048C041F049C089
:108DA80042F0436A446A456A466A32EC4CF041C074
:108DB80060F042C061F0020E601861100DE0615071
:108DC80006E1030E605C03E24A504B1005E160C007
:108DD80048F061C049F01200626A636A62C04CF0F0
:108DE80063C04DF04C3A4D3AF00E4D164C500F0BF7
:108DF8004D12F00E4C164C5048244E6E4D504920E2
:108E08004F6EF50E4E240A6E010E4F200B6ED3ECFA
:108E180052F06250040DF350500FD96EDA6A0AC04E
:108E2800DEFF0BC0DEFF0CC0DEFF0DC0DEFF624AB6
:108E3800632A635003E1040E625CD0E34A504B108E
:108E480003E1626A636A06D0FF0E4A24626EFF0E6F
:108E58004B20636E6250040DF350500FD96EDA6ADE
:108E6800DE50DE10DE10DE1004E1616A030E606E73
:108E780018D048C041F049C042F06250040DF35088
:108E8800500FD96EDA6ADECF43F0DECF44F0DECF82
:108E980045F0DECF46F032EC4CF041C060F042C005
:108EA80061F04A504B1093E1615003E1020E605C9F
:108EB8008EE3624A632A63508AE1040E625C87E2A9
:108EC800C9D7F2C15EF07CD05CEC5FF05E6EF2193F
:108ED80001E185D0290E5D6E960E5C6E7F0EE82E40
:108EE800FED75C2EFCD75D2EFAD7000078D03AEC7E
:108EF8005CF05F6E5F5073E05FA002D001015A2BF7
:108F08005FA202D001015A070F0E01015A17000E85
:108F18000A6EC00EECEC5BF0D4EC5EF0000E0A6E4C
:108F2800C00EECEC5BF001015A510F0D2F0EF3242B
:108F38000E6E090EF4200F6E33EC58F0110E5D6EB4
:108F48003C0E5C6ECB0EE82EFED75C2EFCD75D2E59
:108F5800FAD700005FA443D0070E5F1840E00B6A01
:108F68000A6A5AC10CF0A2EC5DF01B0E0001806F7A
:108F7800FC0E816F5AC182F0836BDAEC5FF05AC144
:108F88005EF0000E0A6E800EECEC5BF0D4EC5EF046
:108F9800000E0A6E800EECEC5BF001015A510F0DC9
:108FA8002F0EF3240E6E090EF4200F6E33EC58F0DA
:108FB800000E0A6EC00EECEC5BF0D4EC5EF00FD045
:108FC80001015D515C6E5D6A5D5009E15C50010A0A
:108FD80001E17AD7030A01E177D7010A88E05E50F8
:108FE800120075C0D9FF76C0DAFFDECFA7F0DDCF5B
:108FF800A8F075C05BF076C05CF0000E5D6E5E6E2A
:109008005F6E606ED2EC31F00001AA6FAA5103E0E6
:109018000001AA511200A7C036F0A8C037F020EE10
:1090280016F07550D9267650DA22DECF38F0DECF2A
:1090380039F0DECF3AF0DECF3BF017EC54F0000108
:10904800AA6FAA51E5E120EE1AF07550D92676509C
:10905800DA22DECFA5F0DDCFA6F0A5C0D9FFA6C0E5
:10906800DAFFDF50A96FA95103E1040EAA6FD0D728
:1090780020EE04F07550D9267650DA2210EE1AF058
:109088007550E1267650E22200EE0BF0E650E92614
:10909800E550EA22EF503F0BDF6E20EE1AF07550D4
:1090A800D9267650DA2210EE0BF0DE50E126DD509C
:1090B800E222E7B618D020EE1AF07550D92676507D
:1090C800DA22DECF0AF0DDCF0BF01C0E75240C6E11
:1090D800000E76200D6E0F6A0B0E0E6E8CEC59F09A
:1090E8000A500B1095E075C070F076C071F0736A85
:1090F800726A38EC30F00001AA6FAA5189E18BD767
:1091080017C00AF018C00BF00D6A0C6A0F6A080E37
:109118000E6EAAEC5EF0226A020E216E2150172410
:10912800D96E22501820DA6E215017241D6E225055
:1091380018201E6E1D28E16E000E1E20E26EE750FC
:109148001F6E1F3AF00E1F161F1621501724E16ECE
:1091580022501820E26EE750206E20380F0B1F10A7
:10916800DF6E214A222A22BED9D7225003E1070EF8
:10917800215CD4E321501724D96E22501820DA6ECE
:1091880019C00AF01AC00BF01BC00CF01CC00DF07F
:109198000A0E0E6E0F6A106A116A5DEC5AF00A3AEE
:1091A800F00E0A1621501724E16E22501820E26EA4
:1091B800E7501D6E1D380F0B0A10DF6E17C0D9FF60
:1091C80018C0DAFFDF2A19C00AF01AC00BF01BC05A
:1091D8000CF01CC00DF00A0E0E6E0F6A106A116AB0
:1091E80070EC58F00AC019F00BC01AF00CC01BF054
:1091F8000DC01CF019501A101B101C108CE117C060
:10920800D9FF18C0DAFFDF06090EDF64090C17C0A2
:10921800D9FF18C0DAFF100EDF6E100C020E0C5EBC
:10922800000E0D5A0E5A0F5A20EE13F00A50D92686
:109238000B50DA22FE0EDE24106EFF0EDE20116EB9
:10924800FF0EDE20126EFF0EDE20136E10500C5C37
:1092580011500D5812500E5813500F5805E30A6A52
:109268000B6A0C6A0D6A120020EE27F00A50D92604
:109278000B50DA22DECF10F0DECF11F0DECF12F085
:10928800DECF13F020EE09F00A50D9260B50DA226F
:10929800DECF14F0DDCF15F01450166E1550176E92
:1092A800186A196A16500C02F3CF1AF0F4CF1BF0A3
:1092B8001C6A1D6A0D02F3501B26F4501C22000E76
:1092C8001D2217500C02F3501B26F4501C22000ECE
:1092D8001D2216500E02F3501C26F4501D22175062
:1092E8000D02F3501C26F4501D2218500C02F350A6
:1092F8001C26F4501D220F501602F3501D2617503D
:109308000E02F3501D2618500D02F3501D26195059
:109318000C02F3501D2610501A240A6E11501B20FF
:109328000B6E12501C200C6E13501D200D6E120077
:10933800000E0001E46F0A0EE36F000EE26F050EE7
:10934800E16F77D0E46B140EE36F6BD02F0E0B6ECA
:10935800FC0E0C6EBFEC5EF082B204D00001E46B30
:109368001E0EE36F090E0001E06F1E0EDF6FE40EA4
:10937800E82EFED7DF2FFCD7E02FFAD7000051D018
:10938800A80E0B6EFE0E0C6EBFEC5EF0000E000118
:10939800A16F050EA26F2C0EA36FF90EA46FA56B1B
:1093A8008DEC55F07B6E7B501AEC5BF07B50DAE16C
:1093B8000001E46B230ED5D7ED0E0B6EFD0E0C6E7F
:1093C800BFEC5EF0000E0001B96F030EBA6FDC0E41
:1093D800BB6F010EBC6F010EBD6F56EC11F07B6EBA
:1093E8007B501AEC5BF07B5009E19CEC22F0000EFC
:1093F800526E030E536EDBEC5DF07B6E7B501AEC05
:109408005BF0010CE3C0DFF0E4C0E0F0E05109E1FB
:10941800DF510A0A97E01E0A99E00A0AB1E03D0AFC
:10942800CBE0140E0001E319E41103E0E107D8A032
:10943800E207E2BF000CE251E5E1E105E3E2000CDE
:10944800898E89800001CE6BCF6BB7EC57F0A6C030
:10945800D0F0A7C0D1F0040E0001D15D07E3000EE3
:10946800D025CE6FFC0ED121CF6F04D0D0C0CEF066
:10947800D1C0CFF001015B5135E0385139113A11B3
:109488003B1130E079500C0D040EF324D96E010E17
:10949800F420DA6E38C1C6F039C1C7F03AC1C8F055
:1094A8000001C56B000EC525C96F010EC621CA6F24
:1094B800000EC721CB6F000EC821CC6FDE50C91932
:1094C80011E1DE50CA190EE1DE50CB190BE1DE5076
:1094D800CC1908E1000E216E040E226E01015B51C9
:1094E8001CEC56F082B415D07950220D000EF324EE
:1094F800706E030EF420716E000E726E040E736EA1
:10950800010E756E746ACE0E766E51EC0BF000018A
:10951800CD6F0001CD5109E0240E806FFD0E816FE3
:10952800CDC082F0836BDAEC5FF07BEC20F0536BFC
:109538008990899E8D0E0001806FFC0E816FCFCFC0
:1095480082F0836BCECF84F0856BDAEF5FF07950D1
:109558001E0D070EF324D96E020EF420DA6EDECF4C
:10956800DBF0DECFDCF0DECFDDF0DECFDEF0DECF0D
:10957800DFF0DECFE0F0DECFE1F0DECFE2F0DBC0FF
:109588000AF0DCC00BF0DDC00CF0DEC00DF0DFC06F
:109598000EF0E0C00FF0E1C010F0E2C011F0795019
:1095A8001E0D1C0EF324D96E020EF420DA6EDECFE7
:1095B800E3F0DDCFE4F0E3C012F0E4C013F0146A86
:1095C800156A166A176A186A196AE9EC4FF00AC030
:1095D800E5F00BC0E6F00CC0E7F00DC0E8F00EC0F7
:1095E800E9F00FC0EAF010C0EBF011C0ECF0E5C0F4
:1095F800EDF0E6C0EEF0E7C0EFF0E8C0F0F031ECD7
:109608003DF0F36FF35102E0F351120082B415D02C
:109618007950220D000EF324706E030EF420716E43
:10962800000E726E040E736E010E756E746AF10E82
:10963800766E51EC0BF00001F46FF4510CE0240E3F
:10964800806FFD0E816FF4C082F0836BDAEC5FF0FF
:109658000001F4511200B4EC4BF0000C36C023F0BA
:1096680037C024F00CEC43F0000901E0010C36C0CF
:109678000AF037C00BF038C00CF039C00DF03AC012
:109688000EF03BC00FF012EC49F00AC040F00BC0DE
:1096980041F00CC042F00DC043F020EE2BF03650E4
:1096A800D9263750DA2240C0DEFF41C0DEFF42C073
:1096B800DEFF43C0DEFF2F0E36240A6E000E372071
:1096C8000B6E0D6A0C6A020E0F6E0E6A49EC5FF0A3
:1096D8002F0E36243E6E000E37203F6E456A010E6F
:1096E800446E466A476A04D044504626455047228D
:1096F80020EE09F03650D9263750DA22DE50465C83
:10970800DE5047581FE23EC019F03FC01AF04650DD
:1097180040241B6E475041201C6E000E42201D6ED7
:10972800000E43201E6E44C01FF045C020F020EEFE
:1097380001F03650D9263750DA22DF5098EC4EF037
:109748000009D2E020EE09F03650D9263750DA2247
:109758004650DE1803E14750DE18D8A4010C000C6F
:1097680079501E0D070EF324D96E020EF420DA6E1E
:10977800DECFB2F0DECFB3F0DECFB4F0DECFB5F09F
:10978800DECFB6F0DECFB7F0DECFB8F0DECFB9F07F
:1097980079501E0D1C0EF324D96E020EF420DA6ED9
:1097A800DECFBAF0DDCFBBF0BA51B225BC6FBB51EA
:1097B800B321BD6F000EB421BE6F000EB521BF6F7F
:1097C800000EB621C06F000EB721C16F000EB82180
:1097D800C26F000EB921C36F79501E0D070EF32416
:1097E800D96E020EF420DA6EBCC0DEFFBDC0DEFF0B
:1097F800BEC0DEFFBFC0DEFFC0C0DEFFC1C0DEFFEF
:10980800C2C0DEFFC3C0DEFF79501E0D070EF32471
:10981800D96E020EF420DA6EDECFC4F0DECFC5F0CA
:10982800DECFC6F0DECFC7F07950220D000EF3244C
:10983800706E030EF420716EC4C072F0C5C073F070
:10984800C6C074F0C7C075F088EC0EF0C86FC85178
:1098580003E0010E786E010C786A120020EE03F026
:109868004150D9264250DA22DF6A20EE2BF04150CF
:10987800D9264250DA22DE68DE68DE68DD6841C03B
:1098880036F042C037F043C038F044C039F045C024
:109898003AF046C03BF017EC54F0000904E0426A85
:1098A800040E416E040C2D0E41240A6E020E422055
:1098B8000B6E49EC5EF0550E0A1803E1AA0E0B1860
:1098C80004E0426A030E416E030C20EE2FF0415073
:1098D800D9264250DA22E90EDE1812E020EE2FF0E7
:1098E8004150D9264250DA22EB0EDE1809E020EE6C
:1098F8002FF04150D9264250DA22E80EDE1827E12F
:10990800650E41240A6E000E42200B6ED30E0C6EBB
:10991800FF0E0D6E0F6A030E0E6E8CEC59F00A5096
:109928000B1003E1416A426A1200810E41240A6E5B
:10993800000E42200B6E8E0E0C6EFF0E0D6E0F6A1F
:10994800050E0E6E8CEC59F00A500B10EBE0426AD3
:10995800020E416E020C760EF66E8C0EF76E000E3D
:10996800F86E09EE2FF011EE2CF00900F5CFEEFF9E
:10997800E550E150FAE1E250F8E1280EF66EB80E33
:10998800F76E000EF86E03EEAAF010EE4CF0090028
:10999800F5CFEEFFE550E150FAE1BE0EF66EB80ED7
:1099A800F76E000EF86E02EE78F010EE48F009003F
:1099B800F5CFEEFFE550E150FAE1280EF66EBD0E48
:1099C800F76E000EF86E01EEC6F010EE2BF00900EF
:1099D800F5CFEEFFE550E150FAE18A0EF66EC00EC3
:1099E800F76E000EF86E0900F5CF7CF005EE00F07A
:1099F80014EE2FF0EE6AE550E150FCE1E250FAE196
:109A080004EE00F011EE00F0EE6AE550E150FCE1E2
:109A1800E250FAE103EE00F0AA0EEE6AE806FDE174
:109A280002EE00F0780EEE6AE806FDE101EE00F0C5
:109A38007A0EEE6AE806FDE10001FF6B7B6A7A6A3E
:109A4800796A786A7D907D920001FEEF07F05C6A82
:109A58005F6A8980990E0001806FFA0E816FCFCFFF
:109A680082F0836BCECF84F0856BDAEC5FF019D08F
:109A78005E0E0A6E0B6A8EEC5FF05D6E2C0E0001B6
:109A8800806FFF0E816F5C2A5CC082F0836B5DC0C3
:109A980084F0856BDAEC5FF05EAA03D05DC05FF0FE
:109AA80005D004EC60F00A500B10E2E1140E00013E
:109AB800806FFD0E816F5FC082F0836BDAEC5FF020
:109AC800020E5F183CE17950130DAE0EF324D96EE7
:109AD800030EF420DA6E020EDF6E7950130DBA0E03
:109AE800F324D96E030EF420DA6E080EDF6E795077
:109AF8000D0D7A0EF324D96E020EF420DA6E4C0E98
:109B0800DF6E79500D0D7D0EF324D96E020EF42010
:109B1800DA6E080EDF6E79500D0D820EF324D96EC1
:109B2800020EF420DA6E050EDF6E79500D0D830EED
:109B3800F324D96E020EF420DA6E690EDF6E786AAD
:109B480089901200646E690E0001806FFC0E816FAF
:109B580064C082F0836BAAC084F0ABC085F0DAECF5
:109B68005FF05ED079EC53F0A6C065F0A7C066F050
:109B7800A8C067F0A9C068F0AAC0D9FFABC0DAFFD7
:109B8800DF6A000120EE01F0AA51D926AB51DA2292
:109B980068C0DFFF20EE02F0AA51D926AB51DA22C5
:109BA800DF6A20EE03F0AA51D926AB51DA2267C04A
:109BB800DFFF20EE04F0AA51D926AB51DA22DF6A82
:109BC80020EE05F0AA51D926AB51DA2266C0DFFF94
:109BD80020EE06F0AA51D926AB51DA22DF6A20EE30
:109BE80007F0AA51D926AB51DA2265C0DFFF12006F
:109BF80079EC53F0A6C065F0A7C066F0A8C067F07E
:109C0800A9C068F0AAC017F0ABC018F065C019F079
:109C180066C01AF067C01BF068C01CF084EF48F0FB
:109C28006450626E636A6350D8A412006250010ADD
:109C380099E0030ADDE012000001CF6B8980898E6C
:109C48006DD0B7EC57F0A6C0CDF0A7C0CEF0040E8B
:109C58000001CE5D03E3010ECF6F03D0D2C0D0F078
:109C6800D16B82B415D07950220D000EF324706E9A
:109C7800030EF420716E000E726E040E736E010EE8
:109C8800756E746AD00E766E51EC0BF00001D26FCF
:109C9800D25109E0240E806FFD0E816FD2C082F090
:109CA800836BDAEC5FF001015B5135E03851391113
:109CB8003A113B1130E079500C0D040EF324D96EA3
:109CC800010EF420DA6E38C1C6F039C1C7F03AC1C6
:109CD800C8F00001C56B000EC525C96F010EC6216D
:109CE800CA6F000EC721CB6F000EC821CC6FDE50A3
:109CF800C91911E1DE50CA190EE1DE50CB190BE18A
:109D0800DE50CC1908E1000E216E040E226E01010E
:109D18005B511CEC56F07BEC20F0536B0001CF51EB
:109D280090E0899E89901200226E2250D8A4040CDB
:109D38001F50201001E1040C7CB0030C7CB4020C11
:109D48007AB608D0090ED8901B361C361D361E363A
:109D5800E82EF9D71F0420101AE11BC013F01CC00D
:109D680014F01DC015F01EC016F0180EF7EC5DF0CB
:109D7800000945E119C00CF01AC00DF0FE0E0E6E78
:109D880070EC5BF000093BE01F6A206A38D07AC0AB
:109D980021F0060E211609E01FC013F020C014F0B0
:109DA800156A166A970EF7EC5DF01BC013F01CC01D
:109DB80014F01DC015F01EC016F0190EF7EC5DF07A
:109DC80000091DE119C00CF01AC00DF0FC0E0E6E52
:109DD80070EC5BF0000908E0020E1A261F06D8A0F6
:109DE80020061F502010EEE10C6A0D6AFD0E0E6E63
:109DF80070EC5BF0000903E1206A010E1F6E31EC84
:109E080060F01F502010D8A4010C000CA5C0D9FF89
:109E1800A6C0DAFFDECFA9F0DDCFAAF0A5C05BF0BF
:109E2800A6C05CF0000E5D6E5E6E5F6E606ED2EC7A
:109E380031F00001AD6FAD5153E1AB6BAC6BA9C014
:109E480036F0AAC037F020EE16F0A551D926A65153
:109E5800DA22DECF38F0DECF39F0DECF3AF0DECFCF
:109E68003BF017EC54F00001AD6FAD5139E120EE35
:109E78001AF0A551D926A651DA22DECF75F0DDCF2A
:109E880076F075C0D9FF76C0DAFFE50EDE1810E06F
:109E980020EE1AF0A551D926A651DA22DECF75F0A8
:109EA800DDCF76F075C0D9FF76C0DAFFDF5009E163
:109EB800AB4BAC2BA751AB1906E1A851AC1910E07C
:109EC80002D0AB6BAC6BA5C070F0A6C071F0736A22
:109ED800010E726E38EC30F00001AD6FAD51AFE09D
:109EE800040EAD1902E1070EAD6FAD511200969444
:109EF80096929690929A110E0F6E3C0E0E6ECB0EA5
:109F0800E82EFED70E2EFCD70F2EFAD70000110E22
:109F18000F6E3C0E0E6ECB0EE82EFED70E2EFCD723
:109F28000F2EFAD70000020E0F6EA00E0E6E920EC4
:109F3800E82EFED70E2EFCD70F2EFAD700D0000E33
:109F48000A6E300EECEC5BF02A0E0E6E8E0EE82ECA
:109F5800FED70E2EFCD7000E0A6E300EECEC5BF02E
:109F6800000E0A6E300EECEC5BF0000E0A6E390E35
:109F7800ECEC5BF0000E0A6E140EECEC5BF0000EDD
:109F88000A6E560EECEC5BF0000E0A6E6D0EECECF1
:109F98005BF0000E0A6E700EECEC5BF0000E0A6EC1
:109FA8000C0EECEC5BF0000E0A6E060EECEC5BF0AF
:109FB800000E0A6E010EECEC5BF0D00E0E6ECA0EAF
:109FC800E82EFED70E2EFCD712001A6A1B6A1C6AEE
:109FD8001D6A1E6A1F6A206A216A12501310141023
:109FE8001510161017101810191045E0010E226EE2
:109FF8000AD0D89012361336143615361636173658
:10A0080018361936222A19AEF4D7D8901A361B36C4
:10A018001C361D361E361F362036213612500A5C75
:10A0280013500B5814500C5815500D5816500E5804
:10A0380017500F58185010581950115811E3125052
:10A048000A5E13500B5A14500C5A15500D5A1650DC
:10A058000E5A17500F5A1850105A1950115A1A8080
:10A06800D890193218321732163215321432133288
:10A078001232222ECAD71AC00AF01BC00BF01CC01D
:10A088000CF01DC00DF01EC00EF01FC00FF020C058
:10A0980010F021C011F01200898E8980716A726AED
:10A0A800736A746A7950220D000EF3245B6E030EF6
:10A0B800F4205C6E2F0E5D6E070E5E6E010E606EF4
:10A0C8005F6A750E616E5DEC19F0706E01015B518F
:10A0D80035E0385139113A113B1130E079500C0D07
:10A0E800040EF324D96E010EF420DA6E38C1B1F0F3
:10A0F80039C1B2F03AC1B3F00001B06B000EB0251F
:10A10800B46F010EB121B56F000EB221B66F000E0B
:10A11800B321B76FDE50B41911E1DE50B5190EE165
:10A12800DE50B6190BE1DE50B71908E12F0EAA6F01
:10A13800070EAB6F01015B51A6EC4DF00392755011
:10A14800D5EC55F06E6E6F6A6E5071266F507222A4
:10A15800000E732274220101536B899E89901200AC
:10A16800AEC0D9FFAFC0DAFFDECFB0F0DDCFB1F0BF
:10A17800AEC0A5F0AFC0A6F0000EA86F010EA76F85
:10A188000AEC4FF0B26FB25147E1B0C036F0B1C03F
:10A1980037F020EE16F0AE51D926AF51DA22DECFD5
:10A1A80038F0DECF39F0DECF3AF0DECF3BF017ECF7
:10A1B80054F00001B26FB2512FE120EE1AF0AE5107
:10A1C800D926AF51DA22DECF0AF0DDCF0BF00D6AC7
:10A1D8000C6A0F6A200E0E6E49EC5FF0000120EE4B
:10A1E8001AF0AE51D926AF51DA22DECF0AF0DDCF10
:10A1F8000BF01C0EAE250C6E000EAF210D6E0F6A13
:10A208000B0E0E6EA4EC5CF020EE03F0B051D926D4
:10A21800B151DA22010EDF6EB25112000101556B05
:10A22800546B406B416B020E536F8990526B516BAC
:10A23800796A030E796401D049D079500C0D030E68
:10A24800F324D96E010EF420DA6EDF6A79500C0D12
:10A25800020EF324D96E010EF420DA6EDF6A79500B
:10A268000C0D000EF324D96E010EF420DA6EDE6AAE
:10A27800DD6A79500C0D040EF324D96E010EF4201A
:10A28800DA6EDE6ADE6ADE6ADD6A79500C0D0B0E64
:10A29800F324D96E010EF420DA6E100EDF6E7950B9
:10A2A8000C0D0A0EF324D96E010EF420DA6E020E9C
:10A2B800DF6E79500C0D080EF324D96E010EF420D0
:10A2C800DA6E240EDE6EDD6A792AB3D7796A010167
:10A2D800506B12008980898E000E0A6E040E0B6E78
:10A2E8000D6A0C68010E0F6E0E6AAAEC5EF00B0E7A
:10A2F8000001806FFE0E816FDAEC5FF00001B56B34
:10A30800B66BB5C077F0010E771677327732895081
:10A3180077187F0B7718896E2E0E1CEC60F082B4CC
:10A3280015D07950220D000EF324706E030EF42020
:10A33800716E000E726E040E736E010E756E746A85
:10A34800B20E766E51EC0BF00001B46F0001B451FF
:10A3580009E0720E806FFF0E816FB4C082F0836BCC
:10A36800DAEF5FF0B54BB62BB6BFCBD7B65103E1EA
:10A378000A0EB55DC6E3180E806FFF0E816FDAEC2A
:10A388005FF0899E89908990786A12000F6A106A36
:10A398000E6A01D00A2A0A50D96EDA6A200EDE182F
:10A3A800F9E00A50D96EDA6ADF500C6EF70E0C2607
:10A3B800040E0C64EFD70A50D96EDA6A2D0EDE1837
:10A3C80004E1010E0E6E0A2A1ED00A50D96EDA6A0E
:10A3D8002B0EDE18F8E017D00A0E0F02F3CF0CF0A0
:10A3E800F4CF0DF01002F3500D260A50D96EDA6A38
:10A3F800DF500C5E000E0D5A300E0C240F6E000E4E
:10A408000D20106EE0D70A50D96EDA6ADF500C6E54
:10A41800D00E0C26090E0C64DFD70E500DE10FC0CC
:10A428000CF010C00DF00C1E0D1E0C4A0D2A0CC0AD
:10A438000AF00DC00BF012000FC00AF010C00BF0AC
:10A4480012000600F2A011D00101652B81A802D0EC
:10A4580089A206D0939403AE02D0939201D093823E
:10A4680081B889B201D09384F290F2A23FD0010161
:10A47800642B81B889B29392831C056E811C066E89
:10A48800038E350EE82EFED70000938481A0FED7F8
:10A4980081A802D089A202D0939401D0938406A8FF
:10A4A80022D005507F0B096E0101DB1902E1898278
:10A4B80005D0DA51091809E1898405D0899413D0A7
:10A4C80089A211D0899489920ED00950076E086A22
:10A4D800085009E10750040AF3E0100AF1E02B0ADA
:10A4E800F2E0600AEBE09392F292F288F28C7D92AD
:10A4F8001100090E146E0B500C103BE00BC0D9FF75
:10A508000CC0DAFFDE50DE1034E00BC0D9FF0CC0FF
:10A51800DAFFDECF0EF0DDCF0FF00EC0D9FF0FC08F
:10A52800DAFFDF5026E00BC0D9FF0CC0DAFF10EECF
:10A5380005F0DE50E126DD50E22220EE02F00B505D
:10A54800D9260C50DA22E650DE1813E1E650DE1860
:10A5580010E10BC0D9FF0CC0DAFF10EE01F0DE509D
:10A56800E126DD50E222E7502BEC60F00E6E0EA0E3
:10A57800146A145003E0126A136A08D00BC0D9FF9A
:10A588000CC0DAFFDECF12F0DDCF13F00D50D96E1C
:10A59800DA6A12C0DEFF13C0DDFF1450120020EE8D
:10A5A80003F00A50D9260B50DA22DF50126E136AD4
:10A5B800146A156A20EE02F00A50D9260B50DA22E6
:10A5C800DF5012C00FF013C010F014C011F00E6A63
:10A5D8000E10126E0F50136E1050146E1150156E2F
:10A5E80020EE01F00A50D9260B50DA22DF5012C0B3
:10A5F8000FF013C010F014C011F00E6A0E10126E96
:10A608000F50136E1050146E1150156E0AC0D9FFFA
:10A618000BC0DAFFDF5012C00FF013C010F014C0E7
:10A6280011F00E6A0E10126E0F50136E1050146E49
:10A638001150156E12C00AF013C00BF014C00CF0C4
:10A6480015C00DF01200216E2150D8A4040C1F5023
:10A65800201001E1040C7CB0030C7AB608D0090E76
:10A66800D8901B361C361D361E36E82EF9D72050DA
:10A6780006E1020E1F5C03E2236A110E02D0236A70
:10A68800120E226E22C024F01BC013F01CC014F05E
:10A698001DC015F01EC016F02450F7EC5DF000093F
:10A6A8001DE119C00AF01AC00BF0020E0D6E0C6AFB
:10A6B800BEEC5AF0000908E0020E1A261F06D8A0C0
:10A6C80020061F502010EDE1120E241807E1136A2E
:10A6D800146A156A166A0C0EF7EC5DF031EC60F03E
:10A6E8001F502010D8A4010C000C13EC5EF0CC0E07
:10A6F8009CEC5FF0660E9CEC5FF07FEC5FF05E6EAA
:10A708005E5006E10001A66BA76BA86BA96B12004F
:10A718005C6A5D6A5C505E0FD96EDA6A7FEC5FF046
:10A72800DF6E5C4A5D2A5DBEF5D75D5003E1040E1D
:10A738005C5CF0E3060E0001806FFC0E816F5EC06A
:10A7480082F0836B5FC084F0856B60C086F0876B96
:10A7580061C088F0896B5EC08AF05FC08BF060C012
:10A768008CF061C08DF0DAEC5FF0615060105F1022
:10A7780003E1060E5E5CC6E35EC0A6F05FC0A7F00C
:10A7880060C0A8F061C0A9F01200156A0B0E146E23
:10A79800070E1426136A1450D96EDA6ADF50166E43
:10A7A800163A0F0E1616161616500CE0C60E16247C
:10A7B800D96EDA6A010EDA22DF501CEC60F0010E65
:10A7C800156E0BD0150409E1C60E1624D96EDA6A87
:10A7D800010EDA22DF501CEC60F01450D96EDA6AF0
:10A7E800DF50166E0F0E161616500CE0C60E162405
:10A7F800D96EDA6A010EDA22DF501CEC60F0010E25
:10A80800156E0BD0150409E1C60E1624D96EDA6A46
:10A81800010EDA22DF501CEC60F01406132A070E32
:10A828001364B9D7070C406A20EE2BF03650D926AE
:10A838003750DA223850DE1809E13950DE1806E1BF
:10A848003A50DE1803E13B50DE1839E036C023F0F9
:10A8580037C024F00CEC43F0406E405030E12F0E2E
:10A868003624196E000E37201A6E38C01BF039C016
:10A878001CF03AC01DF03BC01EF0206A010E1F6E8E
:10A8880020EE01F03650D9263750DA22DF5027EC77
:10A8980053F0000906E0386839683A683B68010EE9
:10A8A800406E20EE2BF03650D9263750DA2238C0C9
:10A8B800DEFF39C0DEFF3AC0DEFF3BC0DEFF40509E
:10A8C800120000019B6B9C6B6EC09DF06FC09EF0E8
:10A8D8007006D8A0710627D072C05BF073C05CF018
:10A8E800970E5D6E5E6A606A010E5F6E9F0E616E06
:10A8F8005DEC19F000019F05A0111EE19751A16FB1
:10A90800A26BA36BA46B9DC0D9FF9EC0DAFFA1C048
:10A91800DFFF9D4B9E2B9B4B9C2B0A0EA119A2116E
:10A92800A311A41109E070509B5D9C51800A746EBC
:10A938007150800A7458D0E39DC0D9FF9EC0DAFFD9
:10A94800DF6A9B519C1103E16E6A6F6A12006EC048
:10A958006EF06FC06FF0120003D00A4A0B2A0C2A5F
:10A968000C50D96EDA6ADF500D6E0AC0F6FF0BC0C4
:10A97800F7FF000EF86E0F0EF76403D00800F550CD
:10A9880005D0F6CFE9FFF7CFEAFFEF500D1813E136
:10A998000AC0F6FF0BC0F7FF000EF86E0F0EF76443
:10A9A80003D00800F55005D0F6CFE9FFF7CFEAFF4E
:10A9B800EF500009D2E10AC0F6FF0BC0F7FF000E06
:10A9C800F86E0F0EF76403D00800F55005D0F6CFE7
:10A9D800E9FFF7CFEAFFEF500D6E0C50D96EDA6A37
:10A9E800DF500D5C0A6E0B6AD8A00B0612000382BA
:10A9F800040E796033D02F0E0A6E070E0B6E795055
:10AA0800050DAC0EF3240C6E020EF4200D6E0F6AC9
:10AA1800050E0E6E83EC5CF0340E0A6E070E0B6E9C
:10AA28007950130DAA0EF3240C6E030EF4200D6E4C
:10AA38000F6A130E0E6E83EC5CF0470E0A6E070E5B
:10AA48000B6E79500D0D780EF3240C6E020EF42067
:10AA58000D6E0F6A0D0E0E6E83EC5CF0030E7964BA
:10AA680009D0010E786E02011B5110091B6F000EF0
:10AA7800E8CF30F7250ED5EC55F0039289901200F7
:10AA8800135014100AE13CC113F03DC114F01350E7
:10AA9800141003E1136A146A120013C00EF014C0F4
:10AAA8000FF015C010F0E6EC5CF00E5013260F50B6
:10AAB800142213C0D9FF14C0DAFFDF5006E10101E8
:10AAC8003C6B3D6B136A146A120013C00EF014C07D
:10AAD8000FF015C010F006EC5DF00E5013240101C4
:10AAE8003C6F0F5014203D6F3CC1D9FF3DC1DAFFC8
:10AAF800DF5008E03CC1D9FF3DC1DAFFDF6A3C4BBB
:10AB08003D2B02D03C6B3D6B13C013F014C014F006
:10AB18001200A3C0A7F0A4C0A8F0A70E0A6E08EC04
:10AB280045F00AC0ABF00BC0ACF00001ACBF0B0C99
:10AB3800D890AB35D96EAC35DA6E480ED926010EF1
:10AB4800DA22DECFA9F0DDCFAAF0A951AA1105E0DB
:10AB5800A9C0D9FFAAC0DAFFDF6AA151A21105E096
:10AB6800A1C0D9FFA2C0DAFFDF6AD890AB35D96E91
:10AB7800AC35DA6E480ED926010EDA22A1C0DEFF06
:10AB8800A2C0DDFFA55101E1000CA30E646EA10E69
:10AB9800656E666A676A09EC00F00001A66FA65147
:10ABA8001200026E07EE2FF08A908A9A0F01F2992E
:10ABB800F297F29E89A4FED7936881A8FED781A850
:10ABC8001DD0020426E0EE508C6E8C1E956A81A87A
:10ABD80015D081A2FCD781A2FAD7939081A80ED074
:10ABE80081B2FCD781A4FED79380938A81A806D02E
:10ABF80081B4FCD781A802D0022EE1D79568F90E5E
:10AC0800936E0F01F293F291F289F287F28E02505D
:10AC1800120081A2FED703B2939AEE508C6E8C1E5E
:10AC2800956ADBD70000EAD70000042EFDD7120092
:10AC3800256E39D020EE01F02150D9262250DA2293
:10AC4800DF50296E20EE03F02150D9262250DA2257
:10AC5800DF50286E20EE05F02150D9262250DA2246
:10AC6800DF50276E20EE07F02150D9262250DA2235
:10AC7800DF50266E26C00DF027C00EF028C00FF05A
:10AC880029C010F09AEF5BF021C00AF022C00BF047
:10AC98001FEC3EF00AC026F00BC027F00CC028F0CD
:10ACA8000DC029F0E7D72550236E246A2450D8A474
:10ACB80012002350010ABEE0030AE6E012001A6AF5
:10ACC8001B6A1C6A1D6A1E6A1F6A206A216A0AA01A
:10ACD80010D012501A2613501B2214501C22155043
:10ACE8001D2216501E2217501F22185020221950BC
:10ACF8002122D890123613361436153616361736E2
:10AD080018361936D890113210320F320E320D32F1
:10AD18000C320B320A320A500B100C100D100E10A8
:10AD28000F1010101110D3E11AC00AF01BC00BF05D
:10AD38001CC00CF01DC00DF01EC00EF01FC00FF09F
:10AD480020C010F021C011F0120017C01AF018C06E
:10AD58001BF035D016C013F01A0E146E19C015F07A
:10AD68001450D96EDA6ADECFF6FFDDCFF7FFF86A46
:10AD7800000EF86E0800F550250A09E101D007D049
:10AD88001450D96EDA6ADE2A000EDD2212D0145071
:10AD9800D96EDA6ADECFF6FFDDCFF7FFF86A000E6C
:10ADA800F86E0800F5500B6E0C6A13C00DF0EEEC4F
:10ADB80056F01450D96EDA6ADE2A000EDD221AC067
:10ADC800F6FF1BC0F7FFF86A0800F550C3E1166AE2
:10ADD800176A12000D5002E00D5003E10B5014EFFA
:10ADE80060F00D50D96EDA6A0A0ED926DE50DE10F0
:10ADF80014E00D50D96EDA6A0A0ED9260D50E16EAC
:10AE0800E26A030EE126DE50E65CE650800A126E26
:10AE1800DE50800A1258D8B012000D50D96EDA6A86
:10AE2800030ED926DECF0EF0DDCF0FF00D50D96E10
:10AE3800DA6ADECF10F0DDCF11F00E501024D96E93
:10AE48000F501120DA6E0BC0DFFF0D50D96EDA6A91
:10AE5800030ED926DE2A000EDD22000C0A500E024F
:10AE6800F3CF12F0F4CF13F0146A156A0A500F02E8
:10AE7800F3501326F4501422000E15220B500E0224
:10AE8800F3501326F4501422000E15220A50100213
:10AE9800F3501426F45015220B500F02F3501426C9
:10AEA800F45015220C500E02F3501426F4501522BB
:10AEB80011500A02F35015260B501002F3501526B4
:10AEC8000C500F02F35015260D500E02F3501526A4
:10AED80012C00AF013C00BF014C00CF015C00DF02E
:10AEE80012000E06D8A00F060E280CE10F280AE162
:10AEF8000A6A0B6A12000A4A0B2A0C4A0D2A0E0625
:10AF0800D8A00F060AC0F6FF0BC0F7FFF86A0800C2
:10AF1800F55016E00CC0D9FF0DC0DAFFDF5010E085
:10AF28000E500F100DE00CC0D9FF0DC0DAFF0AC09B
:10AF3800F6FF0BC0F7FFF86ADE500900F518DBE0F2
:10AF48000AC0F6FF0BC0F7FFF86A0800F5CF10F04B
:10AF58000CC0D9FF0DC0DAFFDF50105C0A6E0B6A17
:10AF6800D8A00B0612005D6A5E6A0101636B5F6A16
:10AF780031D004EC60F00A500B1020E05F0E0A6E2E
:10AF88000B6A8EEC5FF05C6E5FA80CD0CC0E0001F3
:10AF9800806FFE0E816F5CC082F0836BDAEC5FF02D
:10AFA80089900CD0000E01016325D96EDA6A040E6F
:10AFB800DA225CC0DFFF632B5D4A5E2A5FAA08D0F5
:10AFC800000E5D240001A66F040E5E20A76F12001C
:10AFD80081AC02D05E04CDE35DC0A6F05EC0A7F0F0
:10AFE80012000C6E610EF66EF80EF76EF86A090024
:10AFF800F5500C5C31E3620EF66EF80EF76EF86AE7
:10B008000C500900F55C04E30B6A010E0A6E010C92
:10B01800630EF66EF80EF76EF86A0900F5500C5CD0
:10B0280009E3640EF66EF80EF76EF86A0C50090024
:10B03800F55CEAE2650EF66EF80EF76EF86A09003E
:10B04800F5500C5C09E3660EF66EF80EF76EF86ABA
:10B058000C500900F55CD8E20A6A0B6A1200150E5A
:10B06800106EC60EE82EFED7102EFCD700D020D0CA
:10B07800150E106EC60EE82EFED7102EFCD700D087
:10B08800010E0A6E0EC0F6FF0FC0F7FF000EF86E35
:10B098000F0EF76403D00800F55005D0F6CFE9FF8E
:10B0A800F7CFEAFFEF50ECEC5BF00E4A0F2AD7D748
:10B0B8000EC0F6FF0FC0F7FF000EF86E0F0EF76414
:10B0C80003D00800F55005D0F6CFE9FFF7CFEAFF27
:10B0D800EF500009CDE11200126A136A146A156A6A
:10B0E8000E500F101010111029E0010E166E06D028
:10B0F800D8900E360F3610361136162A11AEF8D7FC
:10B10800D89012361336143615360E500A5C0F5086
:10B118000B5810500C5811500D5809E30E500A5E88
:10B128000F500B5A10500C5A11500D5A1280D890CB
:10B13800113210320F320E32162EE2D712C00AF038
:10B1480013C00BF014C00CF015C00DF012001A0E4D
:10B1580013240A6E000E14200B6E49EC5EF00AC030
:10B1680019F00BC01AF01B6A1C6A11C0D9FF12C073
:10B17800DAFF030EDE181CE1140E13240A6E000E0B
:10B1880014200B6E49EC5EF00A50156E0B50166ECB
:10B19800176A186A16C018F015C017F0166A156AEB
:10B1A8001550191216501A1217501B1218501C124B
:10B1B80019C011F01AC012F01BC013F01CC014F013
:10B1C8001200126E0C0E121807E031EC60F0C2EC9F
:10B1D8005FF0000901E1FF0C12504009FBEC5FF041
:10B1E8000F50FBEC5FF00E50FBEC5FF00D50FBECEA
:10B1F8005FF00C50FBEC5FF0010E116E125002E193
:10B20800950E116E080E121802E1870E116E11507C
:10B21800FBEC5FF00C0E121802E124EC60F00A0E51
:10B22800116E24EC60F0106E10AE02D0112EF9D71A
:10B23800105012000E500F10D8B4000C0EC0D9FFD9
:10B248000FC0DAFFDF5001E1000C0EC00AF00FC09A
:10B258000BF0C5EC5CF00AC010F00BC011F0020E48
:10B268001018111001E0000C120E0A6E0EC0D9FF62
:10B278000FC0DAFFDF50C3EC5BF00009D8B4000C54
:10B28800130E0A6E20EE01F00E50D9260F50DA2266
:10B29800DF50C3EC5BF0000901E1000C1238F00B41
:10B2A800131012008980038250050DE1000EE8CFCB
:10B2B8002FF7500EE8CF30F7000EE8CF31F7E8CF80
:10B2C80032F7506B1DD027EE2FF051C1DFFF000E73
:10B2D800E8CF30F70D0EE8CF31F7000EE8CF32F7A0
:10B2E80082A403D0600EE8CF32F782A406D031C71B
:10B2F8000AF0200E0A120AC031F7010EE8CF33F720
:10B30800050ED5EC55F003920101516B899012009E
:10B318000AC011F00BC012F00CC013F00DC014F0ED
:10B3280011C0D9FF12C0DAFFDF50106E13C0F6FF4C
:10B3380014C0F7FF000EF86E0F0EF76403D0080074
:10B34800F55005D0F6CFE9FFF7CFEAFFEF50105CD4
:10B35800156E166AD8A01606134A142A114A122A1C
:10B368000E06D8A00F060E500F1003E01550161049
:10B37800D7E015C00AF016C00BF012000AC0D9FFBA
:10B388000BC0DAFF0CC0DFFF0A4A0B2A0D500C6E07
:10B398000E500D6E0F500E6E0F6A0AC0D9FF0BC00B
:10B3A800DAFF0CC0DFFF0A4A0B2A0D500C6E0E5054
:10B3B8000D6E0F500E6E0F6A0AC0D9FF0BC0DAFF70
:10B3C8000CC0DFFF0A4A0B2A0D500C6E0E500D6E92
:10B3D8000F500E6E0F6A0AC0D9FF0BC0DAFF0CC0FF
:10B3E800DFFF0A4A0B2A1200796A030E796401D03A
:10B3F8002AD079500C0D030EF324D96E010EF420D7
:10B40800DA6EDF6A79500C0D020EF324D96E010E44
:10B41800F420DA6EDF6A79500C0D000EF324D96E31
:10B42800010EF420DA6EDE6ADD6A79500C0D040E26
:10B43800F324D96E010EF420DA6EDE6ADE6ADE6A63
:10B44800DD6A792AD2D7796A8990536B12008C6A9F
:10B458008A6A956893680101636B039E899289944F
:10B468004E6B4F6B09D0000E4E25D96E040E4F213E
:10B47800DA6EDF6A4E4B4F2B4FBFF5D74F5102E1C3
:10B488004E05F1E34E6B4F6B09D02F0E4E25D96E4A
:10B49800070E4F21DA6EDF6A4E4B4F2B4FBFF5D7A1
:10B4A8004F05F3E3CD929D90CF0ECD16CD8ECD8076
:10B4B800CF0C0E500F101010111023E0010E126E59
:10B4C80006D0D8900E360F3610361136122A11AE25
:10B4D800F8D70E500A5C0F500B5810500C581150EA
:10B4E8000D5808E30E500A5E0F500B5A10500C5AB4
:10B4F80011500D5AD890113210320F320E32122ECE
:10B50800E8D70AC00AF00BC00BF00CC00CF00DC055
:10B518000DF01200796A0A6A0B6A79501E0D070E3F
:10B52800F324D96E020EF420DA6E070EDE6AE806FE
:10B53800FDE279501E0D1B0EF324D96E020EF42085
:10B54800DA6EDF6A79501E0D170EF324D96E020EDB
:10B55800F420DA6EDE6ADE6ADE6ADD6A0A4A0B2ADF
:10B568000BBEDBD70B5003E1040E0A5CD6E38990CF
:10B57800786A1200070E0F6ED00E0E6E0FD024ECF4
:10B5880060F0106E10280DE1E40E00D000D0E82E17
:10B59800FCD700D000D00E06D8A00F060E500F1012
:10B5A800EEE1FE0E101801E0000C24EC60F00AC079
:10B5B800D9FF0BC0DAFFDF6E0A4A0B2A0C06D8A0A7
:10B5C8000D060C500D10F1E124EC60F024EC60F055
:10B5D800010C0C6E5D0EF66EF80EF76E000EF86E2E
:10B5E8000900F5500C5C1FE35E0EF66EF80EF76E60
:10B5F800F86A0C500900F55C04E30B6A010E0A6E48
:10B60800010C5F0EF66EF80EF76EF86A0900F55039
:10B618000C5C09E3600EF66EF80EF76EF86A0C50D3
:10B628000900F55CEAE20A6A0B6A12005D6E690EAF
:10B638005E6EF80E5F6E5C6A0BD05EC0F6FF5FC090
:10B64800F7FF5E4A5F2AF86A0800F550F6E15C2ABF
:10B658005D505C1808E05EC0F6FF5FC0F7FFF86A4F
:10B668000800F550EAE1190E0001806FFE0E816FA7
:10B678005DC082F0836B5EC084F05FC085F0DAEF56
:10B688005FF00AC010F00BC011F013D00E06D8A05E
:10B698000F060CC0D9FF0DC0DAFF0C4A0D2A10C0E6
:10B6A800E1FF11C0E2FF104A112ADFCFE7FFE750A0
:10B6B8000BE00E500F1008E0E9D710C0D9FF11C0F9
:10B6C800DAFFDF6A104A112A0E06D8A00F060E28E4
:10B6D800F4E10F28F2E112002EEC5EF0000901E11E
:10B6E800000C0E50FBEC5FF0FD0E0E181EE0020E73
:10B6F800106E0F6A0CC0D9FF0DC0DAFFDF50FBECEB
:10B708005FF00C4A0D2A0F06D8A010060F50101033
:10B71800F1E124EC60F024EC60F024EC60F0116EB0
:10B7280011501F0B050A01E0000C010C0DC011F0AF
:10B738000EC012F00FC013F010C014F013EC5EF03E
:10B74800CC0E9CEC5FF0990E9CEC5FF00C0E9CEC20
:10B758005FF0156A166A1550110FD96EDA6ADF5054
:10B768009CEC5FF0154A162A16BEF5D7165002E073
:10B7780013EF5EF0040E155CEEE313EF5EF00B6E54
:10B788000A5001E1000C2F0E0B6409D03A0E0B6031
:10B7980006D00A50D96EDA6A0B50D00F17D0400E77
:10B7A8000B6409D0470E0B6006D00A50D96EDA6ACE
:10B7B8000B50C90F0BD0600E0B64000C670E0B60AA
:10B7C800000C0A50D96EDA6A0B50A90FDF6E010C13
:10B7D8000B6E8D920A0EE82EFED700D00AB002D06A
:10B7E8008D9401D08D84000E0D6E010E0C6E0BAE83
:10B7F80002D0898A01D0899AD8900B368D900000A2
:10B8080000008D80000000008D900C4A0D2A0DBEAE
:10B81800EED70D5003E1090E0C5CE9E38D821200AE
:10B8280001091220010001001700002D119420D0F9
:10B838000F000101091220010001001700002D115D
:10B848009420D00F00010109122001000100170007
:10B85800002D119420D00F000101091220010001D0
:10B86800001700002D119420D00F0001010E0A6E60
:10B878000B6A92868D828D84000000008D940000F2
:10B8880000000C6A0D6A80A602D00A500B12D890EC
:10B898000A368D90000000008D80000000008D9019
:10B8A8000C4A0D2A0DBEEFD70D5003E1030E0C5CB8
:10B8B800EAE30B50120000004F01000F00000000E7
:10B8C80009FF0000004F01000F0000000009FF0001
:10B8D80000004F01000F0000000009FF0000004FAA
:10B8E80001000F0000000009FF00800102E8058048
:10B8F8000102E805800102E805800102E8050CC0A4
:10B9080012F00DC013F00AC010F00BC011F010D0E7
:10B9180012C0D9FF13C0DAFFDF50146E124A132A7F
:10B9280010C0D9FF11C0DAFF14C0DFFF104A112A76
:10B938000E06D8A00F060E28EBE10F28E9E1120049
:10B948000AC010F00BC011F00CC012F00DC013F0BB
:10B958000E500F10D8B4120012C0D9FF13C0DAFF6E
:10B9680010C0E1FF11C0E2FFDFCFE7FF124A132A40
:10B97800104A112A0E06D8A00F060E500F10ECE13F
:10B9880012000AC00CF00BC00DF002D00A4A0B2AB4
:10B998000AC0F6FF0BC0F7FF000EF86E0F0EF76433
:10B9A80003D00800F55005D0F6CFE9FFF7CFEAFF3E
:10B9B800EF500009EBE10C500A5C0A6E0D500B5871
:10B9C8000B6E1200116A126A04D00E4A0F2A114A2D
:10B9D800122A0EC0D9FF0FC0DAFFDF500EE010C0E8
:10B9E8000AF00EC0D9FF0FC0DAFFDF500B6E0C6AE9
:10B9F80036EC5FF00A500B10E8E111C00EF012C0EF
:10BA08000FF01200116A126A04D00E4A0F2A114A66
:10BA1800122A0EC0D9FF0FC0DAFFDF500EE010C0A7
:10BA28000AF00EC0D9FF0FC0DAFFDF500B6E0C6AA8
:10BA380036EC5FF00A500B10E8E011C00EF012C0AF
:10BA48000FF012001A0E10240A6E000E11200B6E51
:10BA580012C00CF013C00DF0E9EC5EF00EC0D9FF77
:10BA68000FC0DAFF030EDE18D8A41200140E10243B
:10BA78000A6E000E11200B6E14C00CF015C00DF0EC
:10BA8800E9EF5EF08980898E000E0A6E040E0B6E57
:10BA98000D6AF60E0C6E010E0F6E0E6AAAEC5EF0C1
:10BAA8000B0E0001806FFE0E816FDAEC5FF0180E4E
:10BAB8000001806FFF0E816FDAEC5FF0899E89903C
:10BAC800120002D00A4A0B2A0AC0F6FF0BC0F7FF81
:10BAD800F86A0800F5500AE00AC0F6FF0BC0F7FF45
:10BAE800F86A0800F5500C180D10ECE10AC0F6FFD2
:10BAF8000BC0F7FFF86A0800F5500A6E0B6A1200CF
:10BB08000A6E0A500EE038EC60F0200EE82EFED7E0
:10BB18003BEC60F0CC0E00D0E82EFDD700D000D072
:10BB2800120038EC60F0C00E00D0E82EFDD73BECD8
:10BB380060F0350EE82EFED700001200000EF2BEAF
:10BB4800010E0D6E0B50030BAA6E0AC0A9FF0CC0A4
:10BB5800A8FFA69EA69CA684F29E550EA76EAA0EC6
:10BB6800A76EA682A6B2FED7A6940DB002D0F29E0A
:10BB780001D0F28E1200200E206E1CC021F01DC0D4
:10BB880022F0246A256A2B6A2C6A210E166E1EC0C2
:10BB980017F01FC018F0200E196EA9EC56F02450AB
:10BBA8001C24D96E25501D20DA6EDF6A120052C09F
:10BBB8004BF053C04CF067EC44F0566E565011E110
:10BBC80052C00BF053C00CF0540E0D6E7DEC52F0C9
:10BBD800566E565006E152C0D9FF53C0DAFFDE6AEE
:10BBE800DD6A56501200176E17AE0ED0179E0C6AFB
:10BBF8000D6A0E6A0F6A370EE5EC58F0186E010EE2
:10BC0800186402D01850120013C00CF014C00DF0C4
:10BC180015C00EF016C00FF01750E5EF58F038ECCD
:10BC280060F00A0E0B6EF80EE82EFED70B2EFCD72E
:10BC380000D03BEC60F0E00E00D0E82EFDD7F2EC2F
:10BC48005FF0090E0B6E840EE82EFED70B2EFCD784
:10BC58003BEF60F0130E0B6E880E0A6E0ED024ECCC
:10BC680060F0FF0A0DE0E40E00D000D0E82EFCD70B
:10BC780000D000D00A06D8A00B060A500B10EFE13E
:10BC88000A500B10D8A4010C000C20EE01F00A5049
:10BC9800D9260B50DA22DF500F6E106A0AC0D9FF7E
:10BCA8000BC0DAFFDF500C6E0F500D6E0C500F6E8C
:10BCB8000DC010F00FC00AF010C00BF012005BC0EE
:10BCC8003EF15CC03FF15F0E616E176A186A5DC095
:10BCD80019F05EC01AF0610E1B6EBDEC16F03EC185
:10BCE800D9FF3FC1DAFFDF6A01013E6B3F6B1200EB
:10BCF8002F0E0A6E070E0B6E0D6A0C6A010E0F6E80
:10BD08000E6AAAEC5EF0038227EE2FF053C1DFFF24
:10BD18000392010ED5EC55F089800101536B120096
:10BD28003031323334353637383941424344454669
:10BD38002F071F60402068706469736B2E63666705
:0BBD4800004850393132314400000047
:10BD54000AC010F00BC011F008D010C0D9FF11C0F8
:10BD6400DAFF0CC0DFFF104A112A0E06D8A00F0616
:10BD74000E28F3E10F28F1E112000BD00BC0F6FFFF
:10BD84000CC0F7FFF86A0800F5501CEC60F00B4A91
:10BD94000C2A0BC0F6FF0CC0F7FFF86A0800F55038
:10BDA400EDE112000F6A110E0E6E09D00A0EE82E94
:10BDB400FED700D0010E0A6E200EECEC5BF00E06EE
:10BDC400D8A00F060E28F2E10F28F0E112000AC0F5
:10BDD400D9FF0BC0DAFF0CC0DFFF0A4A0B2A0DC0E3
:10BDE4000CF00D6A0AC0D9FF0BC0DAFF0CC0DFFFEC
:10BDF4000A4A0B2A1200B886AC84B898440EAF6E77
:10BE0400B06AAC98AB8EAB88AB9A9D989D9A9F8A8A
:10BE1400F28EAC90AB9CAC9AAC8A120038EC60F019
:10BE2400200EE82EFED73BEC60F0300EE82EFED755
:10BE3400F2EC5FF00B6EB00E00D0E82EFDD70B5085
:10BE440012002F0E0A6E070E0B6E0D6A0C6A010E9D
:10BE54000F6E0E6AAAEC5EF0010EE8CF2FF7038294
:10BE6400D5EC55F0039212000A50D96EDA6A0B50E1
:10BE7400DE1804E10AC00AF00B6A12000A2A0A0456
:10BE8400D96EDA6ADF50F0E10A6A0B6A12000AC05E
:10BE940010F00BC011F010C0D9FF11C0DAFF0CC0B4
:10BEA400DFFF104A112A0E06D8A00F060E500F10FD
:10BEB400F2E11200070E966E8450070B0A6E928A06
:10BEC40080AA02D0080E0A26020E01015D1903E1C0
:10BED4000A1C0F0B0A6E0A50120001013E513F1159
:10BEE40009E03EC1D9FF3FC1DAFF0DC0DFFF3E4B81
:10BEF4003F2B12000D501CEF60F00C6A0D6AD890B5
:10BF04000C3210EC5FF0000901E00C8E0D2A070ED4
:10BF14000D64F5D70C50120003AEFED7F29E0AC092
:10BF2400D9FF0BC0DAFF06C0DFFF039EF28E9382B7
:10BF3400055012000B6E0C6A0B50010B84EC5DF083
:10BF4400D8900B320C2A070E0C64F6D7070C0A6E35
:10BF54000A5007E0C66A010EC66EC00EC76EC68AD6
:10BF6400C00CC66A020EF8D7020E786E400E0201AB
:10BF74001B6F7E0E0001806FFA0E816FDAEF5FF0A7
:10BF840042EC60F024EC60F02EEC5EF0000901E07D
:10BF9400010C31EC60F0000CC2900F0EC16E4F0E1C
:10BFA400C86E946A948894829482010E826E010C05
:10BFB400820E5B6E176A186A80C019F081C01AF08D
:10BFC4005B0E1B6EBDEF16F00B50030BAA6E0AC07E
:10BFD400A9FFA69EA69CA68000000000A8501200FF
:10BFE400928880A803D0010E0A6E01D00A6A0A5012
:10BFF40012000A6E0AC0C9FFC7B0FED7C7A0FED799
:10C00400C950120003AE9382010E03AE000E0A6EF5
:10C014000B6A12000A6E02D0898C899C0A060A28CF
:10C02400FBE112000A6E01D004009EA8FDD70AC0ED
:10C03400ADFF12000A6E01D004009EA8FDD70AC00D
:10C04400ADFF1200C968C7B0FED7C7A0FED7C9505C
:10C0540012000A6E0A5001E0010C7C50120040EC00
:10C0640060F024EF60F08990536B120089989298E5
:10C074001200899892881200039E12008B8012008D
:07C084008B90120012000175
:10F85C0000819FE0FC407E80FC000020004F4B00AC
:10F86C004449534B5F455252004E4F545F524541F1
:10F87C004459004E4F5F46494C45004E4F545F4F24
:10F88C0050454E4544004E4F545F454E41424C4509
:10F89C0044004E4F5F46494C455F53595354454DB8
:10F8AC0000000D0A202532582025325820253273AD
:10F8BC002025327320253273202532732025327394
:10F8CC002025327320253273202532732025347382
:10F8DC00202534732025347320253473202534736C
:10F8EC0020253473202534732025347320000D0A11
:10F8FC0048504469736B204D6B204949202831389E
:10F90C004634363230292025732025732025732068
:10F91C005374617274696E672E2E2E2558200D0A51
:10F92C00000D0A4461746120706F72742069732039
:10F93C002558202D2053686F756C64206265203C1F
:10F94C003E2030784646000D0A5365656B20657283
:10F95C0072202564203E2025642C202564203E2026
:10F96C0025642C202564203E202564000D0A537448
:10F97C006174757320706F72742069732025582020
:10F98C002D2053686F756C64206265203078464674
:10F99C00000D0A4461746120706F727420697320C9
:10F9AC002558202D2053686F756C642062652030BB
:10F9BC00784646000D0A5264207520256420727426
:10F9CC006E2025642C202564206279746573207266
:10F9DC006561640D0A000D0A2530345820535338E4
:10F9EC0030783A5374617475732C20756E69742079
:10F9FC0025643A20256420000D0A4D617820566557
:10FA0C0063746F72206469736B20256420256C64A9
:10FA1C002028256C582920000D0A44736B73656CE3
:10FA2C002069732025642C206E756D6265722069C7
:10FA3C007320256420000D0A4469736B2063686190
:10FA4C006E67656420746F2025642025303258253C
:10FA5C00303258000D0A426C6F636B73697A652003
:10FA6C00666F72206469736B20256420697320258E
:10FA7C0064000D0A5374617475732073657420747B
:10FA8C006F20706F776572206661696C000D0A25B6
:10FA9C00303258253032582053533830783A466D2E
:10FAAC0074206F70747300466F756E6420616E20E5
:10FABC005254432066696C652061742025580D0AE8
:10FACC00004C6F6F6B696E6720666F7220616E20E1
:10FADC005254432066696C650D0A000D0A55736912
:10FAEC006E67206469736B2067656F6D65747279DE
:10FAFC00202573200046696E6446696C652066613A
:10FB0C00696C6564207365617263680D0A000D0A87
:10FB1C0053746174757320706F727420697320252F
:10FB2C0058202D204F4B000D0A5365656B20746FC8
:10FB3C0020256C64206661696C6564202564000D69
:10FB4C000A57726974655F736563746F72732066AC
:10FB5C0061696C202564000D0A454550524F4D20BB
:10FB6C006469736B206E756D626572202564000D7F
:10FB7C000A4469736B2073656C656374206E756DD4
:10FB8C00626572202564005365656B696E6720742D
:10FB9C006F20736563746F722025580D0A004669D7
:10FBAC006E6446696C65206661696C65642072657B
:10FBBC0061640D0A000D0A4F70656E696E672065F1
:10FBCC0078697374696E6720257320000D0A44618F
:10FBDC00746120706F7274206973202558202D2059
:10FBEC004F4B000D0A476F7420256C7520202D207B
:10FBFC00726573657474696E6700202558202558EA
:10FC0C0020255820255820256C752020200A000D11
:10FC1C000A57726F7465206469736B6E6F3A202596
:10FC2C006420000D0A57616974696E6720666F72F3
:10FC3C00206361726420000D0A54726967706F69E9
:10FC4C006E7420697320256420000D0A46696C656A
:10FC5C00202573206973206F70656E20000D0A7269
:10FC6C0074635F726561642825642C2558290041F2
:10FC7C00646472657373202564202020202020206A
:10FC8C00000D0A25303258253032582045786974D9
:10FC9C00200020436F6C642025582C2025582C20E4
:10FCAC002558004E6F742061204C494620646973BE
:10FCBC006B0D0A000D0A52656164206465736372F2
:10FCCC0069626520000D0A46696C6520255820691B
:10FCDC007320257320000D0A4469736B202558206E
:10FCEC00697320257320000D0A4164647265737377
:10FCFC002069733A202564000D0A487374206279D8
:10FD0C0074657332202564000D0A204F7074696F7E
:10FD1C006E732025640D0A000D0A577269746520F4
:10FD2C006661696C202564000D0A52656164696E18
:10FD3C0067205254430D0A000D0A416D69676F200C
:10FD4C0039313231440D0A000D0A53532F3830200B
:10FD5C0039313232440D0A000D0A44736B73656CF1
:10FD6C0020697320256420000D0A526561642025EA
:10FD7C006420627974657300566563746F722069D0
:10FD8C00732025580D0A000D0A535338307820255E
:10FD9C00642025642000222A2B2C3A3B3C3D3E3F1C
:10FDAC005B5D7C7F000D0A4F70656E696E67202568
:10FDBC00732020000D0A4465627567206973202545
:10FDCC006420000D0A436C6F636B206973202564FB
:10FDDC0020000D0A50726F746F2069732025642007
:10FDEC00000D0A5265616420636F6E6669672000BE
:10FDFC000D0A46696C656E616D6520257320000DDA
:10FE0C000A466F726D617474696E67200072633D8F
:10FE1C0025752046525F25730D0A002A2A204E4F65
:10FE2C00204449534B202A2A002A2A2056657269FD
:10FE3C006679202A2A000D0A736279746573312061
:10FE4C002564000D0A41737365727420454F490097
:10FE5C000D0A4173736572742041544E000D0A4EA5
:10FE6C006F2063617264202564006465736372693A
:10FE7C0062652E636667002F6C6966646174612E1F
:10FE8C0062696E000D0A456E61626C65205050000F
:10FE9C00EB76904558464154202020000D0A4D6FBA
:10FEAC00756E74696E6720004A616E2033312032A2
:10FEBC00303234000D0A4173736572742050500057
:10FECC0020255820772041544E20000D0A476F748E
:10FEDC002041544E31000D0A476F742041544E326C
:10FEEC00000D0A476F742041544E33004C6F61640F
:10FEFC00696E672E2E2E002049442025582530325D
:10FF0C0058002A2A20525141202A2A00466D74207A
:10FF1C006578697420000D0A476F742049464300C8
:10FF2C002025643A20253032580020476F74204138
:10FF3C00544E0031393A35323A3037005B2532585D
:10FF4C002025645D004572726F7220256400485054
:10FF5C004469736B20003C6964656E743E004E6F9F
:10FF6C0020636172640072633D2564200044534B2E
:10FF7C0053454C004E414D452558004449534B25A3
:10FF8C0058004641543332004445425547005052C4
:10FF9C004F544F00526561647900302E3237004166
:10FFAC00444452004946432000454F4920005245E5
:10FFBC004E2000535251200044415620004E4441E3
:10FFCC0043004E52464400464154005254430054A0
:10FFDC00524700434C4B002532580044300044310A
:10FFEC0000443200443300443400443500443600AD
:04FFFC004437000086
:020000040020DA
:08000000FFFFFFFFFFFFFFFF00
:020000040030CA
:0E000000FF06131FFF8181FF0FC00FE00F40AE
:00000001FF
